:020000040800F2
:1080000078EC002049810008319A00088994000822
:1080100019990008CB8F000817AC00080000000079
:1080200000000000000000000000000035A1000872
:10803000E390000800000000E99E0008B1A10008DC
:108040006381000863810008638100086381000880
:108050006381000863810008638100086381000870
:108060006381000863810008638100086381000860
:108070006381000863810008638100086381000850
:108080006381000863810008638100086381000840
:1080900093A300086381000863810008EB91000846
:1080A0006381000863810008638100086381000820
:1080B00029A20008D1A200087DA30008638100085E
:1080C0006381000863810008638100086381000800
:1080D00063810008638100086381000863810008F0
:1080E00063810008638100086381000863810008E0
:1080F00063810008638100086381000863810008D0
:1081000063810008638100086381000863810008BF
:1081100063810008638100086381000863810008AF
:10812000638100086381000863810008638100089F
:10813000DFF810D000F06CF80048004755F8000850
:10814000AFF3008078EC00200648804706480047DF
:10815000FEE7FEE7FEE7FEE7FEE7FEE7FEE7FEE7F7
:10816000FEE7FEE7B9A10008318100080649074A89
:108170000868504343F239021044086040087047D1
:108180000149086070470000900600206D4EC6410E
:1081900010B5431A934209D28318881803E010F8E7
:1081A000011D03F8011D521EF9D210BD40EA010362
:1081B0009B0703D009E008C9121F08C0042AFAD29D
:1081C00003E011F8013B00F8013B521EF9D210BD4B
:1081D000D2B201E000F8012B491EFBD27047002209
:1081E000F6E710B513460A4604461946FFF7F0FFB6
:1081F000204610BD30B504460020034600E05B1C5D
:10820000934203D2E05CCD5C401BF8D030BD00004F
:10821000064C074D06E0E06840F0010394E80700D3
:1082200098471034AC42F6D3FFF786FFAC580108EC
:10823000CC58010870B58C1810F8015B15F00703D5
:1082400001D110F8013B2A1106D110F8012B03E0EF
:1082500010F8016B01F8016B5B1EF9D12B0705D4F7
:108260000023521E0DD401F8013BFAE710F8013B40
:10827000CB1A921C03E013F8015B01F8015B521E5C
:10828000F9D5A142D8D3002070BD00002DE9F041FE
:1082900007460C4615461E461EB980200B4908604D
:1082A00003E04FF4807009490860102229462046F7
:1082B00005F062FB8046102241463846FFF768FF12
:1082C000404606F0D3F9BDE8F081000048060020E2
:1082D0002DE9F04784B01F46DDF830A0914688466E
:1082E000060018BFB8F1000F4AD0002F18BFBAF12E
:1082F000000F45D0B9F1000FA8BF19F00F0F1EBF36
:1083000040F61D4004B0BDE8F087307910F0020F50
:108310001EBF40F61E4004B0BDE8F0870024B9F14E
:10832000100FA8BF6D4625DB5FF0000004EB800155
:1083300058F8011009BA45F82010401C0428F5DB54
:108340006846014606F12802736A00F0BFF84FF054
:10835000000C00BF55F82C0004EB8C0100BA0CF1A6
:10836000010C7850BCF1040FF4DB04F12000103450
:108370004845D9DDCAF8004004B00020BDE8F087C8
:1083800004B04FF44260BDE8F087002812BF002A15
:108390004FF442607047017941F002010171002001
:1083A00010607047032300F04BBD00002DE9F0473B
:1083B00084B01F46DDF830A091468846060018BFFD
:1083C000B8F1000F4AD0002F18BFBAF1000F45D006
:1083D000B9F1000FA8BF19F00F0F1EBF40F61D40E6
:1083E00004B0BDE8F087307910F0020F1EBF40F6F0
:1083F0001E4004B0BDE8F0870024B9F1100FA8BFFB
:108400006D4625DB5FF0000004EB800158F8011099
:1084100009BA45F82010401C0428F5DB68460146DF
:1084200006F12802736A00F0DFF94FF0000C00BF7C
:1084300055F82C0004EB8C0100BA0CF1010C7850BB
:10844000BCF1040FF4DB04F1200010344845D9DD01
:10845000CAF8004004B00020BDE8F08704B04FF433
:108460004260BDE8F087002812BF002A4FF4426046
:108470007047017941F002010171002010607047DE
:10848000022300F0DDBC00002DE9F04180460C46DF
:1084900015461E4600271EB980200B49086003E0E0
:1084A0004FF48070084908602946404605F020FDD9
:1084B0000746102239462046FFF76AFE384606F086
:1084C000D5F8BDE8F0810000480600202DE9F80F3E
:1084D0004FF0030C0CEBE308DB1002EB431202F14C
:1084E0006003BE4A4FF0010CC2F808C0D2F808C0C1
:1084F000D2F800C0CDF800C0BCF1FF3F08D1DDF8D4
:1085000000C0C2F800C012680092002A00F0E680A5
:108510004268D3F804C0006882EA0C071A68424037
:1085200094466446AE483D0E02F0FF0A50F82560BE
:10853000C4F3074550F82AA050F8255004F0FF0B6B
:1085400086EA3526C2F3072550F82BB050F825509F
:10855000A8F101084FEA35490CF0FF0550F8255005
:1085600089EA3565754053F8106CC7F307496E40CA
:108570004FEA1C6550F8299050F8255085EA3925B6
:10858000C4F30729240E50F8299050F824404FEAEC
:10859000394989EA3A6985EA090953F80C5CCCF350
:1085A000074A89EA05054FEA1269C2F30742CCF38C
:1085B000072C50F8299050F82AA050F8222050F8A3
:1085C0002CC089EA3A2984EA3222C7F3072A4FEA03
:1085D0003C4407F0FF0C50F82AA050F82CC04FEA9A
:1085E0003A4A8AEA3B6A84EA3C6C89EA0A0982EAE6
:1085F0000C0253F808AC53F804CC203B89EA0A0972
:1086000082EA0C04B8F1000F7ADD320EC4F3074C95
:1086100050F8222050F82CC0EFB282EA3C22C9F375
:10862000072C50F8277050F82CC009F0FF0A4FEAC9
:108630003C4C8CEA376C82EA0C02D3F800C050F84C
:108640002AA082EA0C072A0E04F0FF0B50F822C081
:10865000C6F3074250F82BB050F822208CEA322C97
:10866000C4F30722240E50F8222050F824404FEA89
:10867000324282EA3A628CEA0202D3F804C0C5F3BD
:10868000074A82EA0C0C4FEA196250F82AA050F807
:108690002220C5F3072582EA3A22C6F3072AC9F346
:1086A0000749F6B250F82AA050F8255050F8299002
:1086B00050F826604FEA3A4A4FEA35458AEA3B6A63
:1086C00084EA392485EA366582EA0A026C40D3F8E6
:1086D00008A0DD6882EA0A026C4024E70268D3F849
:1086E00000C09C6882EA0C074268D3F804C082EAA2
:1086F0000C0C8268C0686240DC68444012E7FFE707
:10870000384850FA85F200EB166C12789CF800C0DD
:10871000C9F3072742EA0C62C4F3074CC75D10F89F
:108720000CC04FEA0C4C4CEA072C42EA0C02D3F87E
:1087300000C082EA0C020A6050FA89F200EB156C64
:1087400012789CF800C0C4F3072742EA0C62C6F313
:10875000074CC75D10F80CC04FEA0C4C4CEA072CD4
:1087600042EA0C02D3F804C082EA0C024A6050FAD2
:1087700084F200EB196C12789CF800C0C6F307274E
:1087800042EA0C62C5F3074CC75D10F80CC04FEA13
:108790000C4C4CEA072C42EA0C02D3F808C082EADF
:1087A0000C028A6050FA86F200EB146C12789CF886
:1087B00000C0C5F3072442EA0C62C9F3074C10F865
:1087C0000CC0005D4FEA0C4C4CEA00201043DA6804
:1087D0005040C860BDE8F80F70470000003002400C
:1087E000744301084C3E01082DE9F80F4FF0030CCB
:1087F0000CEBE308C24B4FF0010CC3F808C0D3F8F0
:1088000008C0D3F800C0CDF800C0BCF1FF3F00F0B5
:10881000E5804368D2F804C0006883EA0C07136857
:1088200080EA0304A4466346B6483D0ECCF30746EF
:1088300050F8255050F8266004F0FF0985EA3625E7
:10884000C3F3072650F8299050F8266007F0FF0A76
:108850004FEA364686EA396675401669C3F307491A
:108860006E404FEA1C6550F8299050F8255050F89A
:108870002AA085EA3925C4F307290CF0FF0B50F82C
:108880002990CCF3072C4FEA394989EA3A6985EAFD
:108890000905D2F81490C4F3074A85EA09054FEA9E
:1088A000136950F82AA050F82990240E89EA3A2931
:1088B000C7F3072AC7F30747DBB250F82AA050F8DE
:1088C0002CC050F82BB050F8244050F8277050F8C6
:1088D00023304FEA3A4A4FEA3C4C8AEA3B6A84EA40
:1088E00037248CEA336389EA0A0984EA030CD2F854
:1088F00018A0D3692032A8F1010889EA0A098CEA94
:108900000304B8F1000F7CDD330EC5F3074C50F8BB
:10891000233050F82CC0E7B283EA3C23C9F3072C7C
:1089200050F8277050F82CC006F0FF0A4FEA3C4C74
:108930008CEA376C83EA0C03D2F800C050F82AA006
:1089400083EA0C072B0EC9F3074C50F8233050F87C
:108950002CC005F0FF0B83EA3C23C4F3072CC5F3BE
:10896000072550F82CC050F825504FEA3C4C8CEAB3
:108970003A6C83EA0C03D2F804C0C4F3074A83EAD2
:108980000C0C4FEA196350F82AA050F82330240E3B
:1089900083EA3A23C6F3072AC6F3074650F8244071
:1089A00050F8266050F82AA084EA362409F0FF0621
:1089B00050F82BB050F826604FEA3A4A4FEA354556
:1089C0008AEA3B6A85EA366583EA0A036C40D2F894
:1089D00008A0D56883EA0A036C4026E7DDF800C0EA
:1089E000C3F800C01B68009363B14368D2F804C0A9
:1089F000006883EA0C07136880EA030C6346644648
:108A000012E710E00368D2F800C0946883EA0C070C
:108A10004368D2F804C083EA0C0C8368C0686340E2
:108A2000D468444000E7384850FA84F300EB166CF1
:108A30001B789CF800C0C9F3072743EA0C63C5F311
:108A4000074CC75D10F80CC04FEA0C4C4CEA072CE1
:108A500043EA0C03D2F800C083EA0C030B6050FA1F
:108A600086F300EB156C1B789CF800C0C4F3072755
:108A700043EA0C63C9F3074CC75D10F80CC04FEA1A
:108A80000C4C4CEA072C43EA0C03D2F804C083EAEE
:108A90000C034B6050FA85F300EB196C1B789CF8C3
:108AA00000C0C6F3072743EA0C63C4F3074CC75D55
:108AB00010F80CC04FEA0C4C4CEA072C43EA0C03AC
:108AC000D2F808C083EA0C038B6050FA89F300EBFC
:108AD000146C1B789CF800C0C5F3072443EA0C63B0
:108AE000C6F3074CD26810F80CC0005D4FEA0C4C7E
:108AF0004CEA002018435040C860BDE8F80F7047AA
:108B000000300240743F01084C3D010870B50C462E
:108B10008446002315462046B3EBA20F09DA00BFB6
:108B20005CF8231009BA40F823105B1CB3EBA20FCA
:108B3000F6DB214600F096F8E910052000EB410332
:108B4000002BD8BF70BD04F11002454800F5C56187
:108B5000D2F800C000EB1C64CCF307452478455DD7
:108B600051F8244051F8255084EA3524CCF30725E8
:108B7000455D51F825504FEA354550FA8CFC9CF87C
:108B800000C051F82CC085EA3C6C84EA0C0C42F819
:108B900004CB52F804CB00EB1C64CCF307452478DB
:108BA000455D51F8244051F8255084EA3524CCF332
:108BB0000725455D51F825504FEA354550FA8CFCA4
:108BC0009CF800C051F82CC085EA3C6C84EA0C0C7F
:108BD00042F804CC52F808CB00EB1C64CCF30745F8
:108BE0002478455D51F8244051F8255084EA352415
:108BF000CCF30725455D51F825504FEA354550FA2D
:108C00008CFC9CF800C051F82CC085EA3C6C84EACE
:108C10000C0C42F808CC52F804CC00EB1C64CCF3EA
:108C200007452478455D51F8244051F8255084EAE1
:108C30003524CCF30725455D51F825504FEA3545DD
:108C400050FA8CFC9CF800C05B1E51F82CC085EAE1
:108C50003C6C84EA0C0C42F804CC7FF479AF70BD14
:108C60004C3D010870B400239510002D15DDA0F1D6
:108C7000040C081F12F0040F03D05CF8044F40F8F6
:108C8000044FD21009D000BFDCF8044044605CF807
:108C9000084F40F8084F521EF6D1684C042DA4F539
:108CA000007005D0062D34D0082D6DD070BC7047F3
:108CB000CA6800EB126CC2F307459CF800C0455D22
:108CC0004CEA056CC2F30725455D2D0450FA82F687
:108CD000367845EA06254CEA050C54F823600D6801
:108CE0005B1C75408CEA050CC1F810C04D680A2B5E
:108CF0008CEA050CC1F814C08D688CEA050C8CEA6E
:108D00000202C1F818C0CA61B8BF1031D0DB70BC14
:108D100070474A6900EB126CC2F307459CF800C02B
:108D2000455D4CEA056CC2F30725455D2D0450FAFC
:108D300082F6367845EA06254CEA050C54F823609D
:108D40000D685B1C75408CEA050CC1F818C04D68B5
:108D5000082B8CEA050CC1F81CC08D688CEA050C48
:108D6000C1F820C0CD688CEA050CC1F824C0A4BFAE
:108D700070BC70470D698CEA050C8CEA0202C1F8E0
:108D800028C0CA621831C4E7CA6900EB126CC2F38A
:108D900007459CF800C0455D4CEA056CC2F3072509
:108DA000455D2D0450FA82F6367845EA06254CEAF0
:108DB000050C54F823600D685B1C75408CEA050CAB
:108DC000C1F820C04D68072B8CEA050CC1F824C0FF
:108DD0008D688CEA050CC1F828C0CD688CEA050CBA
:108DE000C1F82CC0A4BF70BC704750FA8CF52D7828
:108DF00000EB1C66367845EA0665CCF30746CCF3F3
:108E0000072C865D10F80CC0360446EA0C2C45EAA7
:108E10000C0C0D698CEA050CC1F830C04D698CEA68
:108E2000050CC1F834C08D698CEA050C8CEA02028D
:108E3000C1F838C0CA632031A6E700004C3F0108E2
:108E40002DE9F0410E46002818BF002E04D003F093
:108E500006012AB9022903D04FF44260BDE8F0812F
:108E6000D0F824C0BCF1100F1CBFBCF1180FBCF12E
:108E7000200F08D102290AD0D0F810C0ACF1010CA3
:108E8000BCF1100F03D340F61F40BDE8F081C26073
:108E900090F804C002292CF0060C80F804C048D0D9
:108EA000002141618161C1610162D0F810C0BCF153
:108EB000000F3EDD1CF0010F4FF01804A2F101027B
:108EC00004D012F8011F0906416101215FEA6C0C10
:108ED0002FD0CF1701EB977727F00307CF1B5578DB
:108EE0007F4204EBC70705FA07F721F003050544A5
:108EF000D5F8148047EA08076F614D1C4FEAE57802
:108F000005EB987828F00308A5EB080512F8027F16
:108F10006D4204EBC505AF404D1C25F0030505442B
:108F2000891CD5F81480BCF1010C47EA08076F6171
:108F3000CFD1017911F0010F0DD113F0010F86602F
:108F40001CBF062131EA030108D000F12801426A62
:108F50003046FFF7DBFD0020BDE8F08100F128017D
:108F6000426A0020B0EBA20F09DA00BF56F82030A9
:108F70001BBA41F82030401CB0EBA20FF6DB0846CC
:108F8000FFF770FEE7E7000030B50246130100204E
:108F900013E000210EE00A4C1C4404EB8004645CE6
:108FA000084D05EB81052D5C6C40064D05EB8105F8
:108FB0002C54491C0429EEDB401C0428E9DB30BD9D
:108FC00025AB002015AB0020704700BFFEE772B64E
:108FD0007047000070B5002600240DE0002508E071
:108FE00005EB84001C49085C1C4901EB8501085510
:108FF0006D1C042DF4DB641C042CEFDB0020FFF758
:10900000C3FF012609E001F0B9F801F095F800F07E
:1090100085FC3046FFF7B8FF761C11480068864291
:10902000F1DB01F0ABF801F087F80D480068FFF7BD
:10903000ABFF00240DE0002508E0084800EB8500A8
:10904000005D05EB8401074A50546D1C042DF4DBD0
:10905000641C042CEFDB70BDE5AA002015AB0020DA
:1090600040060020F5AA0020024600210AE00F4B2E
:1090700013F81100904203D14800401C185C70475F
:10908000481CC1B21229F2DB00210AE04800401C52
:10909000064B185C904202D113F81100EFE7481C10
:1090A000C1B21229F2DB0020E9E70000FA39010819
:1090B00030B591B004460D46402101A8FFF78FF866
:1090C00094208DF804000B208DF805002A462146D7
:1090D0000DF10600FFF75CF801A80AF01BF911B0CA
:1090E00030BD7047FEB506460C4617461D46022D9C
:1090F00001D1012500E000250A484078012809D166
:1091000002A823463A461021CDE90005304600F07A
:109110009DFF05E02B463A4631462046FFF7B6F85C
:10912000FEBD00009C4B00202DE9F04104460E4698
:10913000174605F00DFFA02005F0AAFEC4F3072096
:1091400005F0A6FEE0B205F0A3FE05F001FFA120A8
:1091500005F09EFE002504E005F058FE7055681CE1
:10916000C5B2BD42F8DB05F017FF0120BDE8F08174
:109170002DE9F047054689461646002400BF281908
:1091800000F01F00C0F120008046311B884203DB45
:10919000301B00F0FF0800E000BF05F0D9FEA02062
:1091A00005F076FE2919C1F3072005F071FE291993
:1091B000C8B205F06DFE002706E0E11919F80100BC
:1091C00005F066FE781CC7B24745F6DB05F0E4FE05
:1091D0000A2004F0BBF804EB0800C4B2B44200DB80
:1091E00000E0CCE700BFBDE8F08710B5802005F0B7
:1091F000CDF828B1032008F011FB802005F0C0F85D
:1092000010BD0000FEB506460D4617461C46022C52
:1092100001D1012400E000240A484078012809D146
:1092200002A82B463A461021CDE90004304600F052
:1092300047FF05E023463A4629463046FFF724F922
:10924000FEBD00009C4B002000B587B072211F4876
:1092500005F012FD40F207111D4805F00DFD4FF419
:1092600040711C4805F008FD72200190102002900A
:10927000002003900420049001A9144800F045F850
:1092800040F207100190102002900020039004206B
:10929000049001A90E4800F038F8802001900420C5
:1092A00002900020039001A9084800F02EF84FF426
:1092B0004070019010200290002003900420049040
:1092C00001A9044800F021F807B000BD00100140DA
:1092D00000080140000C014070B504460D462A46C6
:1092E0002146024804F0C2FA70BD00009C0600202E
:1092F00000B5014600F026F8024600BF00F022F853
:10930000801A884200D300BDF8E770B505460C46C8
:109310002846D4E90031E26805F00AFD70BD70B559
:1093200004460D462946204605F060FD012804D17B
:109330002946204605F0A0FC03E02946204605F01A
:109340009DFC70BD01480068704700004403002088
:1093500002480068401C014908607047440300202F
:1093600000B587B040F2026008F07EF840F2046079
:1093700008F07AF84FF4C06008F076F840F20C601C
:1093800008F072F84023042210211F4805F0D0FC99
:10939000A023042218211D4805F0CAFC4023042202
:1093A00011461A4805F0C4FC8023042211461648D1
:1093B00005F0BEFC002001904FF482700090002068
:1093C000029005904FF4007003901020069000204A
:1093D000049069460E4808F008FD0D4808F0F2FCBC
:1093E00000220321172007F07BFA0721022005F055
:1093F00053FC01220021802004F066FF802004F04D
:10940000BFFF07B000BD0000001001400008014090
:10941000003001402DE9F04104460D4616464FF05C
:10942000000800270AE02A466D1C14F8011B0648B4
:1094300000F00CF840EA0808781C87B2B742F2DB6B
:109440000020BDE8F08100000030014070B5064604
:109450000D46144600BF02210A4808F0BEFC002851
:10946000F9D02946074808F0B6FC00BF012105489D
:1094700008F0B3FC0028F9D0024808F0A8FC2070DE
:10948000207870BD0030014000BFFEE770B50026B7
:1094900000240DE0002508E005EB84001C49085C71
:1094A0001C4901EB850108556D1C042DF4DB641C7F
:1094B000042CEFDB18480068FFF766FD16480068CB
:1094C000461E09E000F040F900F05EF93046FFF773
:1094D0005BFD00F025F8761E002EF3DC00F034F979
:1094E00000F052F90020FFF74FFD00240DE00025A9
:1094F00008E0084800EB8500005D084901EB8401A5
:1095000048556D1C042DF4DB641C042CEFDB70BD8E
:10951000E5AA002015AB002040060020F5AA002097
:109520002DE9FF47002107E1DFF8189219F80190B3
:109530008DF80C90DFF80C9209F1040919F80190EC
:109540008DF80890DFF8FC9109F1080919F80190ED
:109550008DF80490DFF8EC9109F10C0919F80190ED
:109560008DF80090012056E00DF10C09814419F8A6
:10957000019C4FEAD91909EBC90909EB49090DF119
:109580000C0A82441AF801AC89EA4A090DF10C0A66
:109590000AF800900DF10809814419F8019C4FEA7E
:1095A000D91909EBC90909EB49090DF1080A8244E7
:1095B0001AF801AC89EA4A090DF1080A0AF8009084
:1095C0000DF10409814419F8019C4FEAD91909EBFE
:1095D000C90909EB49090DF1040A82441AF801ACE2
:1095E00089EA4A090DF1040A0AF800900DEB000916
:1095F00019F8019C4FEAD91909EBC90909EB490986
:109600000DEB000A1AF801AC89EA4A0909F0FF09D2
:109610000DF80090401C0428A6DB9DF80E909DF8E4
:109620000FA089EA0A029DF80C909DF80FA089EA24
:109630000A039DF80A909DF80BA089EA0A049DF898
:1096400008909DF80BA089EA0A069DF806909DF8FF
:1096500007A089EA0A079DF804909DF807A089EA07
:109660000A059DF802909DF803A089EA0A0C9DF86E
:1096700000909DF803A089EA0A089DF80D9089EAF8
:10968000020989EA06099DF809A089EA0A099DF8F4
:1096900004A089EA0A0989EA070989EA0809DFF8C2
:1096A000A4A00AF801909DF8099089EA030989EAC3
:1096B000040989EA05099DF805A089EA0A099DF8C7
:1096C00000A089EA0A0989EA0C09DFF878A00AF102
:1096D000040A0AF801909DF80C9089EA020989EAC7
:1096E00006099DF805A089EA0A0989EA070989EAB5
:1096F00008099DF801A089EA0A09DFF848A00AF1E3
:10970000080A0AF801909DF80D9089EA03099DF86E
:1097100008A089EA0A0989EA040989EA05099DF885
:1097200001A089EA0A0989EA0C09DFF818A00AF100
:109730000C0A0AF80190491C0429FFF6F5AEBDE8B1
:10974000FF87000015AB00200E49C8798A79CA71DD
:109750004A798A710A794A710871087A897A094ABC
:10976000117211468872487ACA7A4A72C872087BA6
:10977000497B044A117311468A7B4A73CA7B8A73F8
:10978000C873704715AB002000200FE000210AE0ED
:10979000084A02EB8002525C074B9A5C054B03EBD4
:1097A00080035A54491C0429F2DB401C0428EDDBD9
:1097B0007047000015AB0020243A0108F8B50025D9
:1097C00000264F48006882004E494F48FEF7E0FCF3
:1097D0004B4804688CE0601E4B4901EB8000006838
:1097E00000904748006894FBF0F100FB114080BBFB
:1097F0009DF800709DF801008DF800009DF80200B2
:109800008DF801009DF803008DF802008DF80370BB
:109810009DF800003D49085C8DF800009DF80100AE
:10982000085C8DF801009DF80200085C8DF80200CC
:109830009DF80300085C8DF803003148006894FB34
:10984000F0F03349085C9DF8001048408DF80000A6
:1098500024E0FFE72A48006806281FDD2848006842
:1098600094FBF0F100FB1140042817D19DF8000093
:1098700005F07EF88DF800009DF8010005F078F8FD
:109880008DF801009DF8020005F072F88DF80200D5
:109890009DF8030005F06CF88DF80300A006050E96
:1098A00017480078201A8006060E1748805D9DF83C
:1098B00000104840144948550846304440789DF807
:1098C000011048401049294448700F4830448078BE
:1098D0009DF8021048400C49294488700A483044D9
:1098E000C0789DF80310484007492944C870641C9B
:1098F00008480068401C8000A0423FF76CAFF8BDEC
:109900004406002051AC002025AB0020243B010878
:10991000243C01084006002000BFFEE730B50020CF
:1099200068E0364C235C245C344D2D1D2D5C6C406E
:10993000324D08352D5C6C40304D0C352D5C84EA81
:1099400005022E4C255C241D245C85EA0401CC090B
:1099500004EBC40404EB440484EA4104E1B2274C60
:10996000245C81EA02056C40244D2C542C1D245C9F
:1099700008352D5C84EA0501CC0904EBC40404EB32
:10998000440484EA4104E1B21C4C241D245C81EAB5
:1099900002056540194C241D2554241D245C174DD7
:1099A0000C352D5C84EA0501CC0904EBC40404EBFE
:1099B000440484EA4104E1B2104C0834245C81EA96
:1099C00002056C400D4D08352C542C1D245C84EA96
:1099D0000301CC0904EBC40404EB440484EA41040D
:1099E000E1B22C1D245C81EA02056C40034D0C356C
:1099F0002C54401C042894DB30BD000015AB002023
:109A00000948008878B108480088401E80B206499D
:109A1000088040B9002005494870C1F82404C1F805
:109A20002804C1F82C047047780500205C4700200A
:109A30007047000070B505460C46002605F070051D
:109A4000204600F0E1F806460E4A32F814100E4A9D
:109A500052F8240005F010F92146272004F016FAE8
:109A600045EA0600214604F011FA064A32F81410BD
:109A7000054A52F8240005F001F9204600F0C4F828
:109A800070BD00007C3901086C39010810B504462E
:109A90000A4A32F814100A4A52F8240005F0ECF889
:109AA0002146E22004F0F2F9044A32F81410044A84
:109AB00052F8240005F0E2F810BD00007C390108DE
:109AC0006C39010810B504460A4A32F814100A4AE3
:109AD00052F8240005F0D0F82146E12004F0D6F930
:109AE000044A32F81410044A52F8240005F0C6F86B
:109AF00010BD00007C3901086C390108F0B5C1B017
:109B000005460E4617461C460D4A32F814100D4AFB
:109B100052F8240005F0B0F82846214604F0B6F9C2
:109B200023463A46314601A804F0BFF9044A32F808
:109B30001410044A52F8240005F0A0F841B0F0BD1A
:109B40007C3901086C39010870B505460C460D4A90
:109B500032F814100C4A52F8240005F08DF828460B
:109B6000214604F093F92146FF2004F08FF90646C0
:109B7000044A32F81410044A52F8240005F07EF822
:109B8000304670BD7C3901086C39010830B5C3B06E
:109B900005460C4621460720FFF7D6FFC0F34200DA
:109BA0004190204600F04EF842909DF80801202890
:109BB00005DD2046FFF76AFF002043B030BD104AA4
:109BC00032F814100F4A52F8240005F055F82146D7
:109BD000612004F05BF923469DF80821294601A87D
:109BE00004F063F9064A32F81410064A52F82400C9
:109BF00005F044F82046FFF749FF9DF80801DCE72F
:109C00007C3901086C39010870B504460B4A32F8FA
:109C100014100B4A52F8240005F02EF821460720B4
:109C200004F034F90546054A32F81410044A52F893
:109C3000240005F023F8284670BD00007C39010897
:109C40006C39010870B504460D4A32F814100D4AFB
:109C500052F8240005F010F82146602004F016F9AF
:109C60002146FF2004F012F90546054A32F8141087
:109C7000044A52F8240005F001F8284670BD00009F
:109C80007C3901086C39010870B504460D46294637
:109C90000620FFF759FF20F0070604F007000643EF
:109CA0002A463146062000F075F870BD2DE9F041D6
:109CB00004460E4615461F46052D01DD052000E031
:109CC00028460546052C01DD052000E02046044617
:109CD00004F10A01C8B23B462A46314600F032F888
:109CE000BDE8F08170B505460E46002431460620D9
:109CF000FFF72AFF044624F0280415B944F0200495
:109D000008E0012D02D124F0280403E0022D01D146
:109D100044F0080432462146062000F03BF870BDAE
:109D200070B505460C461646052C01DD052000E001
:109D300020460446334622462946102000F002F809
:109D400070BD0000F0B5C1B005460E4617461C4672
:109D50000E4A32F814100E4A52F8240004F08CFF18
:109D600045F02000214604F091F823463A4601A927
:109D7000304604F09AF8054A32F81410044A52F8B2
:109D8000240004F07BFF41B0F0BD00007C390108E5
:109D90006C39010870B505460E461446104A32F873
:109DA0001410104A52F8240004F066FF0E4A32F8EC
:109DB00014100E4A52F8240004F05EFF45F0200013
:109DC000214604F063F82146304604F05FF8064A65
:109DD00032F81410054A52F8240004F04FFF70BD09
:109DE000C8390108B83901087C3901086C39010803
:109DF00070B5C0B006460D461446202D00DC0DB9E6
:109E000040B070BD0D4A32F814100D4A52F82400CB
:109E100004F032FF2146B02004F038F823462A46E9
:109E20006946304604F041F8044A32F81410044AF6
:109E300052F8240004F022FF00BFE1E77C3901085A
:109E40006C3901087FB5054611A103C9CDE90201AE
:109E50000020009001902B46052202A91020FFF758
:109E600071FF2B46052269461020FFF747FE0024AC
:109E70000AE002A8005D1DF80410884202D000200C
:109E800004B070BD601CC4B2052CF2DB0120F7E702
:109E90001122A3A4A500000010B5002807DA0A07C4
:109EA000140E054A00F00F031B1FD45403E00A07E9
:109EB000130E024A135410BD18ED00E000E400E058
:109EC000BFF34F8F0648006800F4E060054908437F
:109ED000001D03490860BFF34F8F00BFFEE700007D
:109EE0000CED00E00000FA05704770B504460D4621
:109EF00004F07F012A460520FFF74CFF70BD10B526
:109F0000044621467020FFF795FD10BD10B50446AC
:109F10000A4A32F814100A4A52F8240004F0ACFE3F
:109F20002146012000F00EF8044A32F81410044AC9
:109F300052F8240004F0A2FE10BD0000C839010848
:109F4000B839010870B504460E4600253146002098
:109F5000FFF7FAFD054614B925F0010503E0012CD1
:109F600001D145F00105324629460020FFF712FFD6
:109F700070BD00007CB50446194881696846884771
:109F80007CB99DF800109DF8012011449DF8022035
:109F900002EB01219DF803208818FEF7F1F800205C
:109FA0007CBD012C14D10F4808F06CF89DF800100E
:109FB0009DF8012011449DF8022002EB01219DF83B
:109FC0000320114445182846FEF7DAF80120E7E798
:109FD000FEF7CCF8B0FBF4F104FB1100E0E7000061
:109FE000480300200010004062B6704700B587B0FB
:109FF000182101A8FEF7F3F84FF4007001904820F3
:10A000000290012003900320049001A90248FFF769
:10A010007CF907B000BD0000000C014000B587B01E
:10A02000182101A8FEF7DBF84FF400700190102012
:10A030000290012003900320049001A90248FFF739
:10A0400064F907B000BD0000000C01402DE9F047A5
:10A05000C8B006460F4690469946DDF844A1509C8C
:10A060000025002001908DF80C00BAF1000F02D1FC
:10A0700010200B9001E020200B900022414602A806
:10A08000FEF790F90546BDB901A84B463A46314660
:10A09000009002A8FEF71CF905466DB901982060F2
:10A0A000206800EB090101AA02A8FEF76EF9054637
:10A0B0002068019908442060284648B0BDE8F08730
:10A0C0002DE9F047C8B006460F4690469946DDF8A0
:10A0D00044A1509C0025002001908DF80C00BAF19D
:10A0E000000F02D110200B9001E020200B900022E5
:10A0F000414602A8FEF7C4F90546BDB901A84B4682
:10A100003A463146009002A8FEF750F905466DB96F
:10A1100001982060206800EB090101AA02A8FEF75F
:10A12000A2F905462068019908442060284648B0F5
:10A13000BDE8F087704700000F49087949790E4A59
:10A14000117111468A794A71CA798A71C871087A7F
:10A15000897A094A117211468872487ACA7A4A7213
:10A16000C872087BC97B044A117311468A7BCA7383
:10A170004A7B8A734873704715AB002000200FE0BC
:10A1800000210AE0084A02EB8002525C074B9A5C0D
:10A19000054B03EB80035A54491C0429F2DB401C95
:10A1A0000428EDDB7047000015AB0020243B0108BC
:10A1B00010B5FFF7CDF810BD08B51848006840F499
:10A1C0007000164908601648006840F00100144904
:10A1D00008600846406840F0800048600020009019
:10A1E00002E00098401C009044F6206100988842EC
:10A1F000F7D300200A494860C86208460068094948
:10A200000840074908604FF41F008860084600684E
:10A2100020F48020086007F0A9FE08BD88ED00E06A
:10A2200000100240FFFFF6FE10B50121880707F07D
:10A230008CFF40B10121880707F084FF0249C868FC
:10A24000804708F08DFE10BD480300201FB5002098
:10A25000009001900290039040F2AF40ADF80000F2
:10A260000020ADF80200ADF80400F92002900020B3
:10A27000ADF806008DF80C0069464FF0804007F0FD
:10A280000DFF002203211C2006F02AFB00214FF0C5
:10A29000804007F0FBFE002240F2AF414FF08040CB
:10A2A00007F080FFF921880707F0EAFE01218807FF
:10A2B00007F040FF0121880707F044FF01218807CC
:10A2C00007F03CFF4FF0804007F0E2FE1FBD0000AA
:10A2D00010B50121064807F038FF40B101210448BC
:10A2E00007F030FF03490869804708F034FE10BDCD
:10A2F00000040040480300201FB50020009001909A
:10A300000290039040F2AF40ADF800000020ADF89D
:10A310000200ADF8040040F2CF7002900020ADF8CA
:10A3200006008DF80C006946134807F0B7FE0022BE
:10A3300004211D2006F0D4FA00210F4807F0A6FEE4
:10A34000002240F2AF410C4807F02CFF40F2CF71E1
:10A35000094807F095FE0121074807F0EBFE0121AF
:10A36000054807F0EFFE0121034807F0E7FE024829
:10A3700007F08EFE1FBD00000004004010B5012153
:10A38000880707F0E2FE18B10121880707F0DAFE1E
:10A3900010BD10B508F066FC10BD000000B591B00E
:10A3A000402101A8FDF71BFF2C4890F84E008DF8C6
:10A3B00004002A4890F84F008DF80500274890F8CF
:10A3C00050008DF80600254890F851008DF80700E0
:10A3D000FE208DF8080048208DF80900DE208DF859
:10A3E0000A007F208DF80B0001208DF80C00022060
:10A3F0008DF80D00302219495231002000F030F85C
:10A4000000909DF800008DF80E009DF801008DF879
:10A410000F00124840788DF8100030220F49523159
:10A4200005A8FDF7B5FE30210C485230FDF7D7FEE8
:10A4300000200A4981F88200202101A800F0C4FB15
:10A4400000F0D8FB142000F03FF8202109A800F00C
:10A45000BBFB00F0CFFB11B000BD0000C8630020C3
:10A4600070B506460C4615462946204603F056F9B7
:10A470000646304670BD000010B50446074890F807
:10A48000310440B14FF48062044911312046FDF798
:10A490007FFE002010BD0120FCE70000945F00203B
:10A4A00030B50A46CD1701EB5575C5F3C703CD1777
:10A4B00001EB5575ED10A1EBC505ECB2C25C0125B1
:10A4C000A540AA43C25430BD10B50446204602F050
:10A4D0005AFF10BD30B502460846CD1701EB557541
:10A4E000C5F3C703CD1701EB5575ED10A1EBC505FD
:10A4F000ECB2D05C0125A540284008B1012030BD58
:10A500000020FCE770B505460E4614460948296848
:10A51000C0F84E10A0F88860C0F88440C4F38F20C3
:10A52000044988800846B0F8881003A005F090F927
:10A5300070BD0000C86300200A433A25780000007F
:10A5400001464878AA2808D18878BB2805D1C87860
:10A55000CC2802D10879DD281FD01B4890F84E0086
:10A560004A78904201D002207047174890F84F0077
:10A570008A78904201D00220F6E7134890F8500004
:10A58000CA78904201D00220EEE70F4890F85100BF
:10A590000A79904201D00220E6E748797F2801D06D
:10A5A0000120E1E78879DE2801D00120DCE7C879C5
:10A5B000482801D00120D7E7087AFE2801D00120E1
:10A5C000D2E70020D0E70000C863002070B58AB051
:10A5D00005460C46242101A8FDF701FEE0B28DF8E6
:10A5E0000400224629460DF10500FDF7D1FD01A822
:10A5F000FFF7A6FFA0B99DF80E00822801D00AB08F
:10A6000070BD0120274908702748DDF8111001604E
:10A610009DF80F00254908709DF810004870EEE77E
:10A620002048007801283AD100201E4908702022D5
:10A630000DF10501FFF714FF06461C480088B042E3
:10A640002CD11BA005F004F91B4890F882001028BB
:10A6500010DA194890F882001749523101EB800056
:10A66000114909680160144890F88200401C1249A1
:10A6700081F8820000200FE001AA411C515C49B121
:10A680000D490A31095C01AB421C9A5C11430A4A2C
:10A690000A321154411CC8B22028EDDBAFE700BFDD
:10A6A000ADE700009C050020A00500209E050020CD
:10A6B0000A43524354000000C863002070B58AB0BA
:10A6C00005460C46242101A8FDF789FD00263448E3
:10A6D00090F84E008DF80400314890F84F008DF846
:10A6E00005002F4890F850008DF806002C4890F88F
:10A6F00051008DF8070042208DF8080001208DF8E8
:10A700000900274800788DF80A008DF80B50FF20CB
:10A710008DF80C008DF80D0000208DF80E008DF8DE
:10A720000F008DF810008DF811001D4890F884007E
:10A730008DF812001A4890F885008DF8130018481B
:10A7400090F886008DF81400154890F887008DF871
:10A750001500134890F888008DF81600104890F8FE
:10A7600089008DF817000E4880788DF818001B229C
:10A7700002A90020FFF774FEC6B28DF823600AE03C
:10A78000202101A800F020FA00F034FA3220FFF76F
:10A790009BFE601EC4B2002CF2D10AB070BD000056
:10A7A000C863002030B589B0054624216846FDF70E
:10A7B00016FD344890F84E008DF80000314890F8AE
:10A7C0004F008DF801002F4890F850008DF80200DE
:10A7D0002C4890F851008DF80300FE20294981F89B
:10A7E0004A004821274880F84B10DE2180F84C10A1
:10A7F0007F2180F84D1090F84A008DF80400214820
:10A8000090F84B008DF805001E4890F84C008DF82C
:10A8100006001C4890F84D008DF8070020208DF8A8
:10A82000080001208DF80900164890F88E048DF874
:10A830000A00144890F88F048DF80B001148007836
:10A840008DF80C008DF80D502021684600F0BCF901
:10A8500000F0D0F9C820FFF737FE00240EE00949C8
:10A860008A31202202FB0410114600F0ADF900F0FD
:10A87000C1F91420FFF728FE601CC4B2202CEEDBC7
:10A8800009B030BDC863002010B501200749087029
:10A8900007480078401C0649087041F2707005496D
:10A8A00008600548816B0020884710BD9005002096
:10A8B000C8630020940500204803002070B50546B9
:10A8C0000C460020034981F8310421460A2007F094
:10A8D00033FD70BD945F002070B5AF48006878B15B
:10A8E000AD480068401EAC49086048B9AB480078E4
:10A8F00030B1AA480078052802D00520A749087081
:10A90000A648007806287CD2DFE800F0030443B9AB
:10A91000D8FE3EE11E210120FFF7D0FEA0480088AE
:10A92000401C9F49088008460088282830DD002107
:10A930009C48A0F88A1440F2FF11A0F88C14012062
:10A940009849087200204872302196485230FDF72D
:10A9500046FC0020934981F8820091490880914982
:10A960008871FF2240218F480A30FDF731FC8D4A63
:10A9700092F88A149079FFF7A1FF002189480A30E4
:10A98000FFF78EFD00208749C871022083490870B7
:10A99000FFE08448B0F88A1483A004F059FF81488E
:10A9A000C079012816D07F488A30FFF765FD88B945
:10A9B00001207C49C871002048724FF480628A31BE
:10A9C000FFF74EFD7749A1F88E040846B0F88A14C7
:10A9D000A0F88C147348B0F88C0440F2FF11884240
:10A9E00019D07048407A401CC0B26E494872C828DD
:10A9F00001DDC82048726B4991F88C04FFF7D2FE44
:10AA000000E0C5E04FF4E160FFF75EFD654991F8B5
:10AA10008C04FFF7C7FE6348407A6249097A88428E
:10AA20002CDB6048C079012828D100205D49C8711D
:10AA300000241EE021465B480A30FFF74BFD70B151
:10AA4000214658480A30FFF72BFD5648A0F88A44A3
:10AA5000024692F88A149079FFF730FF0DE05148D2
:10AA60008088401EA04202D103204C490870601C1F
:10AA7000C4B24C488088A042DCDC00BF89E00020E2
:10AA80004749088047488078401C46498870202103
:10AA900044480A30FDF7A3FB0420404908704148B0
:10AAA00041784078401C3F4A5070C82902DD01209F
:10AAB000114648703EA004F0CBFE6AE0FFF76EFC42
:10AAC00037480088401C36490880084600883228EC
:10AAD00046DB002500200880002409E0214631489B
:10AAE0000A30FFF7F7FC08B1681C85B2601C84B21D
:10AAF0002C488088A042F1DC294630A004F0A8FE52
:10AB00002DB90520254900E02BE0087041E02548DB
:10AB10008079401C2349887108200872002416E0BF
:10AB2000214620480A30FFF7D5FC70B121461D4868
:10AB30000A30FFF7B5FC1B48A0F88A44024692F899
:10AB40008A149079FFF7BAFE05E0601CC4B215487C
:10AB50008088A042E4DC00BF02201049087018E0A1
:10AB600017E01E210220FFF7A9FD0D480088401CB8
:10AB70000B49088008460088282808DD002006497F
:10AB80000860074908800549087007F02DFB00E0C0
:10AB900000BF00BF70BD000094050020900500209C
:10ABA0009A050020C86300200A533A25640000007B
:10ABB000444F574E5F515545525900000A4C4E754F
:10ABC0006D3A25640000000070B505460C46002073
:10ABD00007F0A6F80549C86A80470646E1B204486E
:10ABE0003246836A28469847012070BD48030020FA
:10ABF000B802002010B54FF4FA7408E004F01EF813
:10AC000000B110BD0220FFF75FFC601E84B2002C73
:10AC1000F4D100BFF5E700BFFEE7002107E048F2EE
:10AC2000782100BF0A1EA1F1010399B2FAD1021ED8
:10AC3000A0F1010398B2F2D17047000010B590B0B6
:10AC4000044620798DF8000020791E286FD2DFE8B5
:10AC500000F06E1F0F5C2B6E6E6E6EAB9F8B7B6E6B
:10AC60006EC7C26E6ECCCBDECDF1F2EFEE6E6EED46
:10AC70000D22A949601D04F07CFE00F02DFF0D227D
:10AC8000A549C02002F084FA01208DF8000000BF21
:10AC90000D220DF10101A04804F06BFE0E22694661
:10ACA0000B2005F0C7FF34E106229C49601D04F02B
:10ACB00060FE9B4890F8820028B1994890F8820085
:10ACC0009649491E88709548401E807820B1934867
:10ACD000401E8078042803DD01209049491E8870B9
:10ACE0008E48401E80788F49497A884204DD8D481D
:10ACF000407A8A49491E88708849491EC87806F0FA
:10AD0000C1F904208DF8000000BF854890F8840048
:10AD1000292800D1FDE0824890F88400282800D13D
:10AD2000F7E07F4890F88400332801D1F1E0EAE0B1
:10AD300006220DF10101794804F01BFE0722694645
:10AD40000B2005F077FFE4E0754890F87F0000B92C
:10AD5000DFE003227449601D04F00BFE03227249F8
:10AD6000D82002F015FA00BF6D4890F87F0000B9B6
:10AD7000CFE00B208DF8000003220DF101016A489D
:10AD800004F0F7FD042269460B2005F053FFC0E0F4
:10AD9000634890F8800000B9BBE06079012802D1D7
:10ADA0001E206249487000BF5D4890F8800000B9DD
:10ADB000AFE009208DF800005C484078002801DDF4
:10ADC000012000E000208DF80100022269460B20DE
:10ADD00005F030FF9DE05248816A2046884700BF59
:10ADE0004F49C86A804794E000BF92E0182250495A
:10ADF000601D04F0BEFD4E48401E807818B1012051
:10AE000006F052FF02E0002006F04EFF00BF1520C2
:10AE10008DF8000018220DF10101454804F0A9FD4C
:10AE2000192269460B2005F005FF72E066E029E073
:10AE300058E000E01AE00D223E49601D04F099FD43
:10AE400000F04AFE36480C21D0F80C213948401C4D
:10AE500090473349D1F8FC0080470D223549C02086
:10AE600002F096F917208DF8000000BF0D220DF1B9
:10AE70000101304804F07DFD0E2269460B2005F0EB
:10AE8000D9FE46E003222C49601D04F072FD2A48D9
:10AE9000401EC178807801EB00204EF66021884288
:10AEA00007DDEA202449491E887060212248401E9F
:10AEB000C170214A521ED378927803EB022290B2DD
:10AEC000174AD2F8041188471549D1F8FC00804789
:10AED000032219494FF4856002F05AF919208DF8C0
:10AEE000000000BF03220DF10101134804F041FDF1
:10AEF000042269460B2005F09DFE0AE00F48016818
:10AF00002046884705E00648D0F8E41020468847E8
:10AF100000BF00BF10B010BD59080020D7030020AB
:10AF20004404002000110020D3030020D00300209F
:10AF3000DC07002067080020DF0300203804002021
:10AF40002DE9F0418CB00446002620798DF81000E0
:10AF50002079072871D2DFE800F09A04272862716F
:10AF6000900008226946402001F066FB0822A11DDE
:10AF7000684604F0EDFC40B900204B4908700846D3
:10AF800000788DF8110002250DE001204649087077
:10AF9000084600788DF8110008220DF1120168466C
:10AFA00004F0E7FC0A2574E000BF6079042810DD96
:10AFB00000208DF811004C208DF812004F208DF8E4
:10AFC000130043208DF814004B208DF81500062542
:10AFD00024E002208DF8100060798DF811002079AE
:10AFE00002280BD16179502202EB01102F49102267
:10AFF0004B6A0DF11201984712250FE0617950223A
:10B0000002EB0110294910220B6AA11D984710225A
:10B010000DF11201A01D04F0ACFC122539E008224C
:10B020000DF11201402001F007FB03208DF8100004
:10B0300000208DF811000A252BE028E00822A11D30
:10B04000402002F0A5F803F065FD0746A01D02F0C0
:10B0500047FA804615483A460421036C4046984713
:10B0600000208DF811008DF8120008220DF1130157
:10B07000A01D04F07EFC0B250BE000208DF81100D4
:10B080000A4841690DF1120088470E2501E00126AA
:10B0900000BF00BF26B92A4604A9092005F0CAFD51
:10B0A0000CB0BDE8F0810000BC030020B802002015
:10B0B000002106E01E2100BF0A1EA1F1010399B282
:10B0C000FAD1021EA0F1010398B2F3D1704702E059
:10B0D00008C8121F08C1002AFAD170477047002023
:10B0E00001E001C1121F002AFBD1704770B590B07A
:10B0F00004460E461546382D00DD38252A463146D1
:10B1000002A8FDF745F8C5F1380102AA501920221E
:10B11000FDF75EF861208DF8000063208DF80100D6
:10B120006B208DF802002D208DF8030020788DF81B
:10B13000040060788DF80500A0788DF806003A20AC
:10B140008DF807000348402182696846904710B097
:10B1500070BD0000B802002030B591B0044606254D
:10B160002022402101A8FDF733F82A4604F1080106
:10B1700001A8FDF70DF8402201A902A0FFF7B6FFD4
:10B1800011B030BD66756E0070B50546284600F0FA
:10B1900028F8041E00D170BD6178204602F05AFDE7
:10B1A00008B90020F7E70120F5E770B5044600254F
:10B1B00002F098FD051E00D170BD70222146284680
:10B1C000FCF7E6FF02F05EFD06463146284602F037
:10B1D0007DFD0120F0E700B502F05CFD02F066FDA8
:10B1E00000BD70B50646002511E0284602F040FD7E
:10B1F000041E00D10FE00422314604F16000FCF788
:10B20000F9FF10B96570204670BD681CC5B202F028
:10B2100039FDA842E9DC00BF0020F5E700B505F0E4
:10B220009FF905F0A9F901F079F901F083F900BD62
:10B23000704710B50346D3F8A400806868B153F88E
:10B24000A40F806880781C68A468E47840EA042031
:10B25000108053F8A409806810BD0020108000BF42
:10B26000FAE710B5034653F8A40F406880781C68CD
:10B270006468E47840EA0420108053F8A409406828
:10B2800010BD0346D3F8A400006800781080D3F8FE
:10B29000A4000068704770B504460D46E07C50B1CC
:10B2A00000BFD4F8AC10A06C0022CB6A11469847BE
:10B2B00000BF0021E174A078032808D1D4F8A800C9
:10B2C000006920B1D4F8A8000169204688472046CB
:10B2D00007F054F8607830B1D4F8AC00C16820466B
:10B2E00088470020607070BD2DE9F04104460D468E
:10B2F000A078032808D1D4F8A800406920B1D4F878
:10B30000A80041692046884705EB450704F114066B
:10B3100006EB870000210A460B464160028143810B
:10B3200000BF204607F033F8BDE8F0812DE9F04179
:10B3300004460F460125D4F8AC0000221146036BE9
:10B3400004F10B0098470646082E04D0204607F06B
:10B3500028F8BDE8F081E07A00F0600020B12028F4
:10B3600009D0402815D10DE004F10B01204607F06B
:10B37000D7FD05460EE004F10B01204607F030F83A
:10B38000054607E004F10B01204607F0E1FD054604
:10B3900000E000BF00BFC5B9B4F8110018B92046DD
:10B3A00006F0F5FF14E0E07A00F0800048B100BF3D
:10B3B0004C20035B00212046A26C07F0CFF900BFB0
:10B3C00006E0204606F0DAFF02E0204606F0E9FF3C
:10B3D00000BFBEE770B504460D460026287800F091
:10B3E000030020B101282ED002282DD111E0A07831
:10B3F000022802D0032809D100E000BF6888012894
:10B4000003D100212172002070BD00E000BF00BF09
:10B410001BE02E79A078032814D1688890B98EB1EA
:10B42000802E0FD000BFD4F8AC003146826B20468E
:10B43000904700BFD4F8A8002946C268204690472C
:10B440000020E1E701E000E000BF00BF0120DBE7F2
:10B4500070B504460E460125A078022802D00328C4
:10B4600008D103E0207800B9002504E0207800B17D
:10B47000002500E000BF00BF35B901231A46214670
:10B4800004F1440006F09CFF284670BD2DE9F0470A
:10B4900006460D460027B8464FF0010906F1440460
:10B4A000287800F0030020B101284BD0022852D1A7
:10B4B00050E06888070A95F80280102F3FD2DFE835
:10B4C00007F03E08182331323334353E3E3E3E3ECF
:10B4D0003E36781E304951F8203004F108024146CA
:10B4E000304698476060E888402801D108202081D4
:10B4F00026E0781E284951F8203004F10802414620
:10B500003046984760601BE0B8F1060F09DA781EF4
:10B51000214951F8203004F108024146304698474D
:10B5200060600DE000BF00BF00BF00BF08E004F195
:10B53000080241463046FFF77CFE606000E000BF35
:10B5400000BF09E0D6F8A8002946C26830469047F7
:10B55000814601E000E000BF00BF2089C8B1E88853
:10B56000B8B12089E988884201DA208900E0E888BA
:10B5700020812189B6F81100814208DA20892188CA
:10B5800090FBF1F201FB120008B90121F1744FF0B8
:10B5900000094846BDE8F0879400002070B50446D5
:10B5A0000D46A078012804D0022803D0032810D12A
:10B5B00001E00FE00EE0287950B9D4F8A800411C52
:10B5C00001231A4604F1440006F0FAFE002070BD83
:10B5D00000E000BF00BF0120F9E700002DE9F041C5
:10B5E00004460E4635790127307800F0030020B17B
:10B5F000012823D0022845D126E0A078022802D0D5
:10B60000032818D100E000BF207918B10120244997
:10B61000087002E0002022490870207A30B12048EA
:10B62000007840F002001E49087002E000201C492A
:10B630000870002700E000BF00BF24E0A0780328C6
:10B6400001D105B900271EE0A078032819D105F023
:10B65000800080280BD105F07F0000EB400104F151
:10B66000440000EB810080780D49087008E005EB8C
:10B67000450104F1140000EB81008078084908704E
:10B68000002700E000BF00BF37B902231A46044973
:10B6900004F1440006F094FE3846BDE8F081000055
:10B6A000A00000200246012070470246888888B921
:10B6B000C88878B9887800F07F00507090780328A7
:10B6C00008D0507810B10220907001E001209070F5
:10B6D000002070470120FCE770B504460D460126A6
:10B6E000A8782549087008460078012842D8A07833
:10B6F00001283CD0022802D0032839D110E01E488E
:10B70000007858B1D4F8A80042681B480178204658
:10B7100090471948007820700320A070002628E088
:10B720001548007860B9D4F8A800826812480178FA
:10B73000204690471048007820700220A07014E046
:10B7400020780D49097888420FD02178D4F8A800D4
:10B75000826820469047084800782070D4F8A800F6
:10B7600042680548017820469047002601E000E045
:10B7700000BF00BF304670BDA2000020024600207E
:10B78000704770B504460D460026287800F0030087
:10B7900020B1012828D0022827D111E0A078022862
:10B7A00002D0032809D100E000BF6888012803D136
:10B7B00001212172002070BD00E000BF00BF15E034
:10B7C0002E79A07803280ED1688860B95EB1802EEA
:10B7D00009D000BFD4F8AC003146426B20469047F8
:10B7E00000BF0020E7E701E000E000BF00BF01204C
:10B7F000E1E702469078012804D0022803D003280C
:10B800000BD101E00AE009E0087928B98878D2F87C
:10B81000A83058700020704700E000BF00BF012032
:10B82000F9E702460020704710B50346D3F8A4405C
:10B83000E46854F821000478148010BD10B50A485B
:10B8400090F8900000B910BD05F02AFE01200749CC
:10B85000487003F05BF805F03FFE00BF00F06AF8A7
:10B860000028FBD000BFEEE7440400209C4B0020E2
:10B8700070B5124890F8900000B970BD104800787B
:10B8800000B9FAE70E48807800B1F6E70D4806F0F7
:10B89000F9FB0546FCF774FC002407E0FCF766FCA6
:10B8A000C1B2074823300155601CC4B2202CF5DB1F
:10B8B0000348233007F0E6FF00BFDEE74404002022
:10B8C0009C4B00200010004010B50446154890F82D
:10B8D000900000B910BD1448007800B9FAE7134988
:10B8E000086A8047032801DD132060711048007842
:10B8F00080F001000E4908700B480078A0730846DC
:10B90000007808B10320A07207482330084A127853
:10B91000102313FB02011A4604F10F00FCF738FC58
:10B9200000BFD7E7440400209C4B002048030020C0
:10B930008005002030B589B01C208DF80000112052
:10B940008DF801008DF802008DF803008DF80400D9
:10B9500013208DF80500062406E004F15B00C0B258
:10B960000DF80400601CC4B2212CF6DB684605F01B
:10B97000C3FE20208DF80000684605F01FFE202041
:10B980008DF800009DF80600612809D19DF81D0082
:10B99000782805D19DF81E00792801D1012500E005
:10B9A0000025284609B030BD70B51748807B164980
:10B9B000497B00EB012084B2214613480F3001F08F
:10B9C000ADFE1149C978104A927801EB02218842F4
:10B9D00001D0002070BD0C48807A0B49497A00EBF9
:10B9E000012085B20DB90220F4E708494988491EB3
:10B9F000064A0C3202EB01204FF4807202490F31EB
:10BA0000FCF7C6FB0120E5E7D6A90020C8A5002069
:10BA100010B5044644B10121084803F02DF9022174
:10BA2000074803F02BF907E00221054803F024F949
:10BA30000121024803F022F910BD00000008014076
:10BA400000100140194890F87B0020B1174890F889
:10BA50007B0017498870154890F87C00A0B1144805
:10BA60008078022802D1012011498870104880781E
:10BA70001A2802D119200E4988700D488078502864
:10BA800002D14F200A49887009488078002806DDD5
:10BA900007488078054991F87510884204DD012037
:10BAA00003498870002070470120FCE7440400200F
:10BAB000C303002007484078012803DB054840788D
:10BAC000202804DD01200349487000207047012030
:10BAD000FCE70000C3030020114890F87D0020B16E
:10BAE0000F4890F87D000F4948700D4890F881008C
:10BAF00030B10C484078042802DA04200949487023
:10BB000008484078012803DB06484078092804DD0E
:10BB1000012004494870002070470120FCE7000024
:10BB200044040020580800200221084AD170002156
:10BB30009180002006E0064901EB800100220A60A6
:10BB4000411C88B2C828F6DB70470000145F002053
:10BB5000F45B00200146002008E0094A02EB800265
:10BB600001EB80031B681360421CD0B21E28F4DB7B
:10BB70000122034B9B1FDA7000229A80704700005D
:10BB80001A5F002010B50020054948700870087140
:10BB90000449886A8047024948710120C87010BD75
:10BBA000810500204803002010B51A4890F8C40011
:10BBB00000B910BD1848C07B00B9FAE71648407CB0
:10BBC000802800DBF5E7144A517C907C00F02AF8CD
:10BBD0001148407C401CC1B20F484174807C00EB8E
:10BBE00080220E4800EB4200407881420FDB0021AA
:10BBF00009484174007C401CC1B2074801740A29FD
:10BC000005DB0021C1730648816B0120884700BF16
:10BC1000CFE7000044040020DF5B0020E24B00205F
:10BC20004803002070B58AB004460D4620208DF8E8
:10BC30000400274881690DF1050088472449086AF6
:10BC40008047032801DC312000E032208DF8090014
:10BC500000208DF80A008DF80B001D49886C804784
:10BC6000014604EB84221B4810F8120061F31F10F8
:10BC7000C0B28DF8100000208DF8110004EB842173
:10BC8000144800EB410040788DF812008DF81350F5
:10BC900004EB84220F4800EB4200801C00EB0511EE
:10BCA000102205A8FCF774FA1B210DF1090001F020
:10BCB00035FDC0B28DF824000549C86A80470646A4
:10BCC00003483146426B01A890470AB070BD00009E
:10BCD00048030020E24B00202DE9F04190B080465F
:10BCE00020208DF800000DF1010002F071FE00200F
:10BCF0008DF806008DF80700B8F1010F23D100265A
:10BD000018208DF80500704890F87F0080B36F48C8
:10BD10004078002801DD012000E000206B4989788F
:10BD2000002901DD012100E0002100EB410067490D
:10BD3000C978002901DD012100E0002100EB81002C
:10BD40008DF806001AE0052619208DF805005E48DA
:10BD500090F87F0060B15D484078002801DD012047
:10BD600000E0002059498978002902DD012101E025
:10BD700004E0002100EB41008DF8060000259BE067
:10BD80005348C07AA84200D194E0524890F820006D
:10BD900000285CD1002415E005EB4502C2EB8513B9
:10BDA0004B4A0C321A44521C331903EB430302EB87
:10BDB000430002AA052303FB04211A4603F0D9FD20
:10BDC000601CC4B2052CE7DB3F4890F884003328A0
:10BDD0006BD13D4890F88500012866D103F020F929
:10BDE000002862D00424002004EB4401062202EB68
:10BDF00041010DF8010004EB4401072202EB41016F
:10BE00000DF8010004EB4401082202EB41010DF89A
:10BE1000010004EB4401092202EB41010DF801008D
:10BE20001D210DF1050001F079FC0746381204EBE5
:10BE300044010A2202EB41010DF80100F8B204EBC3
:10BE400044010B2202EB41010DF801002DE000241A
:10BE500015E005EB4502C2EB85131D4A0C321A446E
:10BE6000521C331903EB430302EB430002AA0523E0
:10BE700003FB04211A4603F07CFD601CC4B2042CB1
:10BE8000E7DBFF208DF81C008DF81D008DF81E00EB
:10BE90001A210DF1050001F041FC074638128DF81A
:10BEA0001F00F8B28DF8200000BF2946684600F058
:10BEB000BDFF00BF681CC5B20548007AA8423FF725
:10BEC0005FAF10B0BDE8F08144040020D203002031
:10BED000001100209C07002070B588B01C208DF850
:10BEE00000000DF1010002F073FD15208DF8050032
:10BEF000002442E02448C07AA04200D13BE0002563
:10BF000015E004EB4402C2EB84131F4A0C321A44BE
:10BF1000521C05EB450302EB43000DF10602022320
:10BF200003FB05211A4603F024FD681CC5B20A2D47
:10BF3000E7DB164890F88400332817D1134890F8AF
:10BF40008500012812D103F06BF878B100208DF83C
:10BF50001A0016210DF1050001F0E0FB0646301233
:10BF60008DF81B00F0B28DF81C0000BF214668461A
:10BF700000F05CFF00BF601CC4B20348007AA0421E
:10BF8000B8DC08B070BD000000110020440400209F
:10BF90002DE9F04190B0064623208DF800000DF108
:10BFA000010002F015FD16208DF80500012E01D1CB
:10BFB000002000E005208046002569E03848C07A6E
:10BFC000A84200D162E0002417E005EB4502C2EB75
:10BFD0008513334A0C321A44521C08EB040303EB5A
:10BFE000430302EB43000DF10602042303FB04218B
:10BFF0001A4603F0BEFC601CC4B2052CE5DB2948E0
:10C0000090F8840033283CD1264890F88500012818
:10C0100037D103F005F8A0B30424002004EB440159
:10C02000062202EB41010DF8010004EB4401072256
:10C0300002EB41010DF8010004EB4401082202EB80
:10C0400041010DF8010004EB4401092202EB41011A
:10C050000DF801001D210DF1050001F05FFB074601
:10C06000381204EB44010A2202EB41010DF80100F1
:10C07000F8B204EB44010B2202EB41010DF8010080
:10C0800000BF2946684600F0D1FE00BF681CC5B25B
:10C090000348007AA84291DC10B0BDE8F0810000AE
:10C0A000001100204404002010B58AB01548007823
:10C0B00010B900200AB010BD0020124908702020DD
:10C0C0008DF80000104881690DF1010088471A20A1
:10C0D0008DF8050001208DF806000C480068CDF8A9
:10C0E00007000949886A80478DF80B000649086BEC
:10C0F0008047044604482146426B68469047012029
:10C10000D8E70000880500204803002089050020AA
:10C1100010B501201B4908701B48007A1A49C979DB
:10C1200000EB012084B2601C84B220121649C87151
:10C130000846047205F054FF14480078401CC0B251
:10C1400012490870192819DB00200870104890F86F
:10C15000800038B10F48407820B10E484078401E2A
:10C160000C4948700C48807828B90C48806A401CFB
:10C170000A49886202E000200849886205F00EFC46
:10C1800010BD0000F1030020CC070020F2030020C6
:10C1900044040020D0030020F40700209C07002066
:10C1A0007047000010B5012005490870054948682E
:10C1B0008047012801D000F047FD07F06DF810BD61
:10C1C000F0030020DC05002010B50020064988702F
:10C1D000002205210448C01C03F0D6FB00200349BF
:10C1E00081F8200010BD0000F40700209C0700200B
:10C1F0000148807870470000F407002010B500F077
:10C2000039FA03F05BFE07F03BF800F00FFA00F09C
:10C21000D1F903490868804702490868804710BD82
:10C22000DC0500202406002010B500F0CEF903F054
:10C2300077FA05F097FF0548807D28B10020034973
:10C2400088750349C86E804710BD00009C07002018
:10C25000440400200149887070470000F407002062
:10C2600010B50749086A8047032804D00449086AC2
:10C270008047062801D1012010BD0020FCE7000006
:10C28000480300202DE9F04104460D4600260F49E1
:10C290000868804700F06CF9061E05D10B49486814
:10C2A00080470020BDE8F08105F10A0221463046B2
:10C2B000FBF76EFF00F02AF907463946304600F0DA
:10C2C0004BF90249486880470120EBE7B80200209B
:10C2D00000B589B026480078022809D125480178A0
:10C2E0000078401E234A107011B9002020490870C0
:10C2F00000F00CF910B11E48007808B109B000BD7B
:10C3000001201B4908700A201A490870002000F01B
:10C31000DDF81949086005208DF8070001208DF827
:10C3200008000846006800798DF809000846006892
:10C3300040798DF80A0008460068D0F80600CDF86C
:10C340000B0000208DF80F0020208DF810000B4905
:10C35000C86980478DF81100074800680068CDF86B
:10C3600012000F210DF10700FCF7A2FE00BFC5E788
:10C3700008060020090600200406002048030020CB
:10C3800030B5A1B00446402110A8FBF728FF3120AA
:10C390008DF84000E1208DF841002F49C8698047A1
:10C3A0008DF8420017208DF8430002208DF84400DC
:10C3B0002A48006800798DF84500284800684079CF
:10C3C0008DF8460000208DF8470020208DF84800A9
:10C3D00020128DF84900E0B28DF84A00002528129D
:10C3E0008DF84B008DF84C50002C11DD601E1B4A5F
:10C3F00012680A3202EB401120220DF15100FBF7C6
:10C40000C7FE0A201649087002201649087007E086
:10C4100000211248006800F049F800201149087016
:10C4200040216846FBF7DBFEF5208DF80000AA20CE
:10C430008DF801008DF802009DF84000421C10A903
:10C440000DF10300FBF7A4FE07484021826968460E
:10C45000904721B030BD00004803002004060020B2
:10C460000906002008060020B802002010B5044686
:10C470002079022800D010BD60790B49096809793C
:10C48000884200D0F7E7207AE17900EB01202028EC
:10C4900000D0F0E7A17A627A01EB022188B2FFF7BF
:10C4A0006FFF00BFE7E700000406002070B50446F8
:10C4B0000D46FF2084F80A042946034802F046F995
:10C4C0000646304670BD0000F805002010B5044651
:10C4D0002146024802F068F910BD0000F80500206E
:10C4E000002100200CE040F20B424243064B1A446C
:10C4F00092F80A24FF2A01D14A1CD1B2421CD0B2C0
:10C500000428F0DB084670479894002010B50248D4
:10C5100002F060F910BD0000F8050020034804494E
:10C52000086048600020088170470000F005002086
:10C53000F8050020002009E0FF2240F20B414143B2
:10C54000044B194481F80A24411C88B20428F3DB07
:10C55000704700009894002070B504460D462A46A6
:10C560002146024802F03AF970BD0000F8050020AB
:10C57000002118E040F20B4048430D4A104490F867
:10C580000A04FF280DD1012240F20B404843084B1A
:10C59000184480F80A2440F20B4048431A461044DD
:10C5A0007047481C81B20429E4DB0020F8E7000052
:10C5B0009894002010B503F0E1F805F0FBFD02F0BF
:10C5C00099FE012000F0F0F910BD00B591B0684669
:10C5D00004F0E0FC08B911B000BD9DF8010060282E
:10C5E00003D09DF80100612809D19DF8020030B107
:10C5F00002F0DCF99DF80210884200D0EBE704F06D
:10C60000B5FF9DF80100602803D1684604F000FAE8
:10C610000AE09DF80100612803D1684604F05CFB44
:10C6200002E0684604F0A0FC00BFD4E710B504F0B7
:10C63000CBFC05F0CBFD10BD70B5C0B005460E4675
:10C640001446601CC2B20A486946436A28469847A5
:10C650009DF80000F52808D1224631460DF1010071
:10C6600003F087F9012040B070BD0020FBE7000017
:10C67000B802002010B5C0B00D226946C020FFF7F7
:10C68000DBFF88B10D22BA49684603F072F90D222A
:10C69000B849684603F06DF9B7480C21D0F80C2171
:10C6A000B448401C904710E00120B149491E487031
:10C6B00000220C21AE48401C03F066F9AE480C2164
:10C6C000D0F80C21AB48401C9047FFF705FA032235
:10C6D00069464FF48560FFF7AFFF80B10322A74999
:10C6E000684603F046F9A54A521ED378927803EBC8
:10C6F000022290B2A04AD2F80411884704E09E4872
:10C70000D0F8041100208847072269460020FFF76F
:10C7100093FF28B107229A49684603F02AF91EE0E0
:10C720000121974A521E5170917011460979D278B1
:10C7300001EB022188B201200112914A521ED170F0
:10C74000114608718979527901EB022188B20120E2
:10C7500001128B4A521E51711146887100BFFFF7BA
:10C76000A9F9FFF76FF90D2269460820FFF764FF6A
:10C7700028B10D228349684603F0FBF805E0FF224B
:10C7800006218048C01C03F0FFF805F06FFA042270
:10C7900069461820FFF750FF28B104227A496846FD
:10C7A00003F0E7F804E0FF220421774803F0ECF8F7
:10C7B000062269463020FFF73FFF28B10622734961
:10C7C000684603F0D6F80AE000207049491E487018
:10C7D0004870C87008710A204871082088711A22B0
:10C7E0006946A020FFF728FFE0B11A226849684691
:10C7F00003F0BFF8604890F8C400C0B16448401E20
:10C8000080780E2813D16248401EC07814280ED1BB
:10C810005949D1F8D400804748B901205D4981F8D1
:10C82000200004E000221A21594803F0ADF8082244
:10C8300069464020FFF700FF60B100205549888518
:10C840009DF80000402811D0684600F049FE51498B
:10C8500088850BE00924224669464F4803F089F891
:10C8600022466946402000F093FC00BF042269463E
:10C87000D020FFF7E1FE28B104224849684603F0C2
:10C8800078F804E000220421444803F07DF80322F4
:10C890006946D820FFF7D0FE28B1032240496846F8
:10C8A00003F067F806E001203D49491E487000206A
:10C8B0008870C87006226946F020FFF7BDFE48B3B5
:10C8C00006223849684603F054F82B4890F8820055
:10C8D00028B1294890F882003249491E88703148B1
:10C8E000401E807820B12F48401E8078042803DD48
:10C8F00001202C49491E88702A48401EC0782049D2
:10C90000491E8978884219D01D49491E887805F04A
:10C9100041FA13E0184890F8820030B1164890F8B8
:10C9200082002049491E887003E001201D49491EEC
:10C9300088701349491E887805F02CFA012269464F
:10C940004FF4A070FFF778FE20B19DF80000114968
:10C95000C8750AE0084890F8850018B101200D4913
:10C96000C87502E000200B49C87540B010BD00003A
:10C97000590800206708002044040020DF0300203D
:10C98000C40300204B080020CC030020CD0700206A
:10C99000F50700209C070020D0390108BE030020C5
:10C9A000D3030020D703002001490870704700001E
:10C9B000F410002030B58BB000F02AFE08B10BB0A7
:10C9C00030BD02F097FC20208DF804000DF1050029
:10C9D00001F0FEFF10208DF8090001F0E7FF8DF84F
:10C9E0000A00A5208DF80B0001F0ECFF8DF80C007B
:10C9F000554840798DF80D00534880798DF80E0028
:10CA000008220DF10F01514802F0B3FF4F48401EBC
:10CA1000C07800F00F008DF8110001F0CDFF022862
:10CA200003D001F0C9FF052805D19DF8110040F0A1
:10CA300080008DF811004648007820B1012815D0FB
:10CA4000022837D120E001208DF817000C2206A91A
:10CA5000404802F08EFF404890F884001E2801D123
:10CA6000012000E002203A49087027E003208DF8F9
:10CA70001700092206A9394802F07BFF34480078E4
:10CA8000401C3349087019E002208DF81700344823
:10CA900040788DF818003348007A8DF81900042288
:10CAA0000DF11A012F48001D02F063FF00202849F4
:10CAB000087003E000202649087000BF00BF002472
:10CAC00035E02848C07AA04200D12EE002F01AF8E2
:10CAD00020B12448001D005D8DF80C001E4890F820
:10CAE00084001E280CD01C4890F88400332817D1ED
:10CAF000194890F88500012812D102F091FA78B116
:10CB00001A210DF1090000F009FE054628128DF8E2
:10CB10002300E8B28DF8240020208DF8040000BF27
:10CB2000214601A800F082F900BF601CC4B20D4884
:10CB3000007AA042C5DC03200B4908700020487031
:10CB4000887000BF3BE70000C3030020CD07002032
:10CB5000E90300205A08002044040020A90700200F
:10CB6000D603002000110020F410002010B588B07A
:10CB70001F208DF80000134881690DF101008847DE
:10CB800010208DF8050001F011FF8DF80600182225
:10CB90000DF107010C4802F0ECFE002405E02146EF
:10CBA000684600F043F9601CC4B20848007AA0420D
:10CBB000F5DC03200649087000204870887008B032
:10CBC00010BD000048030020DC07002000110020F9
:10CBD000F410002030B589B004461F208DF8040001
:10CBE000154881690DF10500884733208DF809004B
:10CBF00034B917220DF10A01104802F0BAFE05E01F
:10CC000017220DF10A010E4802F0B3FE01F0DAFE20
:10CC10008DF8230001F07CFF0546294601A800F0AD
:10CC200005F903200749087008464078401C487001
:10CC30000020887009B030BD480300203308002070
:10CC400075080020F410002010B503F095F8724824
:10CC5000007800B910BD70480078082872D2DFE86B
:10CC600000F0D70412153A576AAC01F0A5FE03286C
:10CC700006DD6A4890F87A0010B100F037F901E05B
:10CC8000FFF798FEC5E000F031F9C2E06248807815
:10CC9000401CC0B2604988700A2813DA5F48D0F897
:10CCA000F410012088475D48007850B101F084FEFF
:10CCB000082803D001F080FE092802D157490869ED
:10CCC0008047A6E05548D0F8F4100020884704209B
:10CCD000514908709DE001F06FFE032805DCFFF765
:10CCE000FBF806204C49087011E001F065FE0328AE
:10CCF00007DD4A4890F87A0018B10120FEF7ECFFF2
:10CD000002E00120FFF744F905204349087080E064
:10CD100001F052FE032807DD404890F87A0018B170
:10CD20000220FEF7D9FF02E00220FFF731F90620CA
:10CD3000394908706DE003F039F93949886880474E
:10CD400008B187E764E004F0C1F840B1002032493F
:10CD50004872087233484860072008702CE02F485A
:10CD600090F8340068B12D49486C804748B10020E4
:10CD70002949487208722948C06B4860072008702A
:10CD80001AE001F019FE032803DD244890F87A0028
:10CD900048B921484078022805DB00201E49487028
:10CDA000FFF708FE08E002F085FF10B900F09EF8DA
:10CDB00002E00020FFF7F8FD2BE0174948688047A4
:10CDC00070B11548407A401C134948720846407AB1
:10CDD00050281CDB0120144908700F49087016E028
:10CDE0000D49097A491C0C4A11720C4991F88410BA
:10CDF0001E2901D1142000E050200749097A814200
:10CE000004DB0121084A1170034A117000BF00E0E1
:10CE100000BF00BF00BF1DE7F41000204404002045
:10CE200024060020CD0E0108E903002030B591B0A2
:10CE300005460C462878401CC2B26946284602F0D6
:10CE400098FD124890F87E0060B19DF80000001F28
:10CE5000C0B28DF800009DF800200DF10101081D01
:10CE600002F087FD0A49085D04F018FE0748D0F873
:10CE7000A410684688470648025D9DF800100548E2
:10CE8000836A0DF10100984711B030BD44040020C1
:10CE900000110020B802002010B590B00446F52023
:10CEA0008DF80000AA208DF801008DF8020020788E
:10CEB000401CC2B20DF10301204602F05AFD9DF85C
:10CEC0000320D21CC2F14002D1B29DF803206B4670
:10CED0001A44D01C002202F057FD03484021826909
:10CEE0006846904710B010BDB802002030B58BB036
:10CEF00000F0A6FB08B10BB030BD02F0FBF9994879
:10CF0000D0F8D01000208847012800D1F3E700F0C6
:10CF100095FD95484079401C9349487108464079F1
:10CF2000072801DD002048718F48407980B98F487B
:10CF3000007880F001008D4908700846007838B903
:10CF40008B498868804718B1072087494871D2E724
:10CF500088498868804710B107208349487186490D
:10CF60004868804710B107207F4948717D4890F894
:10CF70007F0040B17B4890F87F0000287ED07F483A
:10CF8000C0780028FAD020208DF804000DF10500AB
:10CF900001F01EFD01F010FD032801DC132000E06C
:10CFA00014208DF8090001F007FD032806DD6D4807
:10CFB00090F87A0010B117208DF809007048C079F8
:10CFC0008DF80A006E48007A8DF80B001A2203A92A
:10CFD0006C4802F0CEFC6348007878B101F0ECFCBC
:10CFE000082803D001F0E8FC092807D16548401E55
:10CFF000807840F040008DF80D0006E06148401E4A
:10D00000807820F040008DF80D005648016A01A894
:10D01000884720B15349D1F8B000804778BB01F070
:10D02000CBFC032841DD4F4890F87A0040B317202D
:10D030008DF8090004220DF121014B48401C02F03B
:10D0400098FC494840798DF8200001F0B5FC05288E
:10D0500001D1012000E000204349497808438DF8C0
:10D060002100414880788DF8220001F0ABFC8DF85A
:10D0700023003C4890F88400282802E067E01BE089
:10D0800013E004D0374890F88400292808D11B21E8
:10D090000DF1090000F042FBC0B28DF824000BE056
:10D0A000314800798DF8240006E0A5208DF8210094
:10D0B00001F088FC8DF82200002444E03248C07A58
:10D0C000A04200D13DE001F01DFD20B12E48001D21
:10D0D000005D8DF82200234890F884001E280CD0B3
:10D0E000204890F88400332817D11E4890F8850016
:10D0F000012812D101F094FF78B11A210DF1090035
:10D1000000F00CFB054628128DF82300E8B28DF8DC
:10D11000240020208DF8040000BF9DF80D0058B1B8
:10D120009DF80D0000F0800018B920208DF8040053
:10D1300002E020208DF80400214601A8FFF776FECA
:10D1400000BF601CC4B21048007AA042B6DC0320C5
:10D150000E49087008464078401C487000208870CE
:10D1600000BFC8E644040020BD030020EE030020F9
:10D1700024040020DC05002038040020D203002015
:10D18000CC070020F507002000110020F41000203B
:10D1900070B5C0B006460C461546F5208DF8000067
:10D1A0002A460DF10101204602F0E3FB681CC2B2E1
:10D1B00003486946036A30469847012040B070BD75
:10D1C000B80200200348407808B1012070470020D1
:10D1D000FCE700002C43002000200349487003496D
:10D1E00008800349088070472C4300206805002010
:10D1F0006A05002030B59BB037484078082866D2D1
:10D20000DFE800F065040D10393D575B324AD078F5
:10D21000324A516B8847FF202F49487058E0FFF78A
:10D22000DBFF55E02C4800892B49C98800EB012120
:10D230002B480088401C80B2294A1080814200DCC3
:10D2400046E020208DF84400002403E011A8045596
:10D25000601CC4B2202CF9DB2249C86A804705460D
:10D2600020482946426B11A890471B4A907A1B4AD6
:10D27000D16888472CE000201B49088028E09DF8F1
:10D280000400202801D01BB030BD9DF8050000B17E
:10D29000F9E79DF80600012800D0F4E79DF80700A3
:10D2A000022800D0EFE710480088401C0E49088093
:10D2B0000EE000200D4908700AE00D48007800B922
:10D2C00006E00649886B80470849087000E000BF07
:10D2D00000BF00BFD7E700002C430020B8020020A9
:10D2E00068050020480300206A0500206C05002026
:10D2F0006D050020114A4368136003899380837A87
:10D300009371521E52780A700C4A521E92784A70DB
:10D310000A4A521E12798A70094A12881212CA7079
:10D32000074A12780A71074A128812124A71054A8E
:10D3300012788A71044A1278CA7170472D4300200E
:10D34000680500206A0500206C050020002107E028
:10D3500048F2782100BF0A1EA1F1010399B2FAD167
:10D36000021EA0F1010398B2F2D17047002105E03E
:10D370001E2100BF0A1EA1F10101FBD1021EA0F176
:10D380000100F5D17047002105E01E2100BF0A1EF3
:10D39000A1F10101FBD1021EA0F10100F5D17047FE
:10D3A00010B504464FF4C8714FF4E150FBF70CFE82
:10D3B00010BD000070B586B00446002002900390B6
:10D3C000049005903D48006801900126E0780B2804
:10D3D00004D00C2808D00D2864D15DE03848A1881D
:10D3E0000180A17981705FE02079012802D0207945
:10D3F000022827D1A079802800DB55E02079401E43
:10D40000C5B2217905EB85222D48C01C00F8121009
:10D4100000F6FD708574617905EB8522A0F6FD703C
:10D4200000EB4200417005EB85222549C91C01EB48
:10D430004201891CA27901EB02101022E11DFAF7CA
:10D44000A7FE28E0207900F0800020B3A079802892
:10D4500000DB29E0207920F08000401EC5B205EBFA
:10D4600085211748C01C00EB410040788DF805006D
:10D47000A0798DF8060005EB85221148C01C00EB51
:10D480004200801CA27900EB021110220DF107006E
:10D49000FAF77EFE132607E00A4861680160A1687A
:10D4A000416001E0002600BF00BF2EB1E1783346A5
:10D4B00001AA602005F064FD06B070BD203A0108A5
:10D4C000DF4B0020E65B0020014604488078401EC8
:10D4D000132202EB4010C0B27047000018940020E5
:10D4E00010B5024600230024002108E0505C1844D7
:10D4F000C3B2081D105C2044C4B2481CC1B2042948
:10D50000F4DB83F0A50384F0A50403EB042080B2D0
:10D5100010BD0000014601F10800C0B20246044BF4
:10D5200093F87530984201DD012070471046FCE702
:10D530004404002010B50146132901DC012012E04B
:10D54000A1F11303D81703EBD0604011401C1A4619
:10D55000D41702EBD4646411A2EB44140CB101247F
:10D5600000E000242044C0B210BD014609B90020EB
:10D5700003E0481E132202EB4010C0B2704702467F
:10D580001320704710B501460020002314E04FF629
:10D59000FF7404EA83028C5C4CB9541C0C5D34B9F2
:10D5A000941C0C5D1CB9D41C0C5D04B902E0441C35
:10D5B000E0B200BF5C1CA3B20A2BE8DB10BD000088
:10D5C0000C480078401CC0B20A490870FA2801DAF9
:10D5D00000207047002007490870084640782D2831
:10D5E00003DB002048700120F3E700200149487068
:10D5F0000220EEE7810500200448007820B10348AE
:10D60000007908B1012070470020FCE77005002078
:10D6100010B501F077FA08B9002010BD074800786E
:10D6200080F00100054908700846007818B1FFF73E
:10D630009DFA0120F1E70020EFE70000EA03002057
:10D6400010B5244890F8210080B32348007880F07A
:10D6500001002149087048B31E4890F82300A0B18A
:10D660001C4890F8240080B11C48007818B90020AC
:10D67000FFF7B0FA02E00120FFF7ACFA1748007894
:10D6800080F00100154908700EE0124890F8230060
:10D6900018B10020FFF79EFA06E00E4890F824002B
:10D6A00010B10120FFF796FA012010BDFFE70948ED
:10D6B00090F8220060B10A48807848B900200549F6
:10D6C00081F8220081F8210081F8230081F82400EC
:10D6D0000020EAE79C070020EC030020ED03002077
:10D6E000F40700200020014908707047D805002089
:10D6F0000246002107E00748405C904201D10846FD
:10D700007047481CC1B20348407A8842F3DCFF20CE
:10D71000F6E70000001100207047000070B50246D7
:10D7200000201CE003134FF6FF7404EA0010147885
:10D73000E51704EB157583EA25150C4E36F81550E0
:10D74000684003134FF6FF7404EA0010147804F0E5
:10D750000F045C40354635F814406040521C0C1EE6
:10D76000A1F10105A9B2DDD170BD0000243D010881
:10D770007047000070B505460E46D5F8B040012E42
:10D7800018D12078F52805D16078AA2802D1A07890
:10D79000AA2802D02046FFF7BFFF002004F0ACFA11
:10D7A0000548C16CE01C88474023224601212846D9
:10D7B00004F051FF70BD00004803002070B504461E
:10D7C0000D468121204604F0CFFE0121204604F0C1
:10D7D000CBFE002070BD000070B504460E4643210C
:10D7E0001B48FAF7FCFC1B4B4FF4A07200212046AB
:10D7F00004F020FF174BDB1D4FF480720021204600
:10D8000004F018FF4023124A0121204604F023FFB0
:10D8100011488169C4F88810C169C4F884100C48A3
:10D82000C4F8B000D4F8B40078B100250BE0D4F807
:10D83000B40050F8250020B1D4F8B41051F82500F8
:10D840008047681CC5B2042DF1D3002070BD0000D4
:10D8500058070020D10000208C020020024619B198
:10D86000C2F8B410002070470220FCE770B50646ED
:10D870000C4615462B4622468121304604F06EFFA9
:10D88000002070BD2DE9F04105460C460127D5F872
:10D89000B06060780C2865D2DFE800F0642D394371
:10D8A00064640664644D595F60882221B1EB202FC7
:10D8B0000ED1E088202801D9202000E0E08802462F
:10D8C00000232B4905F1440004F07EFD002711E000
:10D8D00060882121B1EB202F0CD1E088092801D9E3
:10D8E000092000E0E08802460023224905F14400B7
:10D8F00004F06AFD37E0E088022807D10023022205
:10D90000314605F1440004F05FFD00272BE00023C1
:10D91000012206F1410105F1440004F055FD002704
:10D9200021E00023012206F1420105F1440004F048
:10D930004BFD002717E0A07886F84000E28800231E
:10D94000314605F1140004F03FFD00270BE060882C
:10D95000001286F84100002705E0A07886F8420012
:10D96000002700E000BF00BF3846BDE8F08100009E
:10D970004C390108C80000202DE9F04105460E464B
:10D9800090461A490868C11700EBD1614911184A3D
:10D99000116010460068801D16490860102001F0D3
:10D9A000A1FF074610213846FAF719FC002403E0CE
:10D9B000305D11490855641C0D480068B4EB800FB8
:10D9C000F6DB002403E0285D0C490855641C102C8C
:10D9D000F9DBFBF7F3FEFBF759FD10220849384647
:10D9E000FAF7D6FB3846BDE8F08100004806002073
:10D9F000440600204006002051AC0020E5AA00208B
:10DA0000F5AA002010B50A48007978B9084890F8BE
:10DA1000060858B900210748C1730749886E804736
:10DA20000548816B01208847012010BD0020FCE7DC
:10DA3000DF4B0020DF5B00204803002010B50C48BE
:10DA40000078401CC0B20A4908700A280ADD08465E
:10DA500000780C2801DD002008700648816D012047
:10DA6000884703E00348816D0020884710BD00000F
:10DA7000EB030020B80200202DE9F04104462CB948
:10DA80000F488178001D00F089F816E001F042F897
:10DA900006460B4991F863002146FFF770FD0746E3
:10DAA0002046FFF762FD01460548801D0D18054818
:10DAB00032463946836A28469847BDE8F08100001F
:10DAC00018940020B802002070B50446A01CFDF791
:10DAD00088FB051E0CD0B5F86C606978284600F00C
:10DAE000B9F820B1627AA11C012000F01BF900BF37
:10DAF00070BD000030B59DB0054668781E490978B4
:10DB0000884201D11DB030BD68781B4908700224DD
:10DB100000BF285D052800DA2AE0285D401FC0B25A
:10DB20008DF86300601C284400681990601D285C13
:10DB30008DF868005D210DF10600FAF750FB9DF8A5
:10DB40006320A01D29180DF10600FAF721FB00F053
:10DB50009FFF1B900020ADF8700001A8FDF768FB47
:10DB600001A8FDF722FB285D401C044400BFD0E75C
:10DB700000BF00BFC6E70000D805002000B5ADF229
:10DB8000044D0548416801A8884710B101A8FFF776
:10DB9000B1FF0DF2044D00BD14040020F0B589B0B2
:10DBA00004460D4624216846FAF719FB20208DF81B
:10DBB0000000264881690DF10100884737208DF863
:10DBC000050094F8600001066120005D01EB004152
:10DBD0006220005D01EB00216320005D084418B164
:10DBE000206ECDF8060002E00020CDF806008DF88A
:10DBF0000A5094F864008DF80D0094F85F0000213D
:10DC0000FFF7BDFC07463A46A11C0DF10E00FAF7DE
:10DC1000BFFA2846FFF758FC07463946A01CFFF715
:10DC20007DFD064630128DF80B00F0B28DF80C0029
:10DC300000F070FF07469DF8001005483A46836AD9
:10DC40000DF10100984709B0F0BD00004803002025
:10DC5000B802002070B504460D46FF20207029460A
:10DC6000024800F073FD0646304670BDCC0500202A
:10DC700010B504462146024800F096FD10BD000094
:10DC8000CC05002010B5024800F0A4FD10BD000036
:10DC9000CC05002003480449086048600020088142
:10DCA00070470000C4050020CC050020002008E0DB
:10DCB000FF21C0EBC002044B03EB02121170411CA8
:10DCC00088B26428F4DB70475868002070B50446B9
:10DCD0000D462A462146024800F080FD70BD000036
:10DCE000CC050020002116E0C1EBC1000C4A02EB7C
:10DCF00000100078FF280CD10120C1EBC102084BB5
:10DD000003EB02121070C1EBC1001A4602EB0010C7
:10DD10007047481C81B26429E6DB0020F8E7000068
:10DD20005868002070B590B006460C4615460EB1F6
:10DD3000022000E001208DF800002068CDF80100ED
:10DD40000020ADF805008DF807008DF80850092176
:10DD50006846FBF7ADF910B070BD000070B54948DA
:10DD6000806F401C474988670024084690F874007B
:10DD700020B1012835D002286FD16FE0FFF782FF74
:10DD800010B9FFF7FBFE7AE000253E49487800F025
:10DD90003DFC051E0DD1FFF775FF3A494978491C36
:10DDA000C9B2384A5170884202DC002011464870DE
:10DDB00065E070213348001DFAF711FA70222946F8
:10DDC0003048001DFAF7E4F900202E49C87091F898
:10DDD0006300FFF7AFFB2B498870012081F87400C6
:10DDE00000BF2849C878FFF747FE2648C078401C86
:10DDF000C0B22449C870897888422CDB214890F849
:10DE00007C00401CC0B21F4981F87C000A280FDB4F
:10DE1000002081F87C000124022081F874001A4857
:10DE2000816B022088470C20164981F87D0013E0A1
:10DE3000FFF728FF13494978491CC9B2114A5170AC
:10DE4000884202DC002011464870012400200D4960
:10DE500081F8740000E0012411E00FE00224094879
:10DE600090F87D1090F87D00401E064A82F87D00F3
:10DE700019B90020114681F8740000E000BF00BF0E
:10DE8000204670BD189400204803002033B581B0AF
:10DE90000D460122694601A8FBF7BCFA044614B9F5
:10DEA0009DF800003EBD0020FCE72DE9F04104464E
:10DEB0000D4616469846324629462046FBF7AAFAF2
:10DEC000074617B90120BDE8F0810020FBE70021DB
:10DED00007E048F2782100BF0A1EA1F1010399B2C0
:10DEE000FAD1021EA0F1010398B2F2D170470000EE
:10DEF0002DE9F04105460E4619490868C11700EBA7
:10DF0000D1614911174A116010460068801D1649F9
:10DF10000860104600688700102001F0E3FC80468E
:10DF200010214046FAF75BF9002403E0305D0F4909
:10DF30000855641CBC42F9DB002403E0285D0C4951
:10DF40000855641C102CF9DBFBF738FCFBF742F892
:10DF5000102208494046FAF71BF94046BDE8F08117
:10DF600048060020440600204006002051AC002056
:10DF7000E5AA0020F5AA002070B52148807908B9EB
:10DF8000002070BD1E4A9288152A01DC012217E08C
:10DF90001B4A9288A2F11501CA1701EBD2625211F5
:10DFA000521C174B9B88A3F11500C31700EBD363DA
:10DFB0005B11A0EB43130BB1012300E000231A44D3
:10DFC000D5B21049C86E804740F080040D48016FFB
:10DFD0002046884700F01AF80B49D1F880008047A6
:10DFE000012408E0204600F07DF80749D1F88000C0
:10DFF0008047601CC4B2AC42F4DB0120C1E70000E2
:10E000001C04002048030020B802002030B589B06D
:10E0100024216846FAF7E3F820208DF800002E4806
:10E0200081690DF10100884734208DF805002B4AE5
:10E030009288152A01DC012217E0284A9288A2F171
:10E040001501CA1701EBD2625211521C234B9B8857
:10E05000A3F11500C31700EBD3635B11A0EB4313CF
:10E060000BB1012300E000231A44D2B28DF8062040
:10E070009DF80620521E152303EB421291B2174A57
:10E080001268101DFFF74AFB044620128DF80700A6
:10E09000E0B28DF808001049886C80478DF80900BF
:10E0A00000208DF80A008DF80B000C480068011D57
:10E0B000152203A8FAF76CF80948816F00208847F9
:10E0C0000549C86A8047054603482946426B6846A9
:10E0D000904709B030BD0000480300201C04002018
:10E0E000B80200202DE9F0418AB00446242101A89D
:10E0F000FAF775F820208DF80400294A9288152A2D
:10E1000001DC012217E0264A9288A2F11501CA1704
:10E1100001EBD2625211521C214B9B88A3F11500D6
:10E12000C31700EBD3635B11A0EB43130BB10123C7
:10E1300000E000231A44D5B20CB9002003E0601EB1
:10E14000152101EB4010C6B20CB915210EE0691E75
:10E15000A1420AD112498988A1F11500C11700EB2B
:10E16000D1614911A0EB411100E02021CFB20C4850
:10E170000068001D81193A460DF10500FAF708F80C
:10E180000848816F002088470749C86A8047804651
:10E1900005484146426B01A890470AB0BDE8F081AE
:10E1A0001C040020B802002048030020F0B50146FE
:10E1B0000120264AD07110460160C8788A7800EBA9
:10E1C000022080B2214A90801646B688152E01DCC6
:10E1D000012617E01D4EB688A6F11502D61702EBF0
:10E1E000D6667611761C194FBF88A7F11500C717A0
:10E1F00000EBD7677F11A0EB47170FB1012700E0B5
:10E2000000273E44F3B200201CE008B9002203E0DE
:10E21000421E152606EB4212D4B208B915260EE0AE
:10E220005E1E86420AD1094EB688A6F11502D6179F
:10E2300002EBD6667611A2EB461600E02026F5B278
:10E24000421CD0B29842E0DBF0BD00001C0400206C
:10E2500010B50748807900B910BD0649C86E8047DF
:10E2600040F080040348016F2046884700BFF3E771
:10E270001C0400204803002070B5044610480068C4
:10E2800000B970BD7CB90E48807960B100200C499E
:10E29000086088710B49C86E804720F080050948E6
:10E2A000016F28468847012C08D10548C07901280C
:10E2B00004D100200249C8710120887100BFE0E745
:10E2C0001C0400204803002010B52C4B1B6883431E
:10E2D0002A4C2360231D1B688343241D2360231DB8
:10E2E0001B688343241D2360231D1B688343241D57
:10E2F000236011B101290ED105E0204B1B680343B7
:10E300001E4C236008E01D4B1B1D1B6803431B4C68
:10E31000241D236000E000BF00BF22B1012A0FD0FE
:10E32000022A27D119E0154B08331B680343134C0D
:10E3300008342360231D1B688343241D23601AE0D7
:10E340000E4B08331B6883430C4C08342360231D99
:10E350001B680343241D23600DE0084B08331B6832
:10E360000343064C08342360231D1B680343241D0C
:10E37000236000E000BF00BF10BD000000040140AA
:10E380000149086070470000140401400146074835
:10E39000006800EA010205481438006800EA010339
:10E3A00012B10BB1012070470020FCE714040140BA
:10E3B0000448006820B103480068401E0149086015
:10E3C00070470000340400200348006808B10120B1
:10E3D00070470020FCE70000340400201CB5044610
:10E3E00020791D2817D1607908B90A2000E06079EA
:10E3F0000949086008460068322148430649086018
:10E4000020798DF8000060798DF8010002226946BC
:10E410000B2002F00FFC1CBD3404002070B5044634
:10E420006079282819D1A07900B970BD012015495B
:10E430000870607A217A00EB012012494880A079A7
:10E44000012802D10020487002E051200D49487097
:10E450000D49D1F8A000804712E00A48007878B151
:10E460000020084908700949C86A804705460749DD
:10E47000886A8047064606482946C26A3046904761
:10E4800000BFD2E7700500204404002048030020AC
:10E49000B802002070B504462848007808B900206A
:10E4A00070BD27480078B8B92649C86A8047054634
:10E4B000224948782449CA6A294690470120A07217
:10E4C0002049886A8047E0721C4840880012207307
:10E4D0001A488078607323E01A49C86A8047064664
:10E4E0001849886A8047054617483146C26A284657
:10E4F0009047164890F87A0068B10120A07211493F
:10E50000886A8047E0720D484088001220730B48EB
:10E510008078607304E00020A072E0722073607362
:10E520000A48D0F89C10204688470548007880F0BB
:10E530000100034908700120B2E7000070050020C7
:10E540007605002048030020B80200204404002083
:10E5500008B50F208DF80000044800798DF80100FF
:10E56000022269460B2000F003F808BD7005002068
:10E5700070B590B004460D46164640216846F9F73E
:10E580002EFE1F208DF80000E1208DF801000949C2
:10E59000C86980478DF802008DF80340324629464D
:10E5A00001A8F9F7F5FD0348416C6846884710B0AB
:10E5B00070BD0000480300204179014A1171704785
:10E5C00070050020014800787047000070050020A9
:10E5D00001460D48007808B9002070470A48408875
:10E5E00000280EDD48780A7800EB0220064A52889F
:10E5F000904206D104484088401C034A50800120C4
:10E60000EBE70020E9E700007005002070B5054643
:10E6100000242846FFF72CFB041E25D000F038FA12
:10E62000A16E884204D300F033FAA16E401A03E0D1
:10E6300000F02EFAA16E081A0646B6F5487F0DD3F3
:10E6400004F16000FCF7A0FD30B194F8642004F1FF
:10E6500060010020FFF766FB002070BDB4F86C007D
:10E66000401CA4F86C0000BF2046F6E710B5002857
:10E6700021D0114B0022001F196803E0814203D80A
:10E680000A4649680029F9D152B11368841A9C429C
:10E6900004D1006818441060104602E0506000E0A9
:10E6A000186039B102680B1A934203D10B681A44FF
:10E6B00002604968416010BD940600207FB50446A1
:10E6C00026796579B54200DD7FBD012D01DB142D72
:10E6D00000DDF9E7012D03D1A9021A48F9F77FFD02
:10E6E000691E01EB011101EB4101164A8818332222
:10E6F00004F10801F9F74CFD20798DF800006079EC
:10E700008DF80100A0798DF80200E0798DF8030002
:10E71000B54211D10B480078012802D0032809D155
:10E7200003E0084801F080F805E007480168054863
:10E73000884700E000BF00BF0421684602F09AFA53
:10E7400000BFC1E7283F0020240400202DE9F0414C
:10E7500004460E461349086880472089B04205DA0E
:10E760001049486880470020BDE8F08125680020F6
:10E7700002E06D68411C88B2B042FADB6F686868DD
:10E7800040686860D7F800803846FFF76FFF20893F
:10E7900010B12089401E20810249486880474046C8
:10E7A000E2E70000B802002010B502460B461089CF
:10E7B000984201DA002010BD10684168002002E094
:10E7C0004968441CA0B29842FADB09B10868F2E734
:10E7D0000020F0E701460889704700002DE9F0416C
:10E7E0000546884617461749086880472889B84271
:10E7F00005DA1449486880470020BDE8F081082008
:10E8000001F070F8044604E00E4948688047002093
:10E81000F3E7002CF8D000206060C4F800802E6878
:10E8200000BF02E07668411C88B2B842FADB70682B
:10E83000606074602889401C2881024948688047CC
:10E840000120DAE7B80200200146888870470000FE
:10E850002DE9F04104460E46144908688047208897
:10E860006188884206D1A088A189884202DB4FF0E6
:10E87000FF3515E06388E789A16803FB07103A4676
:10E880003146F9F785FC6088401CA18990FBF1F2C4
:10E8900001FB12006080A088401CA080A08805B207
:10E8A0000249486880472846BDE8F081B802002048
:10E8B0002DE9F04104460E46134908688047208838
:10E8C0006188884204D1A08810B94FF0FF3515E067
:10E8D0002388E789A06803FB07013A463046F9F729
:10E8E00057FC2088401CA18990FBF1F201FB12002B
:10E8F0002080A088401EA080A08805B202494868F8
:10E9000080472846BDE8F081B802002010B52021DC
:10E910001448F9F764FC2022134912482030F9F713
:10E9200037FC00240AE00F482030005D0F49095DE4
:10E9300048400C4920310855601CC4B2202CF2DB41
:10E940000023084A3032074901F12000FAF75AFC47
:10E950000023044A2032A2F1100101F12000FAF74D
:10E9600051FC10BD9F4B0020D9390108243A010801
:10E9700001460148405C7047243B010810B504463D
:10E98000202202492046F9F703FC10BDBF4B0020AE
:10E99000044890F8900008B90020704702480078B9
:10E9A000FBE70000440400209C4B00200148407815
:10E9B00070470000C3030020014840787047000002
:10E9C000580800200148007970470000001100201D
:10E9D00010B504460B484078032803D00948407816
:10E9E000062808D1AA202070BB206070CC20A0701F
:10E9F000DD20E07004E004222146034800F0B9FF66
:10EA000010BD000058080020CC0300200148007809
:10EA100070470000F410002017488078282803D1A0
:10EA200004201649C87224E01348807810280FD1BA
:10EA30001248C07A032807D01048C07A022803D0B1
:10EA400002200E49C87214E003200C49C87210E07D
:10EA50000948807818B101200849C87209E00648C1
:10EA6000807818B905200549C87202E000200349E2
:10EA7000C8720248C07A7047F40700209C07002043
:10EA80000421017002214170002181707047000053
:10EA90000148806F704700001894002010B50548A9
:10EAA00090F8740020B9FFF7EDF808B9002010BD08
:10EAB0000120FCE7189400200148407870470000CE
:10EAC000F407002030B501460022002010E00B4C76
:10EAD000235C03EB43040A4D05EB4404A478082CA3
:10EAE00004DD441CE5B2541C0D55E2B2441CE0B2F6
:10EAF000024C647A8442EADC0A7030BD00110020C6
:10EB0000001200200148007870470000E803002050
:10EB10000020704701480078704700000011002075
:10EB2000014601EB8100400070470000F0B503464C
:10EB30000C4606251F201E781D2E46D2DFE806F063
:10EB4000450F1C1E2124274545452A2C2F314545BC
:10EB50004545454534383C454545454041001E4EF8
:10EB6000B67806F07F06052E03D1042107261E7015
:10EB700001E0082103252BE0042129E002210C25D6
:10EB800026E00121172523E00221092520E00121AB
:10EB900015251DE004211BE00121162518E00421A4
:10EBA00016E002210B2513E0032110253C200FE085
:10EBB000032110253C200BE001211B253C2007E010
:10EBC00000BF02211A253C2002E00121162500BFCA
:10EBD00000BF21701570F0BDF407002001480078D7
:10EBE000704700009C070020014800797047000032
:10EBF0009C0700200348017B0020024A107308464E
:10EC0000704700009C0700201EB50146002009E067
:10EC100083061A0E084B1344D3F8E8374DF820301A
:10EC2000431CD8B20328F3DB009B0B60019B4B60B5
:10EC3000029B8B601EBD000000F0FF1F01480078A2
:10EC4000704700004003002000BF06488078052878
:10EC500004D000BF03488078032801D10120704709
:10EC60000020FCE79C0600200248C07A0149085CAD
:10EC7000704700000011002041617047016170473A
:10EC800010B54FF4807303221021024800F050F8B1
:10EC900010BD00000008014010B500228B071C0FBA
:10ECA0000F2303FA04F204290EDA204B9B689343E6
:10ECB0001E4CA36023469B688C07240F00FA04F4C3
:10ECC00023431A4CA3602FE008290EDA174BDB68A8
:10ECD0009343164CE3602346DB688C07240F00FA4D
:10ECE00004F42343114CE3601EE00C290EDA0F4BB1
:10ECF0001B6993430D4C236123461B698C07240F2A
:10ED000000FA04F42343094C23610DE0074B5B69CF
:10ED10009343064C636123465B698C07240F00FA1A
:10ED200004F42343014C636110BD00000000014066
:10ED3000F0B5044616460025002201F00F0501F04B
:10ED4000100747B1042E05D145F00305E76B1F43BB
:10ED5000E76300E0354300201EE0012787401F40A5
:10ED6000C7B122684FEA800C0F2707FA0CF7BA43A5
:10ED7000870005FA07F73A43282904D1012787407D
:10ED80001F40676105E0482903D1012787401F40E4
:10ED900027612260471CB8B20828DED3082022E091
:10EDA000012787401F40E7B16268A0F108074FEADA
:10EDB000870C0F2707FA0CF7BA43A0F10807BF002A
:10EDC00005FA07F73A43282904D1012787401F4055
:10EDD000676105E0482903D1012787401F4027616B
:10EDE0006260471CB8B21028DAD3F0BD02469068C2
:10EDF000084008B1012070470020FCE7002101E035
:10EE00004A1C91B28142FBDB7047000070B50024C0
:10EE1000FBF7ECF800251BE06006040E4FF4807150
:10EE20001A48FFF72BFF0520FFF7E8FF4FF40071AA
:10EE30001648FFF7DBFF08B144F001044FF480717E
:10EE40001248FFF719FF0520FFF7D8FF681CC5B26D
:10EE5000082DE1DBFBF7E2F84FF400710B48FFF7F8
:10EE60000BFF0520FFF7CAFF4FF480710748FFF73B
:10EE700005FF0520FFF7C2FF4FF480710348FFF73D
:10EE8000FBFE0520FFF7BAFF204670BD000C0140D5
:10EE900070B50546FBF7C2F8002427E005FA04F038
:10EEA00000F0800040B14FF400712848FFF7E6FE03
:10EEB0000520FFF7A3FF07E04FF400712348FFF799
:10EEC000DBFE0520FFF79AFF4FF480711F48FFF724
:10EED000D5FE0520FFF792FF4FF480711B48FFF726
:10EEE000CBFE0520FFF78AFF601CC4B2082CD5DBDF
:10EEF000FBF77CF84FF480711448FFF7BFFE052044
:10EF0000FFF77CFF002413E04FF400710F48FFF778
:10EF10006DFF58B94FF480710C48FFF7ADFE052026
:10EF2000FFF76CFFFBF77AF8012070BD601CC4B2DC
:10EF3000642CE9DB4FF480710448FFF79DFE052047
:10EF4000FFF75CFFFBF76AF80020EEE7000C0140DA
:10EF500010B54FF400710F48FFF790FE0520FFF742
:10EF60004DFF4FF480710B48FFF788FE0520FFF737
:10EF700045FF4FF400710748FFF77EFE0520FFF7BD
:10EF80003DFF4FF480710348FFF776FE0520FFF741
:10EF900035FF10BD000C014010B54FF400710F4853
:10EFA000FFF76AFE0520FFF729FF4FF480710B4839
:10EFB000FFF764FE0520FFF721FF4FF400710748BB
:10EFC000FFF75CFE0520FFF719FF4FF4807103483F
:10EFD000FFF752FE0520FFF711FF10BD000C0140A6
:10EFE00030B50B46002100BF16E00A24B4EB107FB9
:10EFF00005D9302404EB107403F8114005E04124D6
:10F0000004EB10740A3C03F81140000100254C0089
:10F01000641C1D554C1CE1B29142E6DB30BD7047CB
:10F0200010B50849D1F8B000804708B1002010BDE4
:10F03000044890F8850008B90020F8E70248C07D30
:10F04000F5E70000440400209C070020F0B591B0D3
:10F0500004460F464E4890F8800028B14D4840784D
:10F0600010B9002011B0F0BDA0780C2807D1607A4B
:10F07000042804D14648D0F8D010012088474448DD
:10F08000007808B3FFF798FC082803D0FFF794FC3A
:10F09000092819D13E4890F87F0010B13E48C07849
:10F0A00020B13E49086A8047082806D13848C1681F
:10F0B000E01C884708B90020D4E73548416920465C
:10F0C000884708B10020CDE7A078042805D116268E
:10F0D00025781B2D26DD1B2524E0A078092802D1E8
:10F0E0001C261B251EE0A078072802D0A07808283F
:10F0F00002D11B261B2515E0A07820280DD1284819
:10F10000416820468847012805D13A460421E01C81
:10F1100000F030F9A6E70020A4E715262578102D89
:10F1200000DD10258DF804602A460DF10501A01CB4
:10F1300000F01FFC607C012814D11549D1F80001B2
:10F140008047227CE17B02EB0121884204D01049F8
:10F15000D1F80001804758B901A804F0DBF838B9AC
:10F1600000207FE701A804F0D5F808B9002079E76E
:10F170003A460421E01C00F0FDF808B9002071E7D0
:10F180000348416A04F10F00884701206AE7000044
:10F1900044040020D0030020D203002048030020B4
:10F1A000240600202DE9F04391B005460E464FF0AD
:10F1B00003090022402101A800F0E6FB05274FF0DB
:10F1C00004082879242857D2DFE800F0121C1E20FA
:10F1D0002428565656565656565656494E56565644
:10F1E0002C2D2E2F30313233345656565639434457
:10F1F0003E4880780E2803D10D244FF0090800E026
:10F200000A243DE001243BE0022439E04FF00A08E3
:10F21000032435E04FF00708052431E04FF01408CF
:10F2200006242DE000BF00BF00BF00BF00BF00BF2D
:10F2300000BF00BF4FF015080424042720E00C2471
:10F240004FF00308052702208DF807004FF004094E
:10F2500016E000BF4FF004080C24042710E04FF024
:10F2600004080C2404270BE04FF014080B2420485A
:10F27000416AA81C884703E0002011B0BDE8F08374
:10F2800000BF8DF80440A8788DF80500E8788DF867
:10F29000060001AA02EB0901E819424600F069FBE9
:10F2A00028790F2802D101208DF80700287922281B
:10F2B00002D02879232809D19DF807001F2805DBF3
:10F2C0009DF807001F38C0B28DF8070001A804F0B0
:10F2D00021F808B90020D0E732460221A81C00F02E
:10F2E00049F808B90020C8E70120C6E7F407002064
:10F2F0004404002070B500241DE0002104EB44000C
:10F30000C0EB84120F488154002510E004EB440147
:10F31000C1EB84120B491144491C05EB450201EB7A
:10F3200042000022042100F02FFB681CC5B20A2D08
:10F33000ECDB601CC4B203480C38407AA042DCDC31
:10F3400070BD00000C110020014688780B280AD1FE
:10F35000487A032807D10548D1F80320026001202C
:10F36000034A107070470020FCE700008905002068
:10F37000880500202DE9F04105460F461446062F6A
:10F3800002DD0020BDE8F081042C01DB0020F9E75C
:10F3900035490868804704EB4400C0EB84113348CA
:10F3A000465C0A2E5ADA04EB4400C0EB84122F4864
:10F3B0001044401C06EB460200EB42013A46284648
:10F3C00000F0D7FA2A4890F87A0060B1297A04EB65
:10F3D0004400C0EB841225481044401C06EB460252
:10F3E00000EB42000171A87B012829D12049D1F806
:10F3F000000180476A7B297B02EB0121884204D00F
:10F400001B49D1F80001804768B90B2104EB440087
:10F41000C0EB841215481044401C06EB460200EB7A
:10F42000420001710CE00A2104EB4400C0EB84129D
:10F430000E481044401C06EB460200EB42000171EE
:10F4400004EB4400C0EB84110848405C401CC1B28E
:10F4500004EB4400C0EB841204488154024948681C
:10F46000804701208EE70000B80200200C11002028
:10F47000440400202DE9F04106468848C168304622
:10F48000884708B1BDE8F0817078042800DAF9E710
:10F490008349086B804728B98148816E701C884772
:10F4A00000B1EFE77E48D0F8A810701C884700B97B
:10F4B000E8E73078FEF71CF90746FF2800D1E1E7BE
:10F4C000741CFFF7ADFD002847D06079912808D063
:10F4D0006079922805D06079932802D060799428C9
:10F4E0003BD16F4890F8850002280BD1207FE17E48
:10F4F00000EB012085B21621601DFEF70FF9A8422E
:10F500002AD0BFE7664890F88500032817D1207FEE
:10F51000E17E00EB012085B21621601DFEF7FEF8AA
:10F52000A84219D094F82000E17F00EB012085B2B9
:10F530001A21601DFEF7F2F8A8420DD0A2E794F858
:10F540002000E17F00EB012085B21A21601DFEF74B
:10F55000E5F8A84200D095E700BF6079912814D063
:10F560006079922811D0607993280ED06079942820
:10F570000BD04B4890F8340038B14948016C204614
:10F58000884710B102F006F87CE7454890F87E0005
:10F5900048BB6079932802D1A0790E2819D0FFF7D3
:10F5A0000BFA032815D0FFF707FA062811D03C48BC
:10F5B000007838B1FFF700FA08280AD0FFF7FCF905
:10F5C000092806D004223749601C00F0C1F900B9AF
:10F5D00058E72078001FC2B2611C601D00F0C9F915
:10F5E0002078001F20706078802800DA4AE701F058
:10F5F000D1FF6078912804D139462046FFF7D2FD2B
:10F6000049E06078922804D13946204600F058F845
:10F6100041E0234890F87A0050B16078932802D0F6
:10F620006078942804D139462046FFF70FFD32E078
:10F630006078B72804D11C48C168204688472AE072
:10F640002078182815D16078A178884211D1607887
:10F65000E17888420DD160782179884209D16078BB
:10F660006179884205D111480068401C0F49086043
:10F6700008E70B48D0F8E81020468847084890F87B
:10F68000340028B10648016C2046884700B1F9E6ED
:10F69000204600F067F800BFF4E6000024060020D2
:10F6A00044040020CC030020DC050020E4030020FB
:10F6B00010B504462046FFF7DDFE012010BD000016
:10F6C00030B589B004460D46A0780C2807D1607A81
:10F6D000042804D11148D0F8D01001208847142004
:10F6E0008DF8040010220DF10501A01C00F041F975
:10F6F00001A803F00FFE10B9002009B030BD2A4662
:10F700000621E01CFFF736FE08B90020F5E70348A4
:10F71000416AE01D88470120EFE700004404002013
:10F7200010B592B00D490868804740230A2201A90C
:10F730000B4801F013FD044608494868804714B996
:10F74000002012B010BD9DF80400801CC0B28DF8DE
:10F75000040001A8FDF7A0FB0120F2E7B802002099
:10F760002012002010B5044640230A2221460248F8
:10F7700001F0BEFC10BD00002012002010B5412396
:10F780000F220249024801F0E1FC10BDE40C002008
:10F79000D80C002010B50446012C04D104210848DF
:10F7A000FFF76AFA0AE0022C04D104210448F9F7B1
:10F7B000B6FD03E004210248FFF760FA10BD000027
:10F7C0000008014010B50446012C04D1022108486C
:10F7D000FFF752FA0AE0022C04D102210448F9F79B
:10F7E0009EFD03E002210248FFF748FA10BD000029
:10F7F00000080140704710B5044600F00DF840B114
:10F80000204600F01BF8002801DA002010BD01207E
:10F81000FCE70020FAE7000010B50248FFF714F8F3
:10F8200010BD00000404002010B504462146024823
:10F83000FFF70EF810BD00000404002010B50446C8
:10F8400021460248FFF734F810BD000004040020F0
:10F85000704700004FF40041080301F0ADF872B6A4
:10F8600001F0A6FD19491A48FDF7F8FF194A1A498F
:10F87000174803F0ADF901F023F8FFF701FA02F0A1
:10F8800079FBF9F7E1FC00BF1148D0F8AC008168C2
:10F890000120884705200E49887000BFF9F760FDF8
:10F8A0000E49486880470E49D1F89400804762B6F7
:10F8B000FAF7CCFCFAF720FD00BF05488078032852
:10F8C000FBD102E0054988688047FBE70000002083
:10F8D0009C0600208C0200207C02002048030020AF
:10F8E00044040020F0B50B30154D20F00701002432
:10F8F000144A0FE003688B420BD38B4205D95E1A82
:10F9000043184768C3E9006700E04368136002C01A
:10F9100004E0021D10680028ECD12046002802D126
:10F92000286808B10020F0BD064A07481060074A61
:10F93000121A22F00702C0E9002401202860D7E74C
:10F9400098060020940600207CAC002078CC002093
:10F9500030B503460C46002107E0585C655CA842C0
:10F9600001D0002030BD481CC1B29142F5DB01201E
:10F97000F8E710B50346002003E01C5C0C54441C5F
:10F98000E0B29042F9DB10BD10B50346002002E062
:10F990001A54441CE0B28842FADB10BD30B591B075
:10F9A00004460D46402101A8F8F719FC1F208DF8E8
:10F9B0000400E1208DF805000B49C86980478DF8E7
:10F9C00006000A208DF807002A46214602A8F8F70B
:10F9D000DFFB0549886D804718B10348416C01A8D9
:10F9E000884711B030BD00004803002000B589B041
:10F9F0003A4890F8600008B909B000BDFDF7E0FD95
:10FA0000012802D0022865D151E03548C07800288D
:10FA100040D033480079314991F87510884218DD9B
:10FA200000202F49C87003208DF804002D49886AF2
:10FA300080478DF805004D208DF8060014208DF8C4
:10FA4000070005208DF80800052101A8FFF7A6FF93
:10FA50002CE023484079401C214948710846007930
:10FA6000401C087108464079002806DD08464079A8
:10FA70001A4991F87510884202DD01201849487131
:10FA800000201749087048700A465079154A516A93
:10FA900088470BE003208DF804001249886A8047EC
:10FAA0008DF80500022101A8FFF778FF13E00C484C
:10FAB000C07800B9A0E700200949C87004208DF87B
:10FAC0000400084640798DF80500022101A8FFF7DF
:10FAD00065FF00E000BF00BF00BF8DE744040020C9
:10FAE000810500204803002010B50446184890F80E
:10FAF000600008B9002010BD6079102805D11549B3
:10FB0000886A8047217A884214D06079132802D00D
:10FB10006079142805D10F49886A8047A17F8842FF
:10FB200008D06079172810D10A49886A8047E17F98
:10FB300088420AD108484078FA2804DA0648407812
:10FB4000401C054948700120D5E70020D3E700009C
:10FB500044040020480300208105002010B504461D
:10FB6000A0B2FDF703FC10BD10B504464F48D0F815
:10FB70002404B8B94FF484614C48801CF8F72FFB7B
:10FB8000A0794A49C1F82804217AE07901EB0010F4
:10FB90004649C1F83004217AE07901EB001098B1B0
:10FBA000012010BD217AE07901EB00103F49D1F826
:10FBB0003014884201D10220F3E7217AE07901EB89
:10FBC00000103A49C1F830043848D0F824043030E5
:10FBD000B0F5846F12D90020344948704FF4846125
:10FBE0003248801CF8F7FBFA00203049C1F82404A1
:10FBF000C1F82804C1F82C040320D2E72B48D0F820
:10FC00002C04401C2949C1F82C040846D0F82C04C7
:10FC1000D1F82814884212D90020244948704FF4A2
:10FC200084612248801CF8F7DAFA00201F49C1F8E5
:10FC30002404C1F82804C1F82C040420B1E71B49AE
:10FC4000D1F82424891C5018302204F10901F8F756
:10FC50009FFA1648D0F8240430301449C1F824041F
:10FC60000520134908801148D0F83004401C0F4982
:10FC7000D1F82814884216D30C48D0F824040B4934
:10FC8000C1F8340401204870084690F82304401C51
:10FC900081F823040020C1F83804012081F83D04D4
:10FCA00000200349088000207BE700005C4700201B
:10FCB0007805002010B51749086D8047052801D048
:10FCC000002010BD1448407808B90020F9E7134817
:10FCD000407907280BD1002010494871012000F01D
:10FCE000BFF80B200C4981F83C040120E9E70A48E1
:10FCF000D0F83804401C0849C1F838040846D0F848
:10FD00003804B0F5967F03D900204870C1F8380454
:10FD10000020D6E7480300205C470020BD030020F8
:10FD200010B51348007800B910BD114890F83D0493
:10FD300090B100200E4981F83D040846811CD0F89E
:10FD400024240C48F8F724FA00200949C1F82404B7
:10FD5000C1F82804C1F82C04064800F025F8022058
:10FD6000FCF722FE00200249087000BFDCE700001B
:10FD70005C470020384300200A4890F83C0480B1DA
:10FD8000084890F83C040B2803DD0B20054981F856
:10FD90003C04044890F83C04401E024981F83C04AD
:10FDA00000BF70475C47002070B58AB00546282127
:10FDB0006846F8F714FA0026002427488169684647
:10FDC0008847FE208DF8040048208DF80500DE20CD
:10FDD0008DF806009E208DF807002048B0F8340406
:10FDE0001F30C0F347108DF8080001208DF809007E
:10FDF0009DF8080041012846FDF790FC06463012A8
:10FE00008DF80A00F0B28DF80B00144890F8230426
:10FE10008DF80C0013210DF10D00F8F7E0F9202109
:10FE2000684600F023F800F037F8C820FFF796FE88
:10FE30000BE02819202100F019F800F02DF83220ED
:10FE4000FFF78CFE04F1200084B20448D0F834049B
:10FE5000A042EED80AB070BD480300205C470020E5
:10FE600001490870704700005C47002070B50546E6
:10FE70000C46002001F054FF0549C86A8047064639
:10FE8000E1B204483246836A28469847012070BD93
:10FE900048030020B802002010B54FF4FA7408E0BF
:10FEA000FEF7CCFE00B110BD0220FFF757FE601E2A
:10FEB00084B2002CF4D100BFF5E7000070B5012535
:10FEC000002035494872002415E0FF2032490855CA
:10FED0003248005DFF2807D03048005DFE2803D07F
:10FEE0002E48005DFB2804D12B48407A401C2A494B
:10FEF0004872601CC4B2042CE7DBFF202649C8729C
:10FF000000241FE02548005DFB280FD0FE2807D005
:10FF1000FF2813D12048047000201F4988720EE08A
:10FF20002846691CCDB21C490C5408E01A48C57219
:10FF30002846691CCDB218490C5400E000BF00BF30
:10FF4000601CC4B2042CDDDB002406E0124A105D04
:10FF5000134AD16B8847601CC4B20F48407AA04254
:10FF6000F4DC104880780C49497A884203DD0A485D
:10FF7000407A0C49887001F0D9FE0B48808D48B159
:10FF8000FEF7C8FD06460849888D054932460B6CC8
:10FF90000421984770BD000000110020BA04002021
:10FFA000B8020020D60300209C07002070B51E4830
:10FFB000407A012800DC70BD1C49086B804700B105
:10FFC000F9E71B480078401CC0B2194908700A289C
:10FFD00000DAF0E700201649087001F05DFD1248D4
:10FFE0000578002405E01049601C085C0855601C79
:10FFF000C4B20D48407A401EA042F4DC0A48407A60
:020000040801F1
:10000000401E09490D54002408E0074B195D1B1DD3
:10001000185D084BDA6A9047601CC4B20248407A07
:10002000A042F2DC00BFC6E700110020440400201B
:10003000FC030020B802002030B589B0044624211A
:100040006846F8F7CCF820208DF800002C4881692C
:100050000DF10100884728208DF805002948006827
:10006000807928490968497900EB0120000A8DF858
:10007000060024480068807922490968497900EB24
:100080000120C0B28DF807001E4800680068029089
:100090001C48006800798DF80C0020128DF80D00C6
:1000A000E0B28DF80E0017480068C0798DF80F0097
:1000B00014480068007A8DF8100012480068807BB0
:1000C00010490968497B00EB0120000A8DF81100F6
:1000D0000C480068807B0B490968497B00EB0120D4
:1000E000C0B28DF81200FEF715FD05469DF8001010
:1000F00005482A46836A0DF10100984709B030BDD2
:100100004803002020060020B802002070B50446F5
:10011000002500F04FFA051E00D170BD11222146C6
:100120002846F8F735F8A08AA88200F011FA0646AA
:100130003146284600F032FA0120EEE72DE9F04181
:1001400006460F46002411E0204600F0F7F9051E90
:1001500000D10FE0042231462846F8F74BF818B9D1
:10016000AC742846BDE8F081601CC4B200F0F0F920
:10017000A042E9DC00BF0020F4E7000070B50546AE
:100180002878FDF7B5FAFF2801D1002070BDAC1C1E
:10019000042225492046FFF7DBFB18B320798F287E
:1001A0001ED16079DE281BD1A079482818D1E079CA
:1001B000FE2815D1207A082801DD082000E0207AE9
:1001C0001A49087000201A4908700120194908705E
:1001D0000F2204F108011848F7F7DAFF0120D5E7EC
:1001E0000020D3E713480078E0B111490978124A9A
:1001F0000F3202EB411020222146F7F7C9FF0C48CD
:100200000078401CC0B20A49087008490978884241
:1002100006DBFBF7C9FB0949087200200549087095
:100220000120B3E70020B1E7CC0300203E06002008
:100230003D0600203C060020D6A90020C8A50020CD
:1002400030B587B0054601AC1122E91C2046F7F70E
:100250009FFF0020A082607A0106A07A01EB004196
:10026000E07A01EB0021207B084410B9002007B0A0
:1002700030BD21792046FFF761FF38B92046FFF7EE
:1002800045FF08B10120F2E70020F0E70120EEE78A
:1002900030B5ADF20C4D9E48407930B101286ED09A
:1002A00002287DD003287CD11CE100F051F9002800
:1002B00062D0FCF715F900285ED09549087900F066
:1002C0003DF99449086080B900F042F990490979F4
:1002D000491CC9B28E4A1171884202DC00201146C5
:1002E000087100200DF20C4D30BD8A480068407A3C
:1002F000010688480068807A01EB00418548006863
:10030000C07A01EB002183480068007B01448148EA
:100310000068807B7F4A1268527B00EB022091FBD1
:10032000F0F17C480068407A02067A480068807ADA
:1003300002EB004277480068C07A02EB0022754861
:100340000068007B024473480068807B714B1B6827
:100350005B7B00EB032092FBF0F300FB132008B162
:10036000012000E0002008446949088001204880FD
:1003700048710020488101E00020B3E700BF6448D5
:10038000B0F80C04401C80B26149A1F80C04282884
:1003900008DB0020A1F80C04032048710020A1E72D
:1003A00010E0B1E05A494888FFF746FE002058495E
:1003B00008720420C88008464089401C48810220F9
:1003C0004871A2E05248007A012812D15048408872
:1003D000401C80B24E4948800988884203DC0120D5
:1003E0004B49487104E00020494948800120487188
:1003F0008BE04748007A022844D16C4645480068A3
:1004000050F8071F616080882081424800680068BA
:10041000206040480068807B3E490968497B00EBCA
:1004200001203B490988484385B2B5F5806F01DD5D
:100430004FF480652A4636490C3104F10A00F7F77B
:10044000A7FE29462046FBF71DFF88B932480078F1
:100450000A280BDA31483049097800EB810021681D
:1004600001602D480078401C2B490870002039E7B6
:10047000274801792748006800F052F800202449F5
:10048000487142E000BF2248C088401E80B2204927
:10049000C88030BB08464089642802DA01204871D0
:1004A0001FE01C480068808A401C80B21949096816
:1004B00088820A2805DB164801791648006800F092
:1004C0002FF800F045F812490979491CC9B2104AC1
:1004D0001171884202DC00201146087100200C498D
:1004E000487112E00A48B0F80C04401C80B2084978
:1004F000A1F80C04022806DD0020A1F80C0401205C
:1005000048710020EEE600E000BF00BF0120E9E6F0
:10051000C8A50020200600200A060020C4A4002050
:1005200070B504460D46FF20607429460248FEF768
:100530000DF90646304670BD1406002010B504467D
:1005400021460248FEF730F910BD000014060020D5
:1005500010B50248FEF73EF910BD00001406002059
:100560000348044908604860002008817047000083
:100570000C0600201406002000200AE0FF2100EBFA
:10058000400202EBC002044B03EB42025174411CD7
:1005900088B20A28F2DB7047ECA4002070B504464C
:1005A0000D462A4621460248FEF718F970BD0000A4
:1005B0001406002000211CE001EB410000EBC1000B
:1005C0000E4A02EB4000407CFF2810D1012001EBD5
:1005D000410202EBC102094B03EB4202507401EBF2
:1005E000410000EBC1001A4602EB40007047481C76
:1005F00081B20A29E0DB0020F8E70000ECA400202B
:1006000010B54FF4C87000F05DF804490870084652
:10061000007808B93C20087010BD0000A405002037
:1006200002460C2901DA00207047044883681360F1
:10063000C3685360006990600120F5E7A4050020BD
:100640000148407D70470000A40500200148407823
:1006500070470000A4050020014880887047000012
:10066000A405002070B504461348807D78B10020B1
:10067000114988751149C86A804705460F49886A3B
:10068000804706460E482946C26A304690478CB1DC
:100690000948007860B108480078401E0649087093
:1006A0000846007830B900F05DF8FFF7A9FF01E0D7
:1006B000FFF7A6FF70BD0000A4050020480300203E
:1006C000B80200202DE9F04106461048808B10B991
:1006D0000120F9F74FFC0D48808BFA2803DD00203C
:1006E0000A49888304E00948808B401C07498883B5
:1006F000B5082846F9F73EFC0446281903498969DC
:10070000471A024884613846BDE8F081A4050020FC
:1007100070B505460C460C2C01DD002070BD22464C
:1007200029460248F7F734FD0120F7E7AC05002021
:1007300018B10121034A517502E00021014A5175A7
:1007400070470000A405002002484078401C014981
:1007500048707047A4050020014988807047000058
:10076000A405002030B58BB0282101A8F7F737FD8C
:1007700020208DF804004E4881690DF1050088475E
:1007800051208DF809004B4840788DF80A004A48FE
:10079000007858B1FEF710F9082803D0FEF70CF9DD
:1007A000092803D102208DF80B0002E001208DF80A
:1007B0000B003F49886A80478DF80C0000208DF8B7
:1007C0000D008DF80E008DF80F008DF810008DF8DB
:1007D00011003848407D30B19DF8110040F0010013
:1007E0008DF8110005E09DF8110000F0FD008DF876
:1007F00011002F49086D8047042806D19DF811008B
:1008000040F002008DF8110005E09DF8110000F0A5
:10081000FD008DF811009DF80B00022806D19DF80F
:10082000110040F004008DF8110005E09DF8110062
:1008300000F0FB008DF811001E488088000A8DF83A
:1008400012001C4800798DF8130000208DF8140068
:100850008DF8150017488168CDF81610C168CDF8DD
:100860001A100069CDF81E001B210DF10900FCF7DC
:1008700055FF0446200A8DF82300E0B28DF82400CD
:1008800001200C4988750A49C86A804705460B480B
:100890002946C26A002090470549C86A8047054634
:1008A00003482946426B01A890470BB030BD0000B9
:1008B00048030020A405002044040020B8020020C2
:1008C00010B54FF4806000F06DF800220221142072
:1008D00000F006F800220121132000F001F810BDFD
:1008E0002DE9F04103460D46164600240027A04698
:1008F0002A48006800F4E060B0F5E06F03D100BF63
:100900004FF0040830E02548006800F4E060B0F5DE
:10091000C06F03D101274FF0030825E01F4800688E
:1009200000F4E060B0F5A06F02D10227B8461BE0EA
:100930001A48006800F4E060B0F5806F03D1032727
:100940004FF0010810E01548006800F4E060B0F5D1
:10095000407F03D104274FF0000805E04FF4A0606A
:1009600000F020F80227B846C7F1040005FA00F4A9
:10097000C8F104010F20C840304004432401084856
:10098000C45403F01F01012088405911890001F16E
:10099000E021C1F80001BDE8F08100000CED00E0AD
:1009A00000E400E002490143024A11607047000080
:1009B0000000FA050CED00E0034A0A400243034B35
:1009C0001A60BFF34F8F704780FFFF1F08ED00E0F4
:1009D00070B590B004460D46164600224021684688
:1009E000FEF7D2FF1F208DF80000E0208DF80100F7
:1009F000FDF7DCFF8DF802008DF80340324601A9B7
:100A00002846FEF7B6FF6846FCF746FA10B070BD00
:100A100038B50446E07810287ED2DFE800F0F21EF8
:100A2000088A249194B29FF2F2BDBEBFECC50E229B
:100A30007849201DFEF79DFF0E2276493020FCF7F5
:100A4000A7FB7448401E407A032805D10922724949
:100A500004F10D00FEF78DFF00BF0E226D4901204D
:100A6000FFF7B6FFD3E020796C494978884204D17A
:100A700060796A498978884202D0204602F0AAFA51
:100A8000207966494978884203D0002062490D39AF
:100A90004883607961498978884204D001205E49A1
:100AA0000D3981F8220060790E2821D1A07914280F
:100AB00002D0A0791E281BD16079584989788842D4
:100AC00009D1607955498978884211D15348C07855
:100AD000A17988420CD05249D1F8CC008047A07946
:100AE000142810D101204C490D3981F820000AE06A
:100AF00060790E2802D1A079142804D0002046493C
:100B00000D3981F820001A224449491C201DFEF7A6
:100B100030FF4449C86800E073E080471A223F492B
:100B2000491CA020FCF734FB3D48C169204688479A
:100B300000BF1A223949491C0320FFF749FF66E02C
:100B400002F0C0FB63E001200090201D02F0FAFBE0
:100B5000012269460620FFF73BFF58E0304890F835
:100B60007A0000B953E004222F49201DFEF701FF4F
:100B700004222D49D020FCF70BFB0520FAF74DF895
:100B800000BF274890F87A0000B940E004222649C7
:100B90000720FFF71DFF3AE000BF00BF2048D0F854
:100BA000C8102046884732E0207901280DD117224D
:100BB0001E49201DFEF7DDFE012017490D3981F881
:100BC0002300002081F822000FE0207902280CD1B8
:100BD00017221749201DFEF7CCFE01200E490D39C2
:100BE00081F82400002081F8220001200A490D39F3
:100BF00081F8210000BF17220C490E20FFF7E8FE04
:100C000005E00748D0F8DC102046884700BF00BF49
:100C1000012038BDCD070020A9070020F4070020DF
:100C20004404002024040020BE03002033080020D8
:100C30007508002070B590B004460D461646002297
:100C400040216846FEF7A0FE1F208DF80000E1203D
:100C50008DF80100FDF7AAFE8DF802008DF8034023
:100C6000324601A92846FEF784FE6846FCF714F9CF
:100C700010B070BD30B591B005460C46402101A8BA
:100C8000F7F7ADFAF5208DF80400AA208DF80500DD
:100C90008DF8060004F10800C0B28DF80700E120CD
:100CA0008DF808000A49C86980478DF809001320AB
:100CB0008DF80A00224629460DF10B00F7F768FA75
:100CC00004484021826901A8904711B030BD00005E
:100CD00048030020B802002030B589B00446E0780F
:100CE0001B2876D2DFE800F0D4360E493C5A4F6319
:100CF000D4767A95999AA5ABACD4D4A6D4D4ADC108
:100D0000D4CAC60007226749201DFEF732FEFAF753
:100D1000D1FEFAF797FE6349491E887800F0CCF9B6
:100D2000FDF7F8FE05465F49491EC8795E490A6B22
:100D300029469047002508E05A49491EC8795A4972
:100D40000A6B29469047681CC5B25848407AA842A9
:100D5000F2DC00BF072253490120FFF76BFF9DE043
:100D60000D225349201DFEF704FE00F07FFF0D22E7
:100D70004F490820FCF70CFA00BF0D224C49032014
:100D8000FFF758FF8AE004224A49201DFEF7F1FDD3
:100D9000042248491820FCF7FBF900BF01A8FDF721
:100DA00017FE042201A90520FFF744FF76E0012089
:100DB0008DF804003C48012201A9036A2E209847BF
:100DC000394988688047012201A90720FFF732FFCF
:100DD00064E05DE02046FAF7B3F85FE0207901288F
:100DE00002D0207902280DD12079012801D00120DC
:100DF00000E000208DF80400012201A90A20FFF77D
:100E000019FF05E02079042802D12B49486E80475C
:100E100044E02046F9F712FF40E03FE0264801A9F0
:100E2000C26D20469047092201A90D20FFF702FF5D
:100E300034E033E021480168204688472EE02DE069
:100E40002CE01F48807858B160791E2808D0002017
:100E50001B498870002205211948C01CFEF794FD2B
:100E60001548816B2046884718E01648416920469E
:100E7000884713E0207900F01DFF00BF1248C07DB5
:100E80008DF80400012201A91920FFF7D3FE05E027
:100E90000948D0F8E0102046884700BF00BF012075
:100EA00009B030BDC4030020B802002000110020AA
:100EB0004B080020CC030020440400201404002030
:100EC000F4070020240600209C07002030B593B0D2
:100ED00040230A2202A9214800F040F910B900205D
:100EE00013B030BD9DF80800001DC0B28DF804009D
:100EF0000DF10500FDF76CFDFDF704FE60B1002467
:100F000005E0214601A8FBF791FF601CC4B214481C
:100F1000007AA042F5DC1FE0124890F884001E28F9
:100F200013D1104890F8850078B11A210DF109000D
:100F3000FCF7F4FB054628128DF82300E8B28DF883
:100F4000240020208DF8040000BFFDF7E1FD0546D8
:100F5000294601A8FBF76AFF0120C1E7AC14002075
:100F6000001100204404002070B5044607490868B9
:100F7000804740230A222146054800F0B9F805467B
:100F8000024948688047284670BD0000B80200202A
:100F9000AC14002070B504464023112221460348BA
:100FA00000F0DCF80546284670BD00008C080020E3
:100FB00010B50446402311222146024800F098F85B
:100FC00010BD00008C08002010B5402311220249FA
:100FD000024800F0BBF810BD980800208C080020E3
:100FE00010B504460D4890F8C40008B9002010BDA3
:100FF000012C07D1FCF706FD08B10020F7E70848EF
:10100000C47409E00648C07C30B100210448C174B2
:1010100000F004FF0120EAE70020E8E74404002094
:10102000DF5B002010B588B00446E078182814D1A2
:1010300020791249087060798870F5208DF80000D9
:1010400020798DF8010060798DF802000C480322A8
:101050006946036A4FF484609847084800788DF821
:101060000000064880788DF8010002236A461721A7
:10107000612001F085FF08B010BD00009C4B0020EE
:10108000B802002010B504460948847000F04EFEF6
:1010900006220849F020FCF77BF80A20FCF717FF2E
:1010A00007220349491C0020FCF772F810BD00001C
:1010B000C3030020D703002010B50446204600F0EB
:1010C00069FE00F033FE06220749F020FCF760F8C5
:1010D0000A20FCF7FCFE054884700722411C002012
:1010E000FCF756F810BD0000D7030020C303002012
:1010F0002DE9F0410446884615461E461249086807
:10110000804720886188884204D1A088A84201DBFA
:10111000002712E06288A06802FB060132464046C2
:10112000FEF727FC6088401C90FBF5F105FB1100E1
:101130006080A088401CA080012703494868804740
:101140003846BDE8F0810000B802002010B581608B
:10115000448804800024848010BD00002DE9F04103
:101160000446884617461D4611490868804720886E
:101170006188884203D1A08808B9002612E022883D
:10118000A16802FB05102A464146FEF7F2FB2088C3
:10119000401C90FBF7F107FB11002080A088401E47
:1011A000A08001260249486880473046BDE8F081AA
:1011B000B802002070B504460E460A490868804708
:1011C00020886188884203D1A08808B9002503E0FF
:1011D00020887043A1680D5C024948688047284612
:1011E00070BD0000B80200202DE9F0470446884693
:1011F00017461D46DDF8209015490868804720886D
:101200006188884203D1A08808B900261AE02088A6
:101210006843A168085C484501D0022612E0228894
:10122000A16802FB05102A464146FEF7A2FB208872
:10123000401C90FBF7F107FB11002080A088401EA6
:10124000A08001260249486880473046BDE8F08703
:10125000B80200202DE9F04F8CB0074600200A901C
:101260004AA090E8004CC068CDE905BECDF810A0BA
:1012700007900FF21C1ADAE9000ACDE9020A0FF210
:10128000101ADAE9000ACDE9000A44484068C0F3C0
:1012900081000B900B9820B1012804D002283FD187
:1012A00003E03F4A3EE03F4A3CE03C48406800F4EF
:1012B000803CBCF5803F12D13848C06A00F08048BD
:1012C000B8F1000F01D1374B00E0374B334840688D
:1012D00000F40039B9F5003F02D15B0800E0334B60
:1012E0002E484068C0F383412C48406800F00060FD
:1012F00008B141F010012948406800F0804008B171
:1013000041F020010F2901D2891C06E00F2903D3E7
:101310003E2901D8491C00E03F2103FB01F201E016
:101320001F4A00BF00BF1D484068C0F3031504A852
:10133000465D22FA06F419484068C0F3022502A867
:10134000465D24FA06F0099014484068C0F3C225AF
:101350001DF8056024FA06F0089037B1012F06D079
:10136000022F06D0032F0AD106E00A9208E00A9461
:1013700006E009980A9003E008980A9000E000BF90
:1013800000BF0A980CB0BDE8F08F0000000000001C
:1013900000000000010203040607080900100240D3
:1013A00000127A000024F400006CDC0200093D0009
:1013B00010B50020FFF74EFF044640F2026000F037
:1013C00053F82548844204D14FF4800000F05CF8C3
:1013D00015E02248844203D1002000F055F80EE0C9
:1013E0001F48844204D14FF4400000F04DF806E05D
:1013F0001C48844203D14FF4000000F045F840F24D
:10140000026000F031F840F2036000F02DF840F285
:10141000046000F029F840F2056000F025F84FF470
:10142000C06000F021F840F2177000F01DF84FF492
:10143000E06000F019F840F2017000F015F840F299
:10144000027000F011F840F20C6000F00DF840F26C
:101450000F7000F009F810BD006CDC0200A24A0415
:1014600000D8B805000E2707064A02EB901109685C
:1014700000F01F0301229A401143024B03EB90122C
:101480001160704700100240044A516821F4400185
:1014900041EA0002014B5A60704700000010024010
:1014A0001CB50B4803226946436A4FF48460984791
:1014B0009DF80000F52807D19DF801000549087046
:1014C0009DF80200887002E00020024908701CBDEF
:1014D000B80200209C4B00201FB52248102269460C
:1014E000436A9001984700240EE0C4F10E001DF8F5
:1014F0000000C4F10F011DF801104840C4F10F01B4
:101500000DF80100601CC4B20F2CEEDB1648037806
:10151000C21C00F123016846F7F7E4FD11481022D0
:101520006946436A4FF48260984700240EE0C4F194
:101530000E001DF80000C4F10F011DF80110484015
:10154000C4F10F010DF80100601CC4B20F2CEEDBDA
:1015500005480378C21C00F133016846F7F7C2FD65
:101560001FBD0000B80200209C4B002010B50748AA
:10157000C16C01208847012005490870002048807F
:10158000012008710020C88010BD0000B8020020B2
:101590009C07002010B50748407A00B910BD002014
:1015A0000449487288720448016D0020884700BFD2
:1015B000F4E700009C070020B8020020F0B58DB0D1
:1015C00005464B4890F8900010B901200DB0F0BDD1
:1015D0004848007808B90120F8E72122294604A8E4
:1015E000F6F7D6FD9DF81500F7F73EFD061E01DD66
:1015F0008DF8156006240DE004A8005D80F0A506B6
:1016000004A9601C085C80F055000855601C0E544D
:10161000A01CC4B21F2CEFDB00240DE0C4F11F009E
:1016200004A9085CC4F1200104AA515C4840C4F13B
:1016300020015054601CC4B21A2CEFDB00240CE0D3
:1016400004F1160004A9085CA11D04AA515C4840DD
:1016500004F116015054601CC4B20B2CF0DB1022B4
:101660000DF116016846F6F793FDFAF7F9FD40B162
:1016700020480378C21C0DF116016846F7F732FDC9
:1016800018E09DF815004C2809D01A48037800F19D
:1016900023020DF116016846F7F724FD0AE015480C
:1016A0000378C21C0DF116016846F7F71BFD1320E5
:1016B0008DF81500212204A92846F6F769FDE87F78
:1016C000002803DC95F8200000280FDD1A21681D92
:1016D000FCF724F80746E87FB0EB272F04D1F8B2D7
:1016E00095F82010884201D000206FE701206DE7B7
:1016F000440400209C4B0020F0B589B005464548C5
:1017000090F8900008B909B0F0BD4348007800B9DE
:10171000F9E71A21681DFCF701F807463812E87747
:1017200085F8207020202870212229466846F6F787
:101730002FFD6879F7F798FC061E01DD8DF805602E
:101740009DF80500412803D09DF8050042280FD1DF
:101750009DF8090028280BD14C208DF805002E4853
:101760000378C21C0DF10601A81DF7F74BFD14E02C
:10177000FAF776FD40B128480378C21C0DF1060146
:10178000A81DF7F73FFD08E02348037800F1230286
:101790000DF10601A81DF7F735FD00240CE004F15A
:1017A0001600285CA11D1DF80110484004F1160127
:1017B0000DF80100601CC4B20B2CF0DB072409E01B
:1017C000601E1DF800001DF8041048400DF80400CC
:1017D000601CC4B2212CF3DB06240FE01DF80400CA
:1017E00080F05506601C1DF8000080F0A5000DF883
:1017F0000400601C0DF80060A01CC4B21F2CEDDBBF
:10180000212269462846F6F7C3FC2020287000BF35
:1018100079E70000440400209C4B002030B591B0D3
:10182000044621460720F8F78FF905462246294647
:101830000720F8F7AFFA05F0400060B18DF80040DE
:1018400021460DF10200F8F7A1F98DF801000D48CD
:10185000016C6846884705F0200010B1012000F0B7
:101860005FFA094A32F81410084A52F82400FDF7CA
:1018700003FA2046F8F743FB2046F8F747FB11B080
:1018800030BD000048030020B0390108A03901082C
:1018900070B506460D461446284A32F81410284AF8
:1018A00052F82400FDF7E8F921460020F8F74AFB3A
:1018B000244A32F81410244A52F82400FDF7DCF9C7
:1018C0002146E120FCF7E2FA1E4A32F814101E4AC3
:1018D00052F82400FDF7D2F9202D00DD2025FBF77A
:1018E0008BFE40B1194A32F81410194A52F82400FC
:1018F000FDF7C2F907E0154A32F81410144A52F8FD
:101900002400FDF7BBF92025224629463046F8F78A
:101910006FFA0A4A32F81410094A52F82400FDF707
:10192000ADF90A20F9F7C4FB044A32F81410044A4E
:1019300052F82400FDF7A0F970BD0000C839010875
:10194000B83901087C3901086C390108B03901083F
:10195000A039010800B591B00022402101A8FEF78E
:1019600013F81F208DF80400E1208DF805000A49C6
:10197000C86980478DF806000A208DF80700062008
:101980008DF808000DF10900FDF79CF80248416C44
:1019900001A8884711B000BD4803002010B51248C7
:1019A0000078012800D010BD0F484068401C0E4947
:1019B000486040F2DC5188420ED20B4840686421F6
:1019C000B0FBF1F201FB120058B90848C16D0120CB
:1019D0008847FFF7BFFF04E002200349087000209A
:1019E000486000BFDFE70000F4030020B8020020D9
:1019F00010B504462046F8F725FA21467020F8F77E
:101A000019F8224601211D20F8F7C4F922462021A9
:101A10001120F8F7BFF922461E210020F8F7BAF985
:101A2000224600210120F8F7B5F9224601210220C3
:101A3000F8F7B0F9224603210846F8F7ABF9154844
:101A400090F87400012803D12146F8F74BF90CE017
:101A5000104890F87400022803D12146F8F742F9A3
:101A600003E021460020F8F73DF921460320F8F76E
:101A70000BF9224605214AF2554000F045F8204670
:101A8000F8F720F82046F8F701F82046F8F73EFA74
:101A900010BD0000440400207047000000EB40012E
:101AA000044A12F81110491C00EB4002014B03F8E4
:101AB000121070470012002070B504460D46FBF767
:101AC0009BFD20B129460720F8F7DEF81BE0012C2A
:101AD00004D0022C07D0032C0FD109E029460220A4
:101AE000F8F7D2F80EE029460120F8F7CDF809E022
:101AF00029460020F8F7C8F804E029460320F8F743
:101B0000C3F800BF00BF70BD7CB504460D46164645
:101B10000AA103C9CDE9000120128DF80200E0B24C
:101B20008DF80300324629466846F8F7F9F833463F
:101B30002A4669460020F8F7B9F87CBD1998A42513
:101B40000100000070B505460C46F7F740FA214643
:101B50002846F8F7CAF92046F8F7D8F9F8F744FA12
:101B600070BD000010B504460548007C28B12178FE
:101B7000601CF8F72BFD012010BD0020FCE70000E1
:101B8000945F002070B5054600240DE0094800EB85
:101B9000840104222846F6F72DFB18B9054800EB0E
:101BA000840070BD601C84B2034800788442EDDB81
:101BB0000020F6E7F45B00208705002030B591B0E7
:101BC00004460D462078401CC2B269462046FDF707
:101BD000D0FE104890F87E0060B19DF80000001F14
:101BE000C0B28DF800009DF800200DF10101081D24
:101BF000FDF7BFFE0748D0F8A410684688479DF857
:101C0000001005482A46836A0DF10100984711B07B
:101C100030BD000044040020B80200202DE9F0414E
:101C200004462078062813D00E480568001D066873
:101C3000001D07683D4455B10822A11C2846FDF748
:101C4000CFF9042204F112013046FDF7C9F906E08C
:101C50000549086810B16080010CA18000BFBDE893
:101C6000F0810000E8F7FF1F00210240A0200C498E
:101C700088720C4890F8700048700D208870012020
:101C8000C870084890F87100C872064890F8721041
:101C900003480173034890F873100148417370477B
:101CA0004A080020440400200149087070470000E1
:101CB000E803002010B504460D4890F8850058B19F
:101CC0000B49D1F8B000804718B101200949C87507
:101CD00005E00848C47502E000200649C8750122E5
:101CE000044917314FF4A070FBF752FA10BD000001
:101CF000440400209C0700200649097801B1704780
:101D000028B90121034A11700349044A916100BFB7
:101D1000F5E70000B3020020D9920008B8020020C5
:101D200001490870704700004003002010B51648B4
:101D3000807816490872002204211448001DFDF71E
:101D400023FE1248027A011D0F48C01CFDF711FE48
:101D50000E48C07A0D49097A884204DA00210B48FE
:101D6000C27A001D8154002408E0084B195D1B1D38
:101D7000185D074BDA6A9047601CC4B20348407A8A
:101D8000A042F2DC10BD0000D603002000110020AC
:101D9000B802002010B504460948C4700146C8784E
:101DA000FBF7B8FB064908710879FBF7B3FB044958
:101DB00048714879FBF7AEFB0149887110BD0000FE
:101DC000D6030020016841F04001016070470146E0
:101DD000C86880B27047C16070470246906808408A
:101DE00008B1012070470020FCE70246002010687F
:101DF00000F441500B6818434B6818438B68184334
:101E0000CB6818430B6918434B6918438B69184317
:101E10001060D36923F40063D361704710B50D4897
:101E200090F8C40000B910BD0B48C07B012800D158
:101E3000F9E70A48816B002088470748007D401C6D
:101E4000C1B2054801750121C173002101744174BB
:101E500000BFE8E744040020DF5B002048030020C7
:101E6000002000213E4A126842F480323C4B1A6046
:101E700000BF401C3A4A126802F4003119B94FF60B
:101E8000FF729042F5D1364A126802F400320AB964
:101E900000BFFEE7324AD26942F08052304BDA612D
:101EA000304A126842F440422E4B1A602C4A526863
:101EB0002B4B5A601A4652685A601A46526842F4CE
:101EC00080625A601A46526822F440325A601A46BA
:101ED000526842F440325A601A465268224B1A4005
:101EE0001F4B5A601A46526842F450125A601A4602
:101EF000126842F080721A6000BF194A126802F03C
:101F00000072002AF9D0174A126842F48032154B49
:101F10001A6000BF134A526802F48032002AF9D0D6
:101F2000104A126842F400320E4B1A6000BF0D4A8C
:101F3000526802F40032002AF9D0094A526822F0AD
:101F40000302074B5A601A46526842F002025A6076
:101F500000BF034A526802F00802002AF9D0704715
:101F60000010024000700040FFFFC3B710B5FFF73C
:101F700077FF10BD10B5124800684FF47A71B0FBBE
:101F8000F1F4601EB0F1807F01D301200FE0601EEC
:101F90004FF0E02148610F214FF0FF30F7F77CFF51
:101FA00000204FF0E021886107200861002008B17F
:101FB00000BFFEE70F214FF0FF30F7F76DFF10BDB8
:101FC0001000002010B5044604480068001B81B2D0
:101FD00002482C3800F05AF810BD00002C040040D4
:101FE00010B50120234988750846407A70B9084623
:101FF000807A401CC0B28872052807DD00208872F4
:10200000012048721C48016D012088471948007A58
:10201000401CC0B21749087232280EDD0020087239
:102020001549C869804720B11348C16C0220884710
:1020300003E01148C16C002088470E484088401CCE
:1020400080B20C49488040F2DC51884203DD002018
:102050000849087048800748C088401C80B205497C
:10206000C880322802DD00200871C88003498868D2
:10207000804710BD9C070020B802002038040020D3
:10208000C162704701460020486A7047416270474C
:10209000016841F001010160704700000A88826216
:1020A0001D4A90420ED0B0F1804F0BD01B4A904297
:1020B00008D01B4A904205D01A4A904202D01A4AD0
:1020C00090420BD1026822F07002026002684B88D5
:1020D0001A43026002688B881A4302608A68C262EF
:1020E000124A90420AD0124A904207D0026822F463
:1020F000407202600268CB881A430260064A90422E
:1021000002D0094A904201D10A7B0263426942F03F
:102110000102426170470000002C014000040040B1
:1021200000080040000C0040003401400010004056
:1021300000140040C2688A43C2607047C2680A4304
:10214000C2607047CA43026170470246D06800EA25
:1021500001031069084010B10BB101207047002045
:10216000FCE7000010B50B48007810B100200949C9
:1021700008700948007810B1002007490870074826
:10218000007828B100200549087005490869804792
:1021900010BD0000EF030020F0030020F103002039
:1021A0002406002081621AB9436943F001034361A8
:1021B0007047000010B540230A2202490248FEF78A
:1021C000C5FF10BDB8140020AC14002010B540238A
:1021D0000A2202490248FEF7B9FF10BD2C12002066
:1021E000201200207047000010B50A48C16B032080
:1021F00088474FF47A70FBF7C6F80748816B0120D7
:1022000088470020054908740021092000F094F84F
:1022100010BD0000B802002048030020945F002099
:1022200010B50748C068401C0549C860052805D39B
:102230000020C860F8F750FBF7F7E2FB10BD000084
:10224000945F00200020704738B5044620790128AB
:1022500002D0072865D140E03348A1680160E168F9
:102260004160218A0181E079012822D12E488079BC
:1022700001062D48C07901EB00412B48007A01EBA3
:1022800000212948407A0D18284881696846884706
:1022900025484079244A127900EB022081B22A466F
:1022A0006846F8F72FF901201F490874F8F7ECFA8F
:1022B0000CE0E079022809D100201B4908740520B0
:1022C0001B4908701948816B012088471A23221D79
:1022D0001621612000F054FE24E01A23221D16214D
:1022E000612000F04DFE60791E2803D12046FDF7E5
:1022F0003BFC15E0207A15280BDC217A01EB41022A
:102300000949113101EB0210302204F10901F5F7FE
:102310003FFF207A152803D10120034981F83104B9
:1023200000E000BF00BF38BD945F002048030020DC
:10233000900500207047704730B589B005460C46BF
:1023400018208DF80400E1208DF805000A49C869BD
:1023500080478DF8060016208DF807008DF808508C
:1023600020128DF80900E0B28DF80A000248416C95
:1023700001A8884709B030BD4803002010B50446C5
:10238000D4F8AC000021826A2046904710BD10B5F9
:102390000446D4F8AC10A06C0022CB6A11469847D2
:1023A00010BD70B504460025D4F8AC002946426B38
:1023B0002046904700BF70BD416002814381704755
:1023C00041600281438170474160028143817047CF
:1023D000417841F08001014A116070474C5C004037
:1023E00070B504460D46A078032808D1287930B985
:1023F000D4F8A8002946C2682046904770BD012045
:10240000FCE7000001200849086000200860091D61
:1024100008600549103108600348006840F41F4017
:102420000149086070470000405C004001200449F9
:1024300008600020091D08600320091F086070471C
:10244000405C004010B50446012C04D1010205484F
:10245000FCF714FC04E04FF480710248FCF70CFC1C
:1024600010BD000000080140F0B50346002400251F
:1024700000266AB9214800EB0110C068C0F30905C5
:102480001E4800EB011080681D4F07EB400627E057
:10249000012A23D11B4F07EB8100D0F8000C00F07C
:1024A000400068B1154800EB01104068C0F3090511
:1024B000124800EB01100068114F07EB40060FE0D7
:1024C0000E4800EB0110C068C0F309050B4800EB93
:1024D000011080680A4F07EB400601E00020F0BDC4
:1024E000002405E036F8047B1F809B1C601C84B22E
:1024F000681CB4EB500FF5D32846F0E700600040AD
:10250000006000400050004070B58AB1134D05EBEB
:1025100001152D68124E06EB4504002303E00588E3
:1025200020C4801C5B1C551CB3EB550FF7D300BFB8
:102530000A4B03EB01135A6000BF0A4C04EB810302
:10254000D3F8003C48F6BF74234083F03003054DB8
:1025500005EB8104C4F8003C00BF70BD0060004082
:10256000006000400050004070B504460D46D4F8AD
:10257000AC002946426A2046904770BD30B50346FC
:1025800001F07F00CA1142B300BF294C04EB800266
:10259000D2F8002C02F040027AB100BF04EB8002B6
:1025A000D2F8002C48F68F74224042F04002204DB1
:1025B00005EB8004C4F8002C00BF00BF00BF1C4C1A
:1025C00004EB8002D2F8002C48F6BF742240184D6C
:1025D00005EB8004C4F8002C28E000BF144C04EB89
:1025E0008002D2F8002C02F480427AB100BF04EBE2
:1025F0008002D2F8002C48F68F74224042F48042C8
:102600000B4D05EB8004C4F8002C00BF00BF00BFD9
:10261000074C04EB8002D2F8002C4BF68F7422405A
:10262000034D05EB8004C4F8002C00BF30BD000052
:10263000005000402DE9F04104460D4616461F4665
:10264000D4F8AC003B4632462946D0F820C020469C
:10265000E047BDE8F0812DE9F04104460D461646FD
:102660001F4605F07F0000EB400104F1140000EB71
:10267000810800233A4631464046FFF79DFED4F8D4
:10268000AC002946826A20469047BDE8F0810000F0
:1026900030B50246002002F14401A023204C236003
:1026A0000023636040230B803039A3600B800B88CC
:1026B0003E2B0AD90B884FF6FF7404EA43135B1EC6
:1026C00043F40043164CE36006E00B885B1C23F0E8
:1026D00001035B02124CE36001200FE0114C04EB9C
:1026E0008003D3F8003C48F68F74A34303430D4D99
:1026F00005EB8004C4F8003C431CD8B20428EDD399
:10270000094B1B689BB2084C236043F220232360D3
:102710008023054C4C3423600123937030BD0000AE
:102720000060004000500040005C004010B500BF59
:102730004A06094B03EBD252D2F8002C4BF68F73AA
:102740001A4082F440524B06034C04EBD353C3F8B7
:10275000002C00BF10BD0000005000402DE9F047E4
:102760000546894616461F4609F07F0A0AEB4A01CC
:1027700005F1440000EB8108B8F80000B84201DD23
:10278000384601E0B8F800000446D5F8AC0022460F
:102790005146C36A30469847381B82B231192346E6
:1027A0004046FFF709FEBDE8F08700002DE9F04341
:1027B00005460C469E7806F07F009988002793F81E
:1027C00003C00CF0030CDFF8508258F82CC04CEA20
:1027D000000CDFF8489209EB8008C8F800CC4FEAFB
:1027E000E61CBCF1000F62D000EB400805F1440C80
:1027F0000CEB88073980B4B9DFF824C20CEB001C5D
:10280000CCF8002000BFC84608EB800CDCF800CCF8
:1028100048F6BF780CEA080C8CF0200C09EB800815
:10282000C8F800CCF6E0012CFCD1DFF8F08108EB11
:10283000800CDCF800CC4CF4807C48F68F780CEAF5
:10284000080CDFF8D89109EB8008C8F800CC1FFA13
:1028500082FCDFF8CC8108EB0018C8F800C04FEA12
:10286000124CDFF8BC8108EB0018C8F808C000BFA4
:10287000C84608EB800CDCF800CC48F6BF780CEAC0
:10288000080C8CF0300C09EB8008C8F800CC00BFB5
:1028900000BFC84608EB800CDCF800CC4BF68F7804
:1028A0000CEA080C09EB8008C8F800CCB2E000EB99
:1028B000400805F1140C0CEB8807398034B9DFF8B7
:1028C00060C10CEB001CCCF808204EE0012C4CD170
:1028D000DFF8488108EB800CDCF800CC4CF4807CFD
:1028E00048F68F780CEA080CDFF8309109EB800885
:1028F000C8F800CC00BFC84608EB800CDCF800CC60
:1029000048F68F780CEA080C4CF0400C09EB800874
:10291000C8F800CC00BF1FFA82FCDFF8048108EB86
:102920000018C8F800C04FEA124CDFF8F48008EB3A
:102930000018C8F808C03E290BD9A446CCEB411CAE
:102940004CF4004CDFF8D88008EB0018C8F804C03D
:102950000BE001F1010C2CF0010C4FEA4C2CDFF8DC
:10296000C08008EB0018C8F804C03E290CD94FF00D
:10297000010CCCEB411C4CF4004CDFF8A48008EBBC
:102980000018C8F80CC00BE001F1010C2CF0010C90
:102990004FEA4C2CDFF8888008EB0018C8F80CC010
:1029A0009CB900BFDFF8748008EB800CDCF800CC29
:1029B0004BF68F780CEA080C8CF4005CDFF85C9026
:1029C00009EB8008C8F800CC24E0012C22D100BF1C
:1029D000DFF8488008EB800CDCF800CC4BF68F78F1
:1029E0000CEA080CDFF8349009EB8008C8F800CC3A
:1029F00000BF00BFC84608EB800CDCF800CC48F6EE
:102A0000BF780CEA080C8CF0200C09EB8008C8F8A1
:102A100000CC00BFBDE8F0833C3901080050004005
:102A20000060004030B5024601F07F00CB1193B347
:102A300000BF334C04EB8003D3F8003C03F04003A9
:102A40007BB100BF04EB8003D3F8003C48F68F74E1
:102A5000234043F040032A4D05EB8004C4F8003CBA
:102A600000BF00BF002400EB400502F1440303EB6C
:102A700085039C7000BF224C04EB8003D3F8003C1C
:102A800048F6BF74234083F030031D4D05EB8004EE
:102A9000C4F8003C33E0FFE700BF194C04EB8003AF
:102AA000D3F8003C03F480437BB100BF04EB800308
:102AB000D3F8003C48F68F74234043F48043104D14
:102AC00005EB8004C4F8003C00BF00BF002400EB0D
:102AD000400502F1140303EB85039C7000BF084C12
:102AE00004EB8003D3F8003C4BF68F74234083F44F
:102AF0004053034D05EB8004C4F8003C00BF30BDDB
:102B00000050004030B5024601F07F00A8B900BF78
:102B1000244B1B6848F6BF74234083F01003214CFC
:102B2000236000BF00BF23461B684BF68F74234011
:102B300083F480531B4C236033E0CB11C3B10124D9
:102B400000EB400502F1440303EB85039C7000BFDA
:102B5000154C04EB8003D3F8003C48F6BF742340C7
:102B600083F01003104D05EB8004C4F8003C18E01E
:102B7000012400EB400502F1140303EB85039C7074
:102B800000BF094C04EB8003D3F8003C4BF68F7474
:102B9000234083F48053044D05EB8004C4F8003CCB
:102BA00000BF30BD005C00400050004010B503463F
:102BB0004806064C04EBD050D0F8002CC81110B1D8
:102BC00002F0300010BD0020FCE700000050004083
:102BD00070B504460D4616460820144908700120B9
:102BE0004870400248800846446074342563666338
:102BF0000F48A0630F4844F874090F49A1670F49B3
:102C0000E167D4F8A4004068C07900F040004009B2
:102C100020710121E171D4F8AC1008688047D4F824
:102C2000A410C968C868FEF7F9FF70BD1400002041
:102C30001C0000202DB30008E9B2000897B200087C
:102C400010B50446A078E0700420A070E07930B19F
:102C500000BFD4F8AC100869804700BF01E0032131
:102C6000A17110BD2DE9FC419A48006880B2019025
:102C7000984800689749091F096801F47F41084096
:102C8000009095484468BDF8000000F4004000281A
:102C90007DD0A5E0BDF8040000F00F05BDF80400EC
:102CA00000F01000002860D08C4901EB8500D0F8BE
:102CB000000C00F4004000281FD000BF01EB85008D
:102CC000D0F8000C40F68F710840844A02EB850171
:102CD000C1F8000C00BF114601EB8500D0F8000CD4
:102CE00000F4006060B14DB905EB450104F17400DA
:102CF00050F8212029462046904770E0BDE8FC812D
:102D000005EB450104F1140000EB81067068D4F86E
:102D1000AC1000220B6B2946984707467068384470
:102D2000706070893844708170893189884202DA14
:102D30003088B84212DD05EB450104F1740000EB68
:102D40008100406880B105EB450104F1740000EB9F
:102D50008100294642682046904705E0D4F8AC003F
:102D60002946826A2046904739E05C4901EB85009C
:102D7000D0F8000C00F0800088B300BF01EB8500A4
:102D8000D0F8000C48F60F710840544A00E030E0DB
:102D900002EB8501C1F8000C00BF05EB450104F111
:102DA000440000EB8106308990B905EB450104F140
:102DB000740000EB8100806880B105EB450104F1EF
:102DC000740000EB8100294682682046904705E0A8
:102DD0003389294620467268FFF7C0FC00BF00BF58
:102DE0003C48006880B2019000F4004000287FF465
:102DF00051AFBDF8000000F4805070B16FF4805006
:102E000034490860E078A070607A30B900BFD4F827
:102E1000AC104869804700BF00BFBDF8000000F457
:102E2000006060B12B48001F006800F0100030B94E
:102E30002046FFF705FF6FF4006026490860BDF8E3
:102E4000000000F4007058B16FF400702149086070
:102E50002348006820B1224800680168204688475E
:102E6000BDF8000000F4807018B36FF48070194949
:102E70000860A079E8B1A079401EC1B2A171C1B9C2
:102E8000607A50B11348001F006820F0100011490B
:102E9000091F0860002161720BE00E48001F0068E6
:102EA00040F010000B49091F08600321A1710121A6
:102EB0006172BDF8000000F4806040B16FF4806082
:102EC00004490860D4F8AC00C1692046884700BFB7
:102ED00014E70000445C0040140000200050004053
:102EE0005C0000200548006820F0040003490860E9
:102EF0000846006820F0080008607047405C004009
:102F000005494968097A012905D10449096841F050
:102F10001001024A1160704714000020405C00401C
:102F200070B505460C466078034951F820202146CB
:102F30002846904770BD00006000002003480068EC
:102F400040F00C000149086070470000405C004000
:102F500002460120704710B5FFF762F910BD00006E
:102F600010B5012003490870F8F71EFE00F0AAFA18
:102F700010BD0000B20200207047704770477047D4
:102F8000F0B589B004460D4616461F46202101A81B
:102F9000F5F725F91F208DF8040004F00F0040F02C
:102FA000E0008DF805000949C86980478DF80600E2
:102FB0008DF807503A46314602A8F5F7E9F803487C
:102FC000416C01A8884709B0F0BD0000480300200B
:102FD0007047000010B50446607920B90448416884
:102FE0000020884703E0024841680120884710BD5F
:102FF00024040020F0B59DB00446002240210DA815
:10300000FCF7C2FC1F208DF83400E0208DF835005D
:10301000FBF7CCFC8DF8360005208DF837008DF8D5
:10302000384094480078A0422ADB04EB440000EBCF
:1030300084109149084490F84100022820D104EB03
:10304000440101EB84118C4B194491F8402004EBAE
:10305000440101EB8411C8180DF13901FCF789FC1A
:1030600004EB440000EB84108349084490F84200CC
:103070008DF834000DA8F9F70FFF01201DB0F0BD49
:1030800020217E48FEF796F8054675B9FF208DF899
:10309000380000208DF839008DF83A008DF83B009B
:1030A0000DA8F9F7F9FE0020E8E70A950CAA0BA98C
:1030B0000AA8FBF73BFD8DF8340004EB440101EB5B
:1030C00084116D4A881800224021FCF75DFC9DF8B0
:1030D000280004EB440101EB8411674A505401209D
:1030E00004EB440101EB8411114481F8400004EB2E
:1030F000440101EB8411114481F841005D480470E2
:10310000002690E0701CC6B22023C82202A95B48AA
:103110000095FEF769F80746012F4CD19DF828006D
:103120000D2820D1012004EB440101EB8411524A07
:10313000114404EB440202EB84124F4B1A4492F800
:103140004020885404EB440000EB841019460844E6
:1031500090F84000401C04EB440101EB84111A4636
:10316000114481F8400004EB440000EB8410424A13
:10317000104404EB440202EB84123F4B1A4492F8D1
:10318000402081189DF830200DF10900FCF7F1FB7B
:1031900004EB440000EB84103749084490F84000E9
:1031A0009DF83010084404EB440101EB8411324ACD
:1031B000114481F840001FB19DF82C00864231DB9C
:1031C000FF2004EB440101EB84112B4A114404EB72
:1031D000440202EB8412284B1A4492F8402088548F
:1031E000FF2104EB440000EB84101A46024404EB78
:1031F000440000EB8410184490F84000401C115427
:1032000004EB440000EB84101946084490F8400099
:10321000801C04EB440101EB84111A46114481F82F
:10322000400005E000BF9DF82C008642FFF66AAF23
:1032300000BF04EB440101EB84110F4B194491F8DA
:10324000402004EB440101EB8411C8180DF1390151
:10325000FCF78FFB9DF8340004EB440101EB841173
:10326000054A114481F842000DA8F9F715FE012026
:1032700004E70000FD030020443000203817002040
:1032800010B500F053F800200249487088700870AB
:10329000C87010BDFF03002010B50948C078401C5D
:1032A000C0B20749C870022800DA10BD00200449E6
:1032B000C8700120887000F013F800BFF5E7000027
:1032C000FF03002010B500F0EBF80120034948701F
:1032D000887000200870C87010BD0000FF03002037
:1032E00010B50B48407890B1094800780A280EDAEA
:1032F0000748807858B106480078401C0449087097
:103300000878FFF777FE024948700020887010BDEA
:10331000FF03002010B504462023C822214602489E
:10332000FDF7E6FE10BD00003817002010B5202381
:10333000C82202490248FDF709FF10BD44170020CA
:1033400038170020FEB50746002600240CE0385D43
:1033500010B1385D0A2800DD08E0385D0DF8040082
:10336000701CC6B2601CC4B20A2CF0DB00BF06B9E8
:10337000FEBD47490868804700240CE000201DF886
:10338000041001EB410202EB8111424A114481F821
:103390004100601CC4B2B442F0DB3F480078864272
:1033A00003DB00203C4908706CE0012501245FE04C
:1033B00004EB440000EB84103649084490F84100C7
:1033C00000B953E03548C08B401C3449C883022003
:1033D00005EB450101EB85112E4A114481F84100AE
:1033E000AC4202D1681CC5B240E004EB440303EBDD
:1033F0008413DFF8A0C0634493F8402005EB450335
:1034000003EB851303EB0C0104EB440303EB841380
:1034100003EB0C00FCF7ADFA04EB440000EB841066
:103420001C49084490F8400005EB450101EB85116B
:10343000184A114481F8400004EB440000EB84106A
:103440001146084490F8420005EB450101EB851157
:10345000114481F84200002004EB440101EB841187
:10346000114481F84100681CC5B200BF601CC4B2A1
:103470000948007884429BDD07480078801B064994
:10348000087000BF02494868804700BF70E700002D
:10349000B802002044300020FD0300209C070020DB
:1034A000704710B54FF4FA7408E0FBF7C7FB00B1A2
:1034B00010BD6420F7F7FCFD601E84B2002CF4D12F
:1034C00000BFF5E710B51448007800B910BD1349E6
:1034D000486D804738B91248807820B901201049DA
:1034E0008870F8F721FB0E48C07800B9EEE70C4869
:1034F0008088401C80B20A498880C82802DA00F01F
:1035000011F807E000200649C870888008460021AD
:10351000C0F8061000BFD9E744040020480300208B
:10352000145F002010B588B03648007810B13648D6
:10353000C07810B9002008B010BD1C208DF8000024
:10354000324881690DF10100884730208DF805006F
:1035500000208DF806008DF8070014208DF8080073
:1035600004208DF8090013210DF10A00F4F737FE4D
:103570002548C07801283AD1FF208DF806008DF843
:103580000700214890F87F001F4991F87E1088427B
:1035900003DB00201C4981F87F001B4890F87F1056
:1035A000801D10F821008DF80E00174890F87F104C
:1035B000801D00EB810040788DF80F00124890F8D4
:1035C0007F10801D00EB810080788DF810000E4880
:1035D00090F87F10801D00EB8100C0788DF81100FD
:1035E000094890F87F00401C074981F87F0007498F
:1035F000C86A8047044605482146426B68469047A2
:10360000012098E744040020145F002048030020B4
:1036100030B591B004460D46402101A8F4F7DFFD16
:103620003C208DF80400E1208DF805000949C869A7
:1036300080478DF806000E208DF807002A462146A7
:1036400002A8F4F7A5FD0348416C01A8884711B012
:1036500030BD0000480300202DE9F04107464FF639
:10366000FF783846F9F78EFF05461248007828445F
:10367000C82806DC2A4639460E48007800F044F98E
:1036800014E00C480078C0F1C800C6B23246394692
:103690000848007800F038F9344605E00120A040E1
:1036A00028EA0008601CC4B2AC42F7DB4046BDE823
:1036B000F0810000870500202DE9F04106464FF615
:1036C000FF773046F9F75EFF05461E2D00DD1E250B
:1036D0000F4880F87E50002414E006EB8400FEF7CB
:1036E00051FAB0F1000803D10120A040874307E060
:1036F0003046F8F72FFAAA2204214046F4F768FD75
:10370000601C84B2AC42E8DB3846BDE8F0810000C2
:10371000145F002070B590B00446207901280BD0CA
:10372000022804D004281DD0052845D11FE0607967
:10373000A11D00F089F800BF60790DF1020100F0D1
:103740005FF820B928210DF10200F4F748FD0120AF
:103750008DF8000060798DF801002A216846FFF796
:1037600057FF2AE0A01DFFF777FF054604E0A01DE4
:10377000FFF7A2FF054600BF02208DF80000C5F349
:10378000090040F2FF31884201D1012000E0002011
:103790008DF80100002608E045FA06F000F001016E
:1037A000B01C0DF80010701CC6B20A2EF4DB0C2100
:1037B0006846FFF72DFF00E000BF00BF10B070BDEE
:1037C00000210B4A11700B4A1170002006E00A49D3
:1037D00001EB800100220A60411C88B2C828F6DB98
:1037E0000021064AD17091809170118070470000CD
:1037F0008805002087050020F45B0020145F00206E
:103800002DE9F04106460F46142E02DB0020BDE8EC
:10381000F0813046FBF784F9054600240DE04FF6B1
:10382000FF7000EA840807EB08002919054A02EB3B
:10383000810109680160601C84B20A2CEFDB012061
:10384000E5E70000F45B00202DE9F04104460E4658
:10385000142C02DB0020BDE8F0811CB9FFF7B0FF9B
:10386000F8F762F93046F9F78DFE05462046FBF77A
:1038700057F907462A46F8B2314600F045F80120CC
:10388000E9E7000030B589B005461D480378C21C41
:1038900001A92846F5F7B6FC002409E001A8005D5F
:1038A000611C01AA515C4840611C5054601CC4B2A8
:1038B0000F2CF3DB1348102201A9036A90019847EB
:1038C0000F480378C21C01A905F11000F5F79AFC16
:1038D000002409E001A8005D611C01AA515C484078
:1038E000611C5054601CC4B20F2CF3DB054810223D
:1038F00001A9036A4FF48260984709B030BD000007
:103900009C4B0020B802002030B50346002009E09F
:103910001C18084D05EB840401EB80052D6825601B
:10392000441CA0B29042F3DB034C24781444024DB3
:103930002C7030BDF45B00208705002000020000E1
:1039400000040000000000000006000006FFFF0960
:10395000FFA10109FF954075081580257F810009A9
:10396000FF954075081580257F9100C00014014027
:10397000000C014000140140001001400020100024
:1039800008004000001401400014014000140140F0
:103990000010014000402000100080000E050407C8
:1039A00000140140001401400014014000100140C7
:1039B0000008400002001000001401400014014003
:1039C000001401400010014000108000040020009D
:1039D0004053554E564F54450053756E566F74659F
:1039E00031393938264A61636B506569313937326C
:1039F000436F6F6C426F62393900104E13411442AD
:103A000015431644174518461947204A304B404D78
:103A10009151925293539454A05AB05BC05C0000F1
:103A20000100000052096AD53036A538BF40A39E78
:103A300081F3D7FB7CE339829B2FFF87348E43448D
:103A4000C4DEE9CB547B9432A6C2233DEE4C950BE9
:103A500042FAC34E082EA16628D924B2765BA24949
:103A60006D8BD12572F8F66486689816D4A45CCC68
:103A70005D65B6926C704850FDEDB9DA5E1546573B
:103A8000A78D9D8490D8AB008CBCD30AF7E4580571
:103A9000B8B34506D02C1E8FCA3F0F02C1AFBD037D
:103AA00001138A6B3A9111414F67DCEA97F2CFCE4E
:103AB000F0B4E67396AC7422E7AD3585E2F937E8E9
:103AC0001C75DF6E47F11A711D29C5896FB7620E2B
:103AD000AA18BE1BFC563E4BC6D279209ADBC0FE0C
:103AE00078CD5AF41FDDA8338807C731B1121059B9
:103AF0002780EC5F60517FA919B54A0D2DE57A9FAB
:103B000093C99CEFA0E03B4DAE2AF5B0C8EBBB3C9F
:103B100083539961172B047EBA77D626E169146323
:103B200055210C7D637C777BF26B6FC53001672B71
:103B3000FED7AB76CA82C97DFA5947F0ADD4A2AFA1
:103B40009CA472C0B7FD9326363FF7CC34A5E5F1AF
:103B500071D8311504C723C31896059A071280E25D
:103B6000EB27B27509832C1A1B6E5AA0523BD6B3B1
:103B700029E32F8453D100ED20FCB15B6ACBBE3921
:103B80004A4C58CFD0EFAAFB434D338545F9027F0D
:103B9000503C9FA851A3408F929D38F5BCB6DA21C6
:103BA00010FFF3D2CD0C13EC5F974417C4A77E3DF2
:103BB000645D197360814FDC222A908846EEB81448
:103BC000DE5E0BDBE0323A0A4906245CC2D3AC620B
:103BD0009195E479E7C8376D8DD54EA96C56F4EA16
:103BE000657AAE08BA78252E1CA6B4C6E8DD741F27
:103BF0004BBD8B8A703EB5664803F60E613557B9EA
:103C000086C11D9EE1F8981169D98E949B1E87E9A3
:103C1000CE5528DF8CA1890DBFE6426841992D0F52
:103C2000B054BB168D01020408102040801B366C76
:103C3000D8AB4D9A2F5EBC63C697356AD4B37DFA74
:103C4000EFC5913972E4D3BD61C29F254A943366B2
:103C5000CC831D3A74E8CB8D01020408102040800B
:103C60001B366CD8AB4D9A2F5EBC63C697356AD4B1
:103C7000B37DFAEFC5913972E4D3BD61C29F254A85
:103C8000943366CC831D3A74E8CB8D01020408108E
:103C90002040801B366CD8AB4D9A2F5EBC63C69714
:103CA000356AD4B37DFAEFC5913972E4D3BD61C2F0
:103CB0009F254A943366CC831D3A74E8CB8D01026C
:103CC0000408102040801B366CD8AB4D9A2F5EBC88
:103CD00063C697356AD4B37DFAEFC5913972E4D3E0
:103CE000BD61C29F254A943366CC831D3A74E8CBEC
:103CF0008D01020408102040801B366CD8AB4D9A11
:103D00002F5EBC63C697356AD4B37DFAEFC591398F
:103D100072E4D3BD61C29F254A943366CC831D3AB9
:103D200074E8CB0000002110422063308440A5508D
:103D3000C660E770088129914AA16BB18CC1ADD1F1
:103D4000CEE1EFF10000000009000000637C777B0A
:103D5000F26B6FC53001672BFED7AB76CA82C97D87
:103D6000FA5947F0ADD4A2AF9CA472C0B7FD932618
:103D7000363FF7CC34A5E5F171D8311504C723C31C
:103D80001896059A071280E2EB27B27509832C1A60
:103D90001B6E5AA0523BD6B329E32F8453D100EDBA
:103DA00020FCB15B6ACBBE394A4C58CFD0EFAAFB9E
:103DB000434D338545F9027F503C9FA851A3408F66
:103DC000929D38F5BCB6DA2110FFF3D2CD0C13EC7E
:103DD0005F974417C4A77E3D645D197360814FDC13
:103DE000222A908846EEB814DE5E0BDBE0323A0AF7
:103DF0004906245CC2D3AC629195E479E7C8376D7B
:103E00008DD54EA96C56F4EA657AAE08BA78252E9F
:103E10001CA6B4C6E8DD741F4BBD8B8A703EB56628
:103E20004803F60E613557B986C11D9EE1F8981119
:103E300069D98E949B1E87E9CE5528DF8CA1890D08
:103E4000BFE6426841992D0FB054BB1652096AD59E
:103E50003036A538BF40A39E81F3D7FB7CE339827F
:103E60009B2FFF87348E4344C4DEE9CB547B9432CE
:103E7000A6C2233DEE4C950B42FAC34E082EA16616
:103E800028D924B2765BA2496D8BD12572F8F664ED
:103E900086689816D4A45CCC5D65B6926C70485068
:103EA000FDEDB9DA5E154657A78D9D8490D8AB001D
:103EB0008CBCD30AF7E45805B8B34506D02C1E8F46
:103EC000CA3F0F02C1AFBD0301138A6B3A91114182
:103ED0004F67DCEA97F2CFCEF0B4E67396AC74226B
:103EE000E7AD3585E2F937E81C75DF6E47F11A71E9
:103EF0001D29C5896FB7620EAA18BE1BFC563E4B22
:103F0000C6D279209ADBC0FE78CD5AF41FDDA833E3
:103F10008807C731B11210592780EC5F60517FA923
:103F200019B54A0D2DE57A9F93C99CEFA0E03B4D52
:103F3000AE2AF5B0C8EBBB3C83539961172B047EC6
:103F4000BA77D626E169146355210C7D0000000183
:103F50000000000200000004000000080000001043
:103F60000000002000000040000000800000001B56
:103F700000000036A56363C6847C7CF8997777EEF1
:103F80008D7B7BF60DF2F2FFBD6B6BD6B16F6FDEF2
:103F900054C5C5915030306003010102A96767CE56
:103FA0007D2B2B5619FEFEE762D7D7B5E6ABAB4D9E
:103FB0009A7676EC45CACA8F9D82821F40C9C9890C
:103FC000877D7DFA15FAFAEFEB5959B2C947478E4A
:103FD0000BF0F0FBECADAD4167D4D4B3FDA2A25F12
:103FE000EAAFAF45BF9C9C23F7A4A453967272E43A
:103FF0005BC0C09BC2B7B7751CFDFDE1AE93933D9E
:104000006A26264C5A36366C413F3F7E02F7F7F55A
:104010004FCCCC835C343468F4A5A55134E5E5D1AC
:1040200008F1F1F9937171E273D8D8AB5331316271
:104030003F15152A0C04040852C7C795652323466B
:104040005EC3C39D28181830A19696370F05050A40
:10405000B59A9A2F0907070E361212249B80801BEF
:104060003DE2E2DF26EBEBCD6927274ECDB2B27FF2
:104070009F7575EA1B0909129E83831D742C2C58A9
:104080002E1A1A342D1B1B36B26E6EDCEE5A5AB441
:10409000FBA0A05BF65252A44D3B3B7661D6D6B74F
:1040A000CEB3B37D7B2929523EE3E3DD712F2F5E32
:1040B00097848413F55353A668D1D1B9000000004A
:1040C0002CEDEDC1602020401FFCFCE3C8B1B179AC
:1040D000ED5B5BB6BE6A6AD446CBCB8DD9BEBE67FC
:1040E0004B393972DE4A4A94D44C4C98E85858B04F
:1040F0004ACFCF856BD0D0BB2AEFEFC5E5AAAA4F38
:1041000016FBFBEDC5434386D74D4D9A55333366B9
:1041100094858511CF45458A10F9F9E90602020414
:10412000817F7FFEF05050A0443C3C78BA9F9F2591
:10413000E3A8A84BF35151A2FEA3A35DC040408069
:104140008A8F8F05AD92923FBC9D9D214838387073
:1041500004F5F5F1DFBCBC63C1B6B67775DADAAF4A
:1041600063212142301010201AFFFFE50EF3F3FD0A
:104170006DD2D2BF4CCDCD81140C0C183513132643
:104180002FECECC3E15F5FBEA2979735CC44448827
:104190003917172E57C4C493F2A7A755827E7EFC09
:1041A000473D3D7AAC6464C8E75D5DBA2B191932AE
:1041B000957373E6A06060C098818119D14F4F9EBE
:1041C0007FDCDCA3662222447E2A2A54AB90903BFB
:1041D0008388880BCA46468C29EEEEC7D3B8B86BE5
:1041E0003C14142879DEDEA7E25E5EBC1D0B0B16C4
:1041F00076DBDBAD3BE0E0DB563232644E3A3A74BC
:104200001E0A0A14DB4949920A06060C6C2424484B
:10421000E45C5CB85DC2C29F6ED3D3BDEFACAC436F
:10422000A66262C4A8919139A495953137E4E4D38C
:104230008B7979F232E7E7D543C8C88B5937376EA7
:10424000B76D6DDA8C8D8D0164D5D5B1D24E4E9C93
:10425000E0A9A949B46C6CD8FA5656AC07F4F4F34B
:1042600025EAEACFAF6565CA8E7A7AF4E9AEAE4741
:1042700018080810D5BABA6F887878F06F25254AE3
:10428000722E2E5C241C1C38F1A6A657C7B4B4733A
:1042900051C6C69723E8E8CB7CDDDDA19C7474E8A9
:1042A000211F1F3EDD4B4B96DCBDBD61868B8B0D08
:1042B000858A8A0F907070E0423E3E7CC4B5B5712D
:1042C000AA6666CCD84848900503030601F6F6F7BF
:1042D000120E0E1CA36161C25F35356AF95757AEE5
:1042E000D0B9B9699186861758C1C199271D1D3A61
:1042F000B99E9E2738E1E1D913F8F8EBB398982BD3
:1043000033111122BB6969D270D9D9A9898E8E0760
:10431000A7949433B69B9B2D221E1E3C9287871533
:1043200020E9E9C949CECE87FF5555AA78282850FB
:104330007ADFDFA58F8C8C03F8A1A15980898909C8
:10434000170D0D1ADABFBF6531E6E6D7C6424284C3
:10435000B86868D0C3414182B0999929772D2D5A08
:10436000110F0F1ECBB0B07BFC5454A8D6BBBB6D55
:104370003A16162C50A7F4515365417EC3A4171A60
:10438000965E273ACB6BAB3BF1459D1FAB58FAAC21
:104390009303E34B55FA3020F66D76AD9176CC88D9
:1043A000254C02F5FCD7E54FD7CB2AC580443526EE
:1043B0008FA362B5495AB1DE671BBA25980EEA454C
:1043C000E1C0FE5D02752FC312F04C81A397468DAC
:1043D000C6F9D36BE75F8F03959C9215EB7A6DBF9F
:1043E000DA5952952D83BED4D32174582969E049F6
:1043F00044C8C98E6A89C27578798EF46B3E589923
:10440000DD71B927B64FE1BE17AD88F066AC20C9A3
:10441000B43ACE7D184ADF6382311AE56033519792
:10442000457F5362E07764B184AE6BBB1CA081FE14
:10443000942B08F95868487019FD458F876CDE94F5
:10444000B7F87B5223D373ABE2024B72578F1FE353
:104450002AAB55660728EBB203C2B52F9A7BC586F7
:10446000A50837D3F2872830B2A5BF23BA6A030262
:104470005C8216ED2B1CCF8A92B479A7F0F207F379
:10448000A1E2694ECDF4DA65D5BE05061F6234D1CE
:104490008AFEA6C49D532E34A055F3A232E18A05AC
:1044A00075EBF6A439EC830BAAEF6040069F715EB2
:1044B00051106EBDF98A213E3D06DD96AE053EDD0A
:1044C00046BDE64DB58D5491055DC4716FD40604AB
:1044D000FF15506024FB981997E9BDD6CC4340895D
:1044E000779ED967BD42E8B0888B8907385B19E7AA
:1044F000DBEEC879470A7CA1E90F427CC91E84F82B
:10450000000000008386800948ED2B32AC70111E3C
:104510004E725A6CFBFF0EFD5638850F1ED5AE3D10
:1045200027392D3664D90F0A21A65C68D1545B9BCC
:104530003A2E3624B1670A0C0FE75793D296EEB4A1
:104540009E919B1B4FC5C080A220DC61694B775AAE
:10455000161A121C0ABA93E2E52AA0C043E0223CD4
:104560001D171B120B0D090EADC78BF2B9A8B62D86
:10457000C8A91E148519F1574C0775AFBBDD99EE1C
:10458000FD607FA39F2601F7BCF5725CC53B6644C6
:10459000347EFB5B7629438BDCC623CB68FCEDB60F
:1045A00063F1E4B8CADC31D7108563424022971327
:1045B0002011C6847D244A85F83DBBD21132F9AE64
:1045C0006DA129C74B2F9E1DF330B2DCEC52860D36
:1045D000D0E3C1776C16B32B99B970A9FA4894113E
:1045E0002264E947C48CFCA81A3FF0A0D82C7D5661
:1045F000EF903322C74E4987C1D138D9FEA2CA8C69
:10460000360BD498CF81F5A628DE7AA5268EB7DAA8
:10461000A4BFAD3FE49D3A2C0D9278509BCC5F6ACD
:1046200062467E54C2138DF6E8B8D8905EF7392EF4
:10463000F5AFC382BE805D9F7C93D069A92DD56FF5
:10464000B31225CF3B99ACC8A77D18106E639CE8C8
:104650007BBB3BDB097826CDF418596E01B79AEC89
:10466000A89A4F83656E95E67EE6FFAA08CFBC2127
:10467000E6E815EFD99BE7BACE366F4AD4099FEA30
:10468000D67CB029AFB2A43131233F2A3094A5C6DD
:10469000C066A23537BC4E74A6CA82FCB0D090E08A
:1046A00015D8A7334A9804F1F7DAEC410E50CD7FC4
:1046B0002FF691178DD64D764DB0EF43544DAACCC1
:1046C000DF0496E4E3B5D19E1B886A4CB81F2CC169
:1046D0007F51654604EA5E9D5D358C01737487FAEF
:1046E0002E410BFB5A1D67B352D2DB92335610E9B1
:1046F0001347D66D8C61D79A7A0CA1378E14F8596E
:10470000893C13EBEE27A9CE35C961B7EDE51CE175
:104710003CB1477A59DFD29C3F73F25579CE1418D9
:10472000BF37C773EACDF7535BAAFD5F146F3DDF58
:1047300086DB447881F3AFCA3EC468B92C34243890
:104740005F40A3C272C31D160C25E2BC8B493C28F6
:1047500041950DFF7101A839DEB30C089CE4B4D873
:1047600090C156646184CB7B70B632D5745C6C4862
:104770004257B8D00000C201840346020807CA06A7
:104780008C044E05100ED20F940D560C1809DA0841
:104790009C0A5E0B201CE21DA41F661E281BEA1A41
:1047A000AC186E193012F213B41176103815FA14D1
:1047B000BC167E1740388239C43B063A483F8A3ED1
:1047C000CC3C0E3D50369237D435163458319A30A1
:1047D000DC321E336024A225E42726266823AA2281
:1047E000EC202E21702AB22BF4293628782DBA2CF1
:1047F000FC2E3E2F807042710473C67288774A7611
:104800000C74CE75907E527F147DD67C98795A7840
:104810001C7ADE7BA06C626D246FE66EA86B6A6A00
:104820002C68EE69B06272633461F660B8657A64D0
:104830003C66FE67C0480249444B864AC84F0A4E50
:104840004C4C8E4DD046124754459644D8411A40A0
:104850005C429E43E05422556457A656E8532A52C0
:104860006C50AE51F05A325B7459B658F85D3A5CF0
:104870007C5EBE5F00E1C2E084E246E308E6CAE790
:104880008CE54EE410EFD2EE94EC56ED18E8DAE940
:104890009CEB5EEA20FDE2FCA4FE66FF28FAEAFB40
:1048A000ACF96EF830F3F2F2B4F076F138F4FAF5D0
:1048B000BCF77EF640D982D8C4DA06DB48DE8ADF50
:1048C000CCDD0EDC50D792D6D4D416D558D09AD1A0
:1048D000DCD31ED260C5A2C4E4C626C768C2AAC380
:1048E000ECC12EC070CBB2CAF4C836C978CCBACDF0
:1048F000FCCF3ECE809142900492C69388964A9710
:104900000C95CE94909F529E149CD69D98985A993F
:104910001C9BDE9AA08D628C248EE68FA88A6A8BFF
:104920002C89EE88B08372823480F681B8847A85CF
:104930003C87FE86C0A902A844AA86ABC8AE0AAFCF
:104940004CAD8EACD0A712A654A496A5D8A01AA19F
:104950005CA39EA2E0B522B464B6A6B7E8B22AB3BF
:104960006CB1AEB0F0BB32BA74B8B6B9F8BC3ABDEF
:104970007CBFBEBE0000201C403860248070A06C4C
:10498000C048E05400E120FD40D960C58091A08D71
:10499000C0A9E0B500040101000000000000010012
:1049A00004040101040001010404010004000000EA
:1049B00000000100000400000004010104040101E2
:1049C00000040000040400010400010100000001D3
:1049D00004000000040400000004000100040001C1
:1049E00000040100000401000000010100000101B9
:1049F000040400010400010004000001040000019F
:104A00000400010000000000040400000404010090
:104A10000000000100000100040401010400000086
:104A2000000001010004010100000001000000017C
:104A30000004000004000101000001000004010066
:104A40000400000100040000040000000404000150
:104A5000040401000404010104000100000001013C
:104A60000404000104000001040400000404010027
:104A7000000401010404000000040001000400011E
:104A8000000000000400010000040100000000001C
:104A90000400010120801080008000800080000060
:104AA0002080100000001000200000002000108076
:104AB00020800080200000802080108000801080F6
:104AC0000000008000800080000010002000000036
:104AD0002000108000801000200010002080008046
:104AE0000000000000000080008000002080100016
:104AF0000000108020001000200000800000000056
:104B000000801000208000000080108000001080D5
:104B10002080000000000000208010002000108095
:104B200000001000208000800000108000801080B5
:104B30000080000000001080008000802000000045
:104B400020801080208010002000000000800000E5
:104B50000000008020800000008010800000100015
:104B600020000080200010002080008020000080B5
:104B70002000100000801000000000000080008075
:104B80002080000000000080200010802080108025
:104B9000008010000802000000020208000000006F
:104BA00008000208000200080000000008020200DD
:104BB00000020008080002000800000808000008C1
:104BC00000000200080202080800020000000208BB
:104BD00008020000000000080800000000020208AF
:104BE00000020000000202000000020808000208A3
:104BF0000802020008020008000202000000020091
:104C00000802000808000000080202080002000074
:104C1000000000080002020800000008080002006E
:104C20000802000000000200000202080002000862
:104C30000000000000020000080002000802020854
:104C40000002000808000008000200000000000048
:104C50000800020808020008000002000000000826
:104C60000802020808000000080202000002020018
:104C700008000008000002080802000808020000FE
:104C800000000208080202000800000008000208F4
:104C9000000202000120800081200000812000002D
:104CA00080000000802080008100800001008000E2
:104CB0000120000000000000002080000020800093
:104CC0008120800081000000000000008000800042
:104CD00001008000010000000020000000008000B2
:104CE0000120800080000000000080000120000002
:104CF0008020000081008000010000008020000072
:104D00008000800000200000802080008120800042
:104D100081000000800080000100800000208000F1
:104D200081208000810000000000000000000000E1
:104D30000020800080200000800080008100800032
:104D4000010000000120800081200000812000007F
:104D50008000000081208000810000000100000030
:104D60000020000001008000012000008020800061
:104D700081008000012000008020000000008000F1
:104D80000120800080000000000080000020000062
:104D900080208000000100000001080200000802DD
:104DA0000001004200000800000100000000004077
:104DB0000000080200010840000008000001000295
:104DC0000001084000010042000008420001080004
:104DD0000000004000000002000008400000084001
:104DE00000000000000100400001084200010842EC
:104DF0000001000200000842000100400000000025
:104E00000000004200010802000000020000004211
:104E1000000108000000080000010042000100003D
:104E200000000002000000400000080200010042F3
:104E3000000108400001000200000040000008429C
:104E4000000108020001084000010000000000020B
:104E50000000084200010842000108000000004272
:104E600000010842000008020000000000000840A5
:104E700000000042000108000001000200010040A3
:104E800000000800000000000000084000010802C7
:104E90000001004010000020000040200040000001
:104EA0001040402000004020100000001040402032
:104EB0000000400000400020104040000000400082
:104EC00010000020100040000040002000000020E2
:104ED00010400000000000001000400010400020C2
:104EE0000040000000404000104000201000000082
:104EF0001000402010004020000000001040400042
:104F00000040402010400000004040000040402091
:104F10000000002000400020100000001000402091
:104F200000404000104040200000400010400000C1
:104F30001000002000004000004000200000002081
:104F400010400000100000201040402000404000B1
:104F500000004020104040000040402000000000C1
:104F60001000402010000000004000000000402021
:104F700010404000004000001000400010400020A1
:104F80000000000000404020000000201000400011
:104F9000104000200000200002002004020800044D
:104FA00000000000000800000208000402082000C1
:104FB0000008200402082004000020000000000077
:104FC00002000004020000000000000402002004AF
:104FD000020800000008000402082000020020006F
:104FE000000800040200000400002004000820045F
:104FF0000200200000002004000800000208000059
:105000000208200400082000020000000000000444
:10501000000820000000000400082000000020001C
:105020000208000402080004020020040200200418
:10503000020000000200200000000004000800043C
:1050400000002000000820040208000002082000E0
:1050500000082004020800000200000402082004E6
:1050600000002004000820000000000002000000F2
:1050700002082004000000000208200000002004B4
:1050800000080000020000040008000400080000FE
:10509000020020004010001000100000000004007A
:1050A00040100410000000104010001040000000EC
:1050B0000000001040000400000004104010041024
:1050C0000010040000100410401004000010000044
:1050D000400000000000041040000010001000100C
:1050E00040100000001004004000040040000410C4
:1050F000001004104010000000000000000000003C
:105100004000041040000010001000104010040087
:10511000000004004010040000000400001004100F
:1051200000100000400000004000041000100000CB
:10513000401004000010001040000000400000106B
:1051400000000410400004100000001000000400E3
:105150004010001000000000401004104000040047
:10516000400000100000041000100010401000105B
:1051700000000000401004100010040000100400A3
:10518000401000004010000040000400000000102B
:1051900000100410982F8A4291443771CFFBC0B59C
:1051A000A5DBB5E95BC25639F111F159A4823F92F2
:1051B000D55E1CAB98AA07D8015B8312BE8531244B
:1051C000C37D0C55745DBE72FEB1DE80A706DC9B0C
:1051D00074F19BC1C1699BE48647BEEFC69DC10FB8
:1051E000CCA10C246F2CE92DAA84744ADCA9B05CF4
:1051F000DA88F97652513E986DC631A8C82703B0B7
:10520000C77F59BFF30BE0C64791A7D55163CA06C4
:1052100067292914850AB72738211B2EFC6D2C4DD0
:10522000130D385354730A65BB0A6A762EC9C281BE
:10523000852C7292A1E8BFA24B661AA8708B4BC254
:10524000A3516CC719E892D1240699D685350EF47E
:1052500070A06A1016C1A419086C371E4C77482735
:10526000B5BCB034B30C1C394AAAD84E4FCA9C5BAB
:10527000F36F2E68EE828F746F63A5781478C884FC
:105280000802C78CFAFFBE90EB6C50A4F7A3F9BEDE
:10529000F27871C60000000022AE28D7982F8A420B
:1052A000CD65EF23914437712F3B4DECCFFBC0B55B
:1052B000BCDB8981A5DBB5E938B548F35BC256395B
:1052C00019D005B6F111F1599B4F19AFA4823F9245
:1052D00018816DDAD55E1CAB420203A398AA07D8E9
:1052E000BE6F7045015B83128CB2E44EBE853124E3
:1052F000E2B4FFD5C37D0C556F897BF2745DBE723D
:10530000B196163BFEB1DE803512C725A706DC9BA1
:10531000942669CF74F19BC1D24AF19EC1699BE486
:10532000E3254F388647BEEFB5D58C8BC69DC10FA0
:10533000659CAC77CCA10C2475022B596F2CE92D00
:1053400083E4A66EAA84744AD4FB41BDDCA9B05C98
:10535000B5531183DA88F976ABDF66EE52513E9889
:105360001032B42D6DC631A83F21FB98C82703B079
:10537000E40EEFBEC77F59BFC28FA83DF30BE0C656
:1053800025A70A934791A7D56F8203E05163CA0608
:10539000706E0E0A67292914FC2FD246850AB7279A
:1053A00026C9265C38211B2EED2AC45AFC6D2C4DD3
:1053B000DFB3959D130D3853DE63AF8B54730A65CD
:1053C000A8B2773CBB0A6A76E6AEED472EC9C28129
:1053D0003B358214852C72926403F14CA1E8BFA284
:1053E000013042BC4B661AA89197F8D0708B4BC223
:1053F00030BE5406A3516CC71852EFD619E892D1AB
:1054000010A96555240699D62A20715785350EF4C2
:10541000B8D1BB3270A06A10C8D0D2B816C1A419D6
:1054200053AB4151086C371E99EB8EDF4C77482700
:10543000A8489BE1B5BCB034635AC9C5B30C1C394C
:10544000CB8A41E34AAAD84E73E363774FCA9C5B89
:10545000A3B8B2D6F36F2E68FCB2EF5DEE828F7404
:10546000602F17436F63A57872ABF0A11478C884DE
:10547000EC39641A0802C78C281E6323FAFFBE9019
:10548000E9BD82DEEB6C50A41579C6B2F7A3F9BE74
:105490002B5372E3F27871C69C6126EACE3E27CA8E
:1054A00007C2C021C7B886D11EEBE0CDD67DDAEAAF
:1054B00078D16EEE7F4F7DF5BA6F1772AA67F0064E
:1054C000A698C8A2C57D630AAE0DF9BE04983F1127
:1054D0001B471C13350B711B847D0423F577DB28D8
:1054E0009324C7407BABCA32BCBEC9150ABE9E3CE2
:1054F0004C0D109CC4671D43B6423ECBBED4C54C78
:105500002A7E65FC9C297F59ECFAD63AAB6FCB5FBB
:105510001758474A8C19446C657870616E64203363
:10552000322D62797465206B657870616E6420310C
:10553000362D62797465206BEDD3F55C1A631258D1
:10554000D69CF7A2DEF9DE14000000000000000087
:1055500000000000000000101B132C0AA3E59CEDC6
:10556000A72963085D210621EBFFFFFFFFFFFFFF77
:10557000FFFFFFFFFFFFFFFF0F000000A37859139D
:10558000CA4DEB75ABD841414D0A700098E8797768
:105590007940C78C73FE6F2BEE6C03521AD5258FA2
:1055A000602D56C9B2A7259560C72C695CDCD6FD75
:1055B00031E2A4C0FE536ECDD336692158666666CB
:1055C000666666666666666666666666666666667B
:1055D0006666666666666666666666660100000002
:1055E00000000000000000000000000000000000BB
:1055F000000000000000000000000000A3DDB7A5CF
:10560000B38ADE6DF5525177809FF0207DE3AB6465
:105610008E4EEA6665768BD70F5F876759F1B226A3
:10562000949BD6EB56B183829A14E00030D1F3EE0E
:10563000F2808E19E7FCDF56DCD90624B0A00E4AB2
:10564000271BEEC478E42FAD0618432FA7D7FB3DE8
:1056500099004D2B0BDFC14F8024832B800040002D
:10566000200010000800040002000100000080007B
:1056700000004000000020000000100000000800B2
:105680000000040000000200000001000080000093
:105690000040000000200000001000000008000092
:1056A0000004000000020000000100008000000073
:1056B0004000000020000000100000000800000072
:1056C0000400000002000000010000008000000053
:1056D00000000000000000000000000000000000CA
:1056E00000000000000000000000000000000000BA
:1056F00000000000000000000000000000000000AA
:105700000000000000000000000000000000000099
:1057100000000000000000000000000063636362FE
:10572000636363626363636263636362C998989B44
:10573000AAFBFBF9C998989BAAFBFBF950349790F8
:10574000FACF6C693357F4F299AC0F0B7BDA06EEA3
:1057500081156A87B2429E752BEE917E882B2E7F33
:10576000093E44F8BB7CDA8D90924BF3854B61EC9B
:105770008C7525143709FF99A79BB46A8717752183
:105780000B6250353C6BAFAC9BF01BC63303F90E7C
:105790003861A93B040A06979FFA1D51E2D8D4B19B
:1057A000DAB97D8ADEB37B1D4149664CCB5BEFB431
:1057B00011E2923ECF51E9238E188F6F0302010050
:1057C000070605040B0A09080F0E0D0CFD74AAD676
:1057D000FA72AFD2F178A6DAFE76ABD60BCF92B6DC
:1057E000F1BD3D6400C59BBEFEB330684E74FFB68C
:1057F000BFC9C2D2BF0C596C41BF6904BCF7F7479F
:10580000033E3595BC326CF9FD8D05FDE8A3AA3C3D
:10581000EB9D9FA957AFF350AA22F6AD7D0F395EDD
:105820009692A6F7C13D55A76B1FA30A1A70F914EB
:105830008CE25FE34DDF0A4426C0A94E358743471B
:10584000B9651CA4F4BA16E0D27ABFAED13299542D
:10585000685785F09CED93104E972CBE7F1D111359
:10586000174A94E38BA707F3C5302B4D00000000C7
:105870000000000001000000FFFFFFFF010000002A
:10588000FFFFFFFF0000000000000000000000001C
:105890000000000000000000010000000000000007
:1058A000010000000100000001000000CC580108C8
:1058B000000000209C060000348200081C5C0108E7
:1058C0009C060020DCE50000DEB00008131FF01489
:1058D00008F5F79208840E27071E052401082D04F9
:1058E0001A4504180ED12301083D2F0108E52E01A9
:1058F000080108180B91260108AD2701087D252411
:1059000019081A09081A69281F052B0108252A1CDD
:1059100019084113DDB51408D5B31408A5B64C0811
:1059200083B7081AAB04138DB41B087D101A5108F5
:105930001AD9101A9D281AF3101B23B82812B21B6B
:105940000863041A290C4113120132021640702F09
:1059500010EA1009020102030109022913010125BD
:10596000C032090433020315092111011401222058
:105970001607058103402D010705010710080403E0
:1059800009041003531255124E1256124F125402AC
:105990007345140C034312311A3002027742038319
:1059A0001A0322DF1B20E3041365011B20E7041AFE
:1059B000A40C1AB60441136C023320FF13D9D71B71
:1059C00008BD041385D882081A71101A7504C11312
:1059D000CF8F1408E99F1408C19E1408F19214088F
:1059E0006DD3140809EC1B08D90C1A4908137191DE
:1059F0001B082904780C91180108451B0108B91AE5
:105A000001401EF11901080914811395F71B08C5FF
:105A100004411311BA1B08A14C0114180AE5210115
:105A200008211D01083D608FA3340108C51F4413E0
:105A300081EA1C08FDC17412C21B08A5081A1104D2
:105A40001AA10413D1E91B08AD042AB9041A1034B1
:105A500019081315EB1B0869441ABD8413A9C91B47
:105A6000080D3C13B1F61C0899CE24290C1D0F011A
:105A70000819081ADD281AE9041AF504811AC9540C
:105A80001AF1041A55680132021D0113283323202C
:105A9000031404BDE68C08F7F76013ADE11C087928
:105AA000E20412DF1B0851084113DDE31B08C9049F
:105AB0001AB104411EC137010815042A85D412C049
:105AC000140849F32A086E131DE41B0895041BD122
:105AD000E5DC19041A51041AC504291C180A4922C4
:105AE00001083523010865341A450C1A370C2918AA
:105AF00013F5D11B08D9041AC5044BF5D22C138514
:105B0000BB1408E9FA1408EDF91408D26434090149
:105B1000505AFFD01907E32902133DB81F0825107A
:105B20000108C9081A7104100BF9160108BD150106
:105B3000087DE91B0891040110294A13B5D3180CFC
:105B4000081D1E0108E10F010805DAB41D2F010828
:105B50007B041A7D041A7F041A79041359B11408BE
:105B600021FD1F08650601084D041B49071419088B
:105B70001A59081A21081A11081A41081A3108017D
:105B80001259B0012F323C233F12280D43313030DF
:105B900042414243444546474BF26413C4052A2020
:105BA00004811AD7AC135DDD14089DEA1B08C9D027
:105BB0008BE5D6F81AF02829040114130C062A20C4
:105BC0000481131DB21F08410201089104177D01D1
:105BD0000108D1C28C086DC44C415280599DE03AF5
:105BE00048494A4B4C4D4E4F5051525354555657BD
:105BF00058595A6162636465666768696A6B6C6D5F
:105C00006E6F707172737475767778797A3031321D
:0C5C1000333435363738392B2F000000B4
:04000005080081313D
:00000001FF
